
 Start         Length     Name                   Class
 0001:00401000 00034728H .text                   CODE
 0002:00436000 0000029CH .itext                  ICODE
 0003:00437000 000000E8H .data                   DATA
 0004:00438000 00000080H .bss                    BSS
 0005:00000000 00000000H .tls                    TLS


Detailed map of segments

 0001:00000000 0000021E C=CODE     S=.text    G=(none)   M=System   ACBP=A9
 0001:00000220 000001C3 C=CODE     S=.text    G=(none)   M=SysInit  ACBP=A9
 0001:000003E4 000001B0 C=CODE     S=.text    G=(none)   M=Windows  ACBP=A9
 0001:00000594 00000176 C=CODE     S=.text    G=(none)   M=Classes  ACBP=A9
 0001:0000070C 00000006 C=CODE     S=.text    G=(none)   M=TypInfo  ACBP=A9
 0001:00000714 0000010E C=CODE     S=.text    G=(none)   M=SysUtils ACBP=A9
 0001:00000824 0000000E C=CODE     S=.text    G=(none)   M=Variants ACBP=A9
 0001:00000834 00000006 C=CODE     S=.text    G=(none)   M=VarUtils ACBP=A9
 0001:0000083C 000000AE C=CODE     S=.text    G=(none)   M=ovccmbx  ACBP=A9
 0001:000008EC 00000006 C=CODE     S=.text    G=(none)   M=Menus    ACBP=A9
 0001:000008F4 00000006 C=CODE     S=.text    G=(none)   M=ActnList ACBP=A9
 0001:000008FC 0000001E C=CODE     S=.text    G=(none)   M=ImgList  ACBP=A9
 0001:0000091C 0000010E C=CODE     S=.text    G=(none)   M=Graphics ACBP=A9
 0001:00000A2C 00000006 C=CODE     S=.text    G=(none)   M=Registry ACBP=A9
 0001:00000A34 00000006 C=CODE     S=.text    G=(none)   M=IniFiles ACBP=A9
 0001:00000A3C 00000006 C=CODE     S=.text    G=(none)   M=Themes   ACBP=A9
 0001:00000A44 0000045E C=CODE     S=.text    G=(none)   M=Controls ACBP=A9
 0001:00000EA4 00000006 C=CODE     S=.text    G=(none)   M=UxTheme  ACBP=A9
 0001:00000EAC 00000006 C=CODE     S=.text    G=(none)   M=MultiMon ACBP=A9
 0001:00000EB4 00000006 C=CODE     S=.text    G=(none)   M=DwmApi   ACBP=A9
 0001:00000EBC 0000015E C=CODE     S=.text    G=(none)   M=Forms    ACBP=A9
 0001:0000101C 00000006 C=CODE     S=.text    G=(none)   M=HelpIntfs ACBP=A9
 0001:00001024 00000016 C=CODE     S=.text    G=(none)   M=Dialogs  ACBP=A9
 0001:0000103C 000001EE C=CODE     S=.text    G=(none)   M=StdCtrls ACBP=A9
 0001:0000122C 00000006 C=CODE     S=.text    G=(none)   M=Printers ACBP=A9
 0001:00001234 00000006 C=CODE     S=.text    G=(none)   M=ExtCtrls ACBP=A9
 0001:0000123C 00000006 C=CODE     S=.text    G=(none)   M=GraphUtil ACBP=A9
 0001:00001244 00000006 C=CODE     S=.text    G=(none)   M=Clipbrd  ACBP=A9
 0001:0000124C 00000006 C=CODE     S=.text    G=(none)   M=FlatSB   ACBP=A9
 0001:00001254 00000006 C=CODE     S=.text    G=(none)   M=ovcexcpt ACBP=A9
 0001:0000125C 00000016 C=CODE     S=.text    G=(none)   M=ovcintl  ACBP=A9
 0001:00001274 00000026 C=CODE     S=.text    G=(none)   M=ovcdate  ACBP=A9
 0001:0000129C 00000006 C=CODE     S=.text    G=(none)   M=ovcstr   ACBP=A9
 0001:000012A4 0000000E C=CODE     S=.text    G=(none)   M=ovcdata  ACBP=A9
 0001:000012B4 00000006 C=CODE     S=.text    G=(none)   M=o32sr    ACBP=A9
 0001:000012BC 0000003E C=CODE     S=.text    G=(none)   M=ovceditf ACBP=A9
 0001:000012FC 00000026 C=CODE     S=.text    G=(none)   M=ovcmisc  ACBP=A9
 0001:00001324 0000000E C=CODE     S=.text    G=(none)   M=Buttons  ACBP=A9
 0001:00001334 000000EE C=CODE     S=.text    G=(none)   M=ovcbase  ACBP=A9
 0001:00001424 0000000E C=CODE     S=.text    G=(none)   M=ovccmd   ACBP=A9
 0001:00001434 000001D6 C=CODE     S=.text    G=(none)   M=ovcef    ACBP=A9
 0001:0000160C 00000046 C=CODE     S=.text    G=(none)   M=ovcedpop ACBP=A9
 0001:00001654 00000006 C=CODE     S=.text    G=(none)   M=ovccalc  ACBP=A9
 0001:0000165C 0000006E C=CODE     S=.text    G=(none)   M=ovcedclc ACBP=A9
 0001:000016CC 00000006 C=CODE     S=.text    G=(none)   M=ovcuser  ACBP=A9
 0001:000016D4 00000016 C=CODE     S=.text    G=(none)   M=ovccolor ACBP=A9
 0001:000016EC 00000006 C=CODE     S=.text    G=(none)   M=ovccaret ACBP=A9
 0001:000016F4 0000019E C=CODE     S=.text    G=(none)   M=DB       ACBP=A9
 0001:00001894 00000006 C=CODE     S=.text    G=(none)   M=WideStrings ACBP=A9
 0001:0000189C 00000006 C=CODE     S=.text    G=(none)   M=FMTBcd   ACBP=A9
 0001:000018A4 00000006 C=CODE     S=.text    G=(none)   M=SqlTimSt ACBP=A9
 0001:000018AC 00000006 C=CODE     S=.text    G=(none)   M=ComObj   ACBP=A9
 0001:000018B4 000003A6 C=CODE     S=.text    G=(none)   M=ovcdbhll ACBP=A9
 0001:00001C5C 00000A0E C=CODE     S=.text    G=(none)   M=ovcdbtcb ACBP=A9
 0001:0000266C 00000B22 C=CODE     S=.text    G=(none)   M=ovcdbacb ACBP=A9
 0001:00003190 00000016 C=CODE     S=.text    G=(none)   M=DBTables ACBP=A9
 0001:000031A8 00000026 C=CODE     S=.text    G=(none)   M=ovcdlg   ACBP=A9
 0001:000031D0 00000C96 C=CODE     S=.text    G=(none)   M=ovcdbadg ACBP=A9
 0001:00003E68 00000036 C=CODE     S=.text    G=(none)   M=DBCtrls  ACBP=A9
 0001:00003EA0 00000006 C=CODE     S=.text    G=(none)   M=ComCtrls ACBP=A9
 0001:00003EA8 00000006 C=CODE     S=.text    G=(none)   M=ExtActns ACBP=A9
 0001:00003EB0 00000006 C=CODE     S=.text    G=(none)   M=ExtDlgs  ACBP=A9
 0001:00003EB8 00000006 C=CODE     S=.text    G=(none)   M=Mapi     ACBP=A9
 0001:00003EC0 00000006 C=CODE     S=.text    G=(none)   M=DBPWDlg  ACBP=A9
 0001:00003EC8 00000006 C=CODE     S=.text    G=(none)   M=DBLogDlg ACBP=A9
 0001:00003ED0 00000086 C=CODE     S=.text    G=(none)   M=ovcnf    ACBP=A9
 0001:00003F58 00000066 C=CODE     S=.text    G=(none)   M=ovcpb    ACBP=A9
 0001:00003FC0 00001F8E C=CODE     S=.text    G=(none)   M=ovcdbnf  ACBP=A9
 0001:00005F50 00000056 C=CODE     S=.text    G=(none)   M=ovcpf    ACBP=A9
 0001:00005FA8 00002ACE C=CODE     S=.text    G=(none)   M=ovcdbpf  ACBP=A9
 0001:00008A78 0000004E C=CODE     S=.text    G=(none)   M=ovcsf    ACBP=A9
 0001:00008AC8 00002336 C=CODE     S=.text    G=(none)   M=ovcdbsf  ACBP=A9
 0001:0000AE00 0000603E C=CODE     S=.text    G=(none)   M=ovcdbae  ACBP=A9
 0001:00010E40 00000096 C=CODE     S=.text    G=(none)   M=ovccal   ACBP=A9
 0001:00010ED8 00000FB2 C=CODE     S=.text    G=(none)   M=ovcdbcal ACBP=A9
 0001:00011E8C 0000002E C=CODE     S=.text    G=(none)   M=ovcclrcb ACBP=A9
 0001:00011EBC 00000DA2 C=CODE     S=.text    G=(none)   M=ovcdbccb ACBP=A9
 0001:00012C60 00002AA2 C=CODE     S=.text    G=(none)   M=ovcdbcl  ACBP=A9
 0001:00015704 0000004E C=CODE     S=.text    G=(none)   M=ovcclock ACBP=A9
 0001:00015754 0000097E C=CODE     S=.text    G=(none)   M=ovcdbclk ACBP=A9
 0001:000160D4 000000CE C=CODE     S=.text    G=(none)   M=ovcedcal ACBP=A9
 0001:000161A4 00001A6E C=CODE     S=.text    G=(none)   M=ovcdbdat ACBP=A9
 0001:00017C14 0000006E C=CODE     S=.text    G=(none)   M=ovcrlbl  ACBP=A9
 0001:00017C84 000008CE C=CODE     S=.text    G=(none)   M=ovcdbdLb ACBP=A9
 0001:00018554 00000216 C=CODE     S=.text    G=(none)   M=ovcedit  ACBP=A9
 0001:0001876C 00000006 C=CODE     S=.text    G=(none)   M=ovcfxfnt ACBP=A9
 0001:00018774 0000187A C=CODE     S=.text    G=(none)   M=ovcdbed  ACBP=A9
 0001:00019FF0 00000EF2 C=CODE     S=.text    G=(none)   M=ovcdbfcb ACBP=A9
 0001:0001AEE4 00001C72 C=CODE     S=.text    G=(none)   M=ovcdbidx ACBP=A9
 0001:0001CB58 00000026 C=CODE     S=.text    G=(none)   M=ovciseb  ACBP=A9
 0001:0001CB80 00001172 C=CODE     S=.text    G=(none)   M=ovcdbise ACBP=A9
 0001:0001DCF4 0000092E C=CODE     S=.text    G=(none)   M=ovcdbmdg ACBP=A9
 0001:0001E624 00001622 C=CODE     S=.text    G=(none)   M=ovcdbnum ACBP=A9
 0001:0001FC48 0000006E C=CODE     S=.text    G=(none)   M=ovcplb   ACBP=A9
 0001:0001FCB8 00000C56 C=CODE     S=.text    G=(none)   M=ovcdbplb ACBP=A9
 0001:00020910 0000004E C=CODE     S=.text    G=(none)   M=ovcrvidx ACBP=A9
 0001:00020960 0000001E C=CODE     S=.text    G=(none)   M=ovcdlm   ACBP=A9
 0001:00020980 00000006 C=CODE     S=.text    G=(none)   M=ovcrvexpdef ACBP=A9
 0001:00020988 000002BE C=CODE     S=.text    G=(none)   M=ovcrptvw ACBP=A9
 0001:00020C48 0000006E C=CODE     S=.text    G=(none)   M=ovcvlb   ACBP=A9
 0001:00020CB8 00002ADA C=CODE     S=.text    G=(none)   M=ovcdbrpv ACBP=A9
 0001:00023794 0000008E C=CODE     S=.text    G=(none)   M=ovcedsld ACBP=A9
 0001:00023824 00000076 C=CODE     S=.text    G=(none)   M=ovcslide ACBP=A9
 0001:0002389C 0000165E C=CODE     S=.text    G=(none)   M=ovcdbsed ACBP=A9
 0001:00024EFC 00000C2A C=CODE     S=.text    G=(none)   M=ovcdbsld ACBP=A9
 0001:00025B28 00000016 C=CODE     S=.text    G=(none)   M=ovctcbef ACBP=A9
 0001:00025B40 00000006 C=CODE     S=.text    G=(none)   M=ovctcstr ACBP=A9
 0001:00025B48 00000026 C=CODE     S=.text    G=(none)   M=ovctcell ACBP=A9
 0001:00025B70 00000056 C=CODE     S=.text    G=(none)   M=ovctcmmn ACBP=A9
 0001:00025BC8 00000096 C=CODE     S=.text    G=(none)   M=ovctbcls ACBP=A9
 0001:00025C60 00000006 C=CODE     S=.text    G=(none)   M=ovctbclr ACBP=A9
 0001:00025C68 0000000E C=CODE     S=.text    G=(none)   M=ovctgpns ACBP=A9
 0001:00025C78 00000006 C=CODE     S=.text    G=(none)   M=ovctchdr ACBP=A9
 0001:00025C80 00000006 C=CODE     S=.text    G=(none)   M=ovctgres ACBP=A9
 0001:00025C88 0000000E C=CODE     S=.text    G=(none)   M=ovctcedt ACBP=A9
 0001:00025C98 00000006 C=CODE     S=.text    G=(none)   M=ovctcnum ACBP=A9
 0001:00025CA0 0000001E C=CODE     S=.text    G=(none)   M=ovctcpic ACBP=A9
 0001:00025CC0 00000006 C=CODE     S=.text    G=(none)   M=ovctcsim ACBP=A9
 0001:00025CC8 0000ABBE C=CODE     S=.text    G=(none)   M=ovcdbtbl ACBP=A9
 0001:00030888 00000036 C=CODE     S=.text    G=(none)   M=ovcedtim ACBP=A9
 0001:000308C0 00001866 C=CODE     S=.text    G=(none)   M=ovcdbtim ACBP=A9
 0001:00032128 000000C6 C=CODE     S=.text    G=(none)   M=o32flxed ACBP=A9
 0001:000321F0 00000006 C=CODE     S=.text    G=(none)   M=o32rxvld ACBP=A9
 0001:000321F8 00000006 C=CODE     S=.text    G=(none)   M=o32vlreg ACBP=A9
 0001:00032200 00000006 C=CODE     S=.text    G=(none)   M=o32pvldr ACBP=A9
 0001:00032208 00000006 C=CODE     S=.text    G=(none)   M=o32ovldr ACBP=A9
 0001:00032210 00000016 C=CODE     S=.text    G=(none)   M=o32editf ACBP=A9
 0001:00032228 00000006 C=CODE     S=.text    G=(none)   M=OvcUtils ACBP=A9
 0001:00032230 00001E6E C=CODE     S=.text    G=(none)   M=o32dbfe  ACBP=A9
 0001:000340A0 00000687 C=CODE     S=.text    G=(none)   M=.O406br2005 ACBP=A9
 0002:00000000 00000006 C=ICODE    S=.itext   G=(none)   M=System   ACBP=A9
 0002:00000008 00000011 C=ICODE    S=.itext   G=(none)   M=Windows  ACBP=A9
 0002:0000001C 00000006 C=ICODE    S=.itext   G=(none)   M=Classes  ACBP=A9
 0002:00000024 00000006 C=ICODE    S=.itext   G=(none)   M=TypInfo  ACBP=A9
 0002:0000002C 00000006 C=ICODE    S=.itext   G=(none)   M=SysUtils ACBP=A9
 0002:00000034 00000006 C=ICODE    S=.itext   G=(none)   M=Variants ACBP=A9
 0002:0000003C 00000006 C=ICODE    S=.itext   G=(none)   M=VarUtils ACBP=A9
 0002:00000044 00000006 C=ICODE    S=.itext   G=(none)   M=Menus    ACBP=A9
 0002:0000004C 00000006 C=ICODE    S=.itext   G=(none)   M=ActnList ACBP=A9
 0002:00000054 00000006 C=ICODE    S=.itext   G=(none)   M=Graphics ACBP=A9
 0002:0000005C 00000006 C=ICODE    S=.itext   G=(none)   M=Registry ACBP=A9
 0002:00000064 00000006 C=ICODE    S=.itext   G=(none)   M=IniFiles ACBP=A9
 0002:0000006C 00000006 C=ICODE    S=.itext   G=(none)   M=Themes   ACBP=A9
 0002:00000074 00000006 C=ICODE    S=.itext   G=(none)   M=Controls ACBP=A9
 0002:0000007C 00000006 C=ICODE    S=.itext   G=(none)   M=UxTheme  ACBP=A9
 0002:00000084 00000006 C=ICODE    S=.itext   G=(none)   M=MultiMon ACBP=A9
 0002:0000008C 00000006 C=ICODE    S=.itext   G=(none)   M=DwmApi   ACBP=A9
 0002:00000094 00000006 C=ICODE    S=.itext   G=(none)   M=Forms    ACBP=A9
 0002:0000009C 00000006 C=ICODE    S=.itext   G=(none)   M=HelpIntfs ACBP=A9
 0002:000000A4 00000006 C=ICODE    S=.itext   G=(none)   M=Dialogs  ACBP=A9
 0002:000000AC 00000006 C=ICODE    S=.itext   G=(none)   M=Printers ACBP=A9
 0002:000000B4 00000006 C=ICODE    S=.itext   G=(none)   M=ExtCtrls ACBP=A9
 0002:000000BC 00000006 C=ICODE    S=.itext   G=(none)   M=GraphUtil ACBP=A9
 0002:000000C4 00000006 C=ICODE    S=.itext   G=(none)   M=Clipbrd  ACBP=A9
 0002:000000CC 00000006 C=ICODE    S=.itext   G=(none)   M=FlatSB   ACBP=A9
 0002:000000D4 00000006 C=ICODE    S=.itext   G=(none)   M=ovcintl  ACBP=A9
 0002:000000DC 00000006 C=ICODE    S=.itext   G=(none)   M=ovcdate  ACBP=A9
 0002:000000E4 00000006 C=ICODE    S=.itext   G=(none)   M=ovcdata  ACBP=A9
 0002:000000EC 00000006 C=ICODE    S=.itext   G=(none)   M=o32sr    ACBP=A9
 0002:000000F4 00000006 C=ICODE    S=.itext   G=(none)   M=Buttons  ACBP=A9
 0002:000000FC 00000006 C=ICODE    S=.itext   G=(none)   M=ovcbase  ACBP=A9
 0002:00000104 00000006 C=ICODE    S=.itext   G=(none)   M=ovccalc  ACBP=A9
 0002:0000010C 00000006 C=ICODE    S=.itext   G=(none)   M=ovcuser  ACBP=A9
 0002:00000114 00000006 C=ICODE    S=.itext   G=(none)   M=DB       ACBP=A9
 0002:0000011C 00000006 C=ICODE    S=.itext   G=(none)   M=WideStrings ACBP=A9
 0002:00000124 00000006 C=ICODE    S=.itext   G=(none)   M=FMTBcd   ACBP=A9
 0002:0000012C 00000006 C=ICODE    S=.itext   G=(none)   M=SqlTimSt ACBP=A9
 0002:00000134 00000006 C=ICODE    S=.itext   G=(none)   M=ComObj   ACBP=A9
 0002:0000013C 00000008 C=ICODE    S=.itext   G=(none)   M=ovcdbhll ACBP=A9
 0002:00000144 00000008 C=ICODE    S=.itext   G=(none)   M=ovcdbtcb ACBP=A9
 0002:0000014C 00000008 C=ICODE    S=.itext   G=(none)   M=ovcdbacb ACBP=A9
 0002:00000154 00000006 C=ICODE    S=.itext   G=(none)   M=DBTables ACBP=A9
 0002:0000015C 00000008 C=ICODE    S=.itext   G=(none)   M=ovcdbadg ACBP=A9
 0002:00000164 00000006 C=ICODE    S=.itext   G=(none)   M=DBCtrls  ACBP=A9
 0002:0000016C 00000006 C=ICODE    S=.itext   G=(none)   M=ComCtrls ACBP=A9
 0002:00000174 00000006 C=ICODE    S=.itext   G=(none)   M=ExtActns ACBP=A9
 0002:0000017C 00000006 C=ICODE    S=.itext   G=(none)   M=ExtDlgs  ACBP=A9
 0002:00000184 00000006 C=ICODE    S=.itext   G=(none)   M=Mapi     ACBP=A9
 0002:0000018C 00000006 C=ICODE    S=.itext   G=(none)   M=DBPWDlg  ACBP=A9
 0002:00000194 00000006 C=ICODE    S=.itext   G=(none)   M=DBLogDlg ACBP=A9
 0002:0000019C 00000008 C=ICODE    S=.itext   G=(none)   M=ovcdbnf  ACBP=A9
 0002:000001A4 00000008 C=ICODE    S=.itext   G=(none)   M=ovcdbpf  ACBP=A9
 0002:000001AC 00000008 C=ICODE    S=.itext   G=(none)   M=ovcdbsf  ACBP=A9
 0002:000001B4 00000008 C=ICODE    S=.itext   G=(none)   M=ovcdbae  ACBP=A9
 0002:000001BC 00000008 C=ICODE    S=.itext   G=(none)   M=ovcdbcal ACBP=A9
 0002:000001C4 00000008 C=ICODE    S=.itext   G=(none)   M=ovcdbccb ACBP=A9
 0002:000001CC 00000008 C=ICODE    S=.itext   G=(none)   M=ovcdbcl  ACBP=A9
 0002:000001D4 00000008 C=ICODE    S=.itext   G=(none)   M=ovcdbclk ACBP=A9
 0002:000001DC 00000008 C=ICODE    S=.itext   G=(none)   M=ovcdbdat ACBP=A9
 0002:000001E4 00000008 C=ICODE    S=.itext   G=(none)   M=ovcdbdLb ACBP=A9
 0002:000001EC 00000006 C=ICODE    S=.itext   G=(none)   M=ovcfxfnt ACBP=A9
 0002:000001F4 00000008 C=ICODE    S=.itext   G=(none)   M=ovcdbed  ACBP=A9
 0002:000001FC 00000008 C=ICODE    S=.itext   G=(none)   M=ovcdbfcb ACBP=A9
 0002:00000204 00000008 C=ICODE    S=.itext   G=(none)   M=ovcdbidx ACBP=A9
 0002:0000020C 00000008 C=ICODE    S=.itext   G=(none)   M=ovcdbise ACBP=A9
 0002:00000214 00000008 C=ICODE    S=.itext   G=(none)   M=ovcdbmdg ACBP=A9
 0002:0000021C 00000008 C=ICODE    S=.itext   G=(none)   M=ovcdbnum ACBP=A9
 0002:00000224 00000008 C=ICODE    S=.itext   G=(none)   M=ovcdbplb ACBP=A9
 0002:0000022C 00000006 C=ICODE    S=.itext   G=(none)   M=ovcrvexpdef ACBP=A9
 0002:00000234 00000006 C=ICODE    S=.itext   G=(none)   M=ovcrptvw ACBP=A9
 0002:0000023C 00000008 C=ICODE    S=.itext   G=(none)   M=ovcdbrpv ACBP=A9
 0002:00000244 00000008 C=ICODE    S=.itext   G=(none)   M=ovcdbsed ACBP=A9
 0002:0000024C 00000008 C=ICODE    S=.itext   G=(none)   M=ovcdbsld ACBP=A9
 0002:00000254 00000006 C=ICODE    S=.itext   G=(none)   M=ovctgres ACBP=A9
 0002:0000025C 00000008 C=ICODE    S=.itext   G=(none)   M=ovcdbtbl ACBP=A9
 0002:00000264 00000008 C=ICODE    S=.itext   G=(none)   M=ovcdbtim ACBP=A9
 0002:0000026C 00000006 C=ICODE    S=.itext   G=(none)   M=o32rxvld ACBP=A9
 0002:00000274 00000006 C=ICODE    S=.itext   G=(none)   M=o32vlreg ACBP=A9
 0002:0000027C 00000006 C=ICODE    S=.itext   G=(none)   M=o32pvldr ACBP=A9
 0002:00000284 00000006 C=ICODE    S=.itext   G=(none)   M=o32ovldr ACBP=A9
 0002:0000028C 00000008 C=ICODE    S=.itext   G=(none)   M=o32dbfe  ACBP=A9
 0002:00000294 00000005 C=ICODE    S=.itext   G=(none)   M=.O406br2005 ACBP=A9
 0003:00000000 00000030 C=DATA     S=.data    G=DGROUP   M=SysInit  ACBP=A9
 0003:00000030 00000006 C=DATA     S=.data    G=DGROUP   M=ovcdbnf  ACBP=A9
 0003:00000038 00000006 C=DATA     S=.data    G=DGROUP   M=ovcdbpf  ACBP=A9
 0003:00000040 00000006 C=DATA     S=.data    G=DGROUP   M=ovcdbsf  ACBP=A9
 0003:00000048 00000008 C=DATA     S=.data    G=DGROUP   M=ovcdbae  ACBP=A9
 0003:00000050 00000006 C=DATA     S=.data    G=DGROUP   M=ovcdbcal ACBP=A9
 0003:00000058 00000006 C=DATA     S=.data    G=DGROUP   M=ovcdbccb ACBP=A9
 0003:00000060 00000006 C=DATA     S=.data    G=DGROUP   M=ovcdbclk ACBP=A9
 0003:00000068 00000006 C=DATA     S=.data    G=DGROUP   M=ovcdbdat ACBP=A9
 0003:00000070 00000008 C=DATA     S=.data    G=DGROUP   M=ovcdbidx ACBP=A9
 0003:00000078 00000008 C=DATA     S=.data    G=DGROUP   M=ovcdbise ACBP=A9
 0003:00000080 00000006 C=DATA     S=.data    G=DGROUP   M=ovcdbnum ACBP=A9
 0003:00000088 00000001 C=DATA     S=.data    G=DGROUP   M=ovcdbrpv ACBP=A9
 0003:0000008C 00000006 C=DATA     S=.data    G=DGROUP   M=ovcdbsed ACBP=A9
 0003:00000094 00000006 C=DATA     S=.data    G=DGROUP   M=ovcdbsld ACBP=A9
 0003:0000009C 00000006 C=DATA     S=.data    G=DGROUP   M=ovcdbtbl ACBP=A9
 0003:000000A4 00000006 C=DATA     S=.data    G=DGROUP   M=ovcdbtim ACBP=A9
 0003:000000AC 00000006 C=DATA     S=.data    G=DGROUP   M=o32dbfe  ACBP=A9
 0004:00000000 0000000C C=BSS      S=.bss     G=DGROUP   M=SysInit  ACBP=A9
 0004:0000000C 00000008 C=BSS      S=.bss     G=DGROUP   M=Windows  ACBP=A9
 0004:00000014 00000004 C=BSS      S=.bss     G=DGROUP   M=ovcdbhll ACBP=A9
 0004:00000018 00000004 C=BSS      S=.bss     G=DGROUP   M=ovcdbtcb ACBP=A9
 0004:0000001C 00000004 C=BSS      S=.bss     G=DGROUP   M=ovcdbacb ACBP=A9
 0004:00000020 00000004 C=BSS      S=.bss     G=DGROUP   M=ovcdbadg ACBP=A9
 0004:00000024 00000004 C=BSS      S=.bss     G=DGROUP   M=ovcdbnf  ACBP=A9
 0004:00000028 00000004 C=BSS      S=.bss     G=DGROUP   M=ovcdbpf  ACBP=A9
 0004:0000002C 00000004 C=BSS      S=.bss     G=DGROUP   M=ovcdbsf  ACBP=A9
 0004:00000030 00000004 C=BSS      S=.bss     G=DGROUP   M=ovcdbae  ACBP=A9
 0004:00000034 00000004 C=BSS      S=.bss     G=DGROUP   M=ovcdbcal ACBP=A9
 0004:00000038 00000004 C=BSS      S=.bss     G=DGROUP   M=ovcdbccb ACBP=A9
 0004:0000003C 00000004 C=BSS      S=.bss     G=DGROUP   M=ovcdbcl  ACBP=A9
 0004:00000040 00000004 C=BSS      S=.bss     G=DGROUP   M=ovcdbclk ACBP=A9
 0004:00000044 00000004 C=BSS      S=.bss     G=DGROUP   M=ovcdbdat ACBP=A9
 0004:00000048 00000004 C=BSS      S=.bss     G=DGROUP   M=ovcdbdLb ACBP=A9
 0004:0000004C 00000004 C=BSS      S=.bss     G=DGROUP   M=ovcdbed  ACBP=A9
 0004:00000050 00000004 C=BSS      S=.bss     G=DGROUP   M=ovcdbfcb ACBP=A9
 0004:00000054 00000004 C=BSS      S=.bss     G=DGROUP   M=ovcdbidx ACBP=A9
 0004:00000058 00000004 C=BSS      S=.bss     G=DGROUP   M=ovcdbise ACBP=A9
 0004:0000005C 00000004 C=BSS      S=.bss     G=DGROUP   M=ovcdbmdg ACBP=A9
 0004:00000060 00000004 C=BSS      S=.bss     G=DGROUP   M=ovcdbnum ACBP=A9
 0004:00000064 00000004 C=BSS      S=.bss     G=DGROUP   M=ovcdbplb ACBP=A9
 0004:00000068 00000004 C=BSS      S=.bss     G=DGROUP   M=ovcdbrpv ACBP=A9
 0004:0000006C 00000004 C=BSS      S=.bss     G=DGROUP   M=ovcdbsed ACBP=A9
 0004:00000070 00000004 C=BSS      S=.bss     G=DGROUP   M=ovcdbsld ACBP=A9
 0004:00000074 00000004 C=BSS      S=.bss     G=DGROUP   M=ovcdbtbl ACBP=A9
 0004:00000078 00000004 C=BSS      S=.bss     G=DGROUP   M=ovcdbtim ACBP=A9
 0004:0000007C 00000004 C=BSS      S=.bss     G=DGROUP   M=o32dbfe  ACBP=A9


  Address             Publics by Name

 0002:00000294       .O406br2005..O406br2005
 0001:00034708       .O406br2005.@GetPackageInfoTable
 0001:00034710       .O406br2005.@PackageLoad
 0001:0003471C       .O406br2005.@PackageUnload
 0004:0000007C       o32dbfe..2
 0001:00032230       o32dbfe..TO32DbFlexEdit
 0001:00034070       o32dbfe.Finalization
 0002:0000028C       o32dbfe.o32dbfe
 0003:000000AC       o32dbfe.SupportedFieldTypes
 0001:00032E20       o32dbfe.TO32DbFlexEdit.CMEnter
 0001:00032E3C       o32dbfe.TO32DbFlexEdit.CMExit
 0001:00032E44       o32dbfe.TO32DbFlexEdit.CMGetDataLink
 0001:00032E50       o32dbfe.TO32DbFlexEdit.Create
 0001:00032F34       o32dbfe.TO32DbFlexEdit.CreateWnd
 0001:00032F64       o32dbfe.TO32DbFlexEdit.CutToClipboard
 0001:00032EE8       o32dbfe.TO32DbFlexEdit.Destroy
 0001:00033064       o32dbfe.TO32DbFlexEdit.DoOnChange
 0001:00033FF8       o32dbfe.TO32DbFlexEdit.ExecuteAction
 0001:00033340       o32dbfe.TO32DbFlexEdit.fedbDataChange
 0001:000333A8       o32dbfe.TO32DbFlexEdit.fedbEditingChange
 0001:000333CC       o32dbfe.TO32DbFlexEdit.fedbGetFieldValue
 0001:000336C8       o32dbfe.TO32DbFlexEdit.fedbSetFieldProperties
 0001:0003372C       o32dbfe.TO32DbFlexEdit.fedbSetFieldValue
 0001:00033B50       o32dbfe.TO32DbFlexEdit.fedbUpdateData
 0001:00033084       o32dbfe.TO32DbFlexEdit.GetDataField
 0001:000330A0       o32dbfe.TO32DbFlexEdit.GetDataSource
 0001:000330B4       o32dbfe.TO32DbFlexEdit.GetField
 0001:00033134       o32dbfe.TO32DbFlexEdit.Notification
 0001:00032FE4       o32dbfe.TO32DbFlexEdit.PasteFromClipboard
 0001:0003317C       o32dbfe.TO32DbFlexEdit.Restore
 0001:0003319C       o32dbfe.TO32DbFlexEdit.SetDataField
 0001:00033254       o32dbfe.TO32DbFlexEdit.SetDataSource
 0001:00033288       o32dbfe.TO32DbFlexEdit.SetFieldType
 0001:00033328       o32dbfe.TO32DbFlexEdit.SetUseTFieldMask
 0001:00034034       o32dbfe.TO32DbFlexEdit.UpdateAction
 0001:00033C00       o32dbfe.TO32DbFlexEdit.WMChar
 0001:00033B98       o32dbfe.TO32DbFlexEdit.WMKeyDown
 0001:00033C28       o32dbfe.TO32DbFlexEdit.WMKillFocus
 0001:00033C70       o32dbfe.TO32DbFlexEdit.WMLButtonDblClk
 0001:00033C84       o32dbfe.TO32DbFlexEdit.WMLButtonDown
 0001:00033C98       o32dbfe.TO32DbFlexEdit.WMLButtonUp
 0001:00033CBC       o32dbfe.TO32DbFlexEdit.WMPaint
 0001:00033FC8       o32dbfe.TO32DbFlexEdit.WMSetFocus
 0004:0000001C       ovcdbacb..2
 0001:0000266C       ovcdbacb..TOvcDbAliasComboBox
 0001:00003160       ovcdbacb.Finalization
 0002:0000014C       ovcdbacb.ovcdbacb
 0001:00002FF8       ovcdbacb.TOvcDbAliasComboBox.GetAliasName
 0001:000030B0       ovcdbacb.TOvcDbAliasComboBox.GetDriverName
 0001:00003034       ovcdbacb.TOvcDbAliasComboBox.GetPath
 0001:00002F5C       ovcdbacb.TOvcDbAliasComboBox.Loaded
 0001:0000312C       ovcdbacb.TOvcDbAliasComboBox.Notification
 0001:00002F78       ovcdbacb.TOvcDbAliasComboBox.Populate
 0001:00002F98       ovcdbacb.TOvcDbAliasComboBox.SelectionChanged
 0004:00000020       ovcdbadg..3
 0001:000034EC       ovcdbadg..TOvcDbAliasDialog
 0001:000031D0       ovcdbadg..TOvcfrmAliasDlg
 0001:000036F8       ovcdbadg.ExpandAlias
 0001:00003E38       ovcdbadg.Finalization
 0002:0000015C       ovcdbadg.ovcdbadg
 0001:000038B0       ovcdbadg.TOvcDbAliasDialog.Create
 0001:00003978       ovcdbadg.TOvcDbAliasDialog.Execute
 0001:00003A50       ovcdbadg.TOvcDbAliasDialog.GetPath
 0001:00003A88       ovcdbadg.TOvcDbAliasDialog.GetTableName
 0001:00003A9C       ovcdbadg.TOvcfrmAliasDlg.btnBrowseClick
 0001:00003B30       ovcdbadg.TOvcfrmAliasDlg.cbAliasListChange
 0001:00003D24       ovcdbadg.TOvcfrmAliasDlg.edTableNameChange
 0001:00003D44       ovcdbadg.TOvcfrmAliasDlg.FileListBox1Change
 0001:00003DC0       ovcdbadg.TOvcfrmAliasDlg.FileListBox1DblClick
 0001:00003DE0       ovcdbadg.TOvcfrmAliasDlg.FormCreate
 0001:00003DFC       ovcdbadg.TOvcfrmAliasDlg.FormShow
 0004:00000030       ovcdbae..8
 0001:0000B3D8       ovcdbae..TOvcBaseDbArrayEditor
 0001:0000CAF4       ovcdbae..TOvcDbNumericArrayEditor
 0001:0000B220       ovcdbae..TOvcDbNumericCell
 0001:0000C034       ovcdbae..TOvcDbPictureArrayEditor
 0001:0000B068       ovcdbae..TOvcDbPictureCell
 0001:0000B5BC       ovcdbae..TOvcDbSimpleArrayEditor
 0001:0000AEB4       ovcdbae..TOvcDbSimpleCell
 0001:00010E10       ovcdbae.Finalization
 0002:000001B4       ovcdbae.ovcdbae
 0003:00000048       ovcdbae.ScrollBar
 0001:0000D524       ovcdbae.TOvcBaseDbArrayEditor.aeActiveChange
 0001:0000D540       ovcdbae.TOvcBaseDbArrayEditor.aeAdjustIntegralHeight
 0001:0000D57C       ovcdbae.TOvcBaseDbArrayEditor.aeAdjustRowHeight
 0001:0000D668       ovcdbae.TOvcBaseDbArrayEditor.aeColorChanged
 0001:0000D670       ovcdbae.TOvcBaseDbArrayEditor.aeDataChange
 0001:0000D6E8       ovcdbae.TOvcBaseDbArrayEditor.aeEditingChange
 0001:0000D704       ovcdbae.TOvcBaseDbArrayEditor.aeGetEditString
 0001:0000D710       ovcdbae.TOvcBaseDbArrayEditor.aeGetSampleDisplayData
 0001:0000D724       ovcdbae.TOvcBaseDbArrayEditor.aeMoveCell
 0001:0000D740       ovcdbae.TOvcBaseDbArrayEditor.aeReadRangeHi
 0001:0000D760       ovcdbae.TOvcBaseDbArrayEditor.aeReadRangeLo
 0001:0000D780       ovcdbae.TOvcBaseDbArrayEditor.aeRefresh
 0001:0000D79C       ovcdbae.TOvcBaseDbArrayEditor.aeUpdateActive
 0001:0000D7D4       ovcdbae.TOvcBaseDbArrayEditor.aeUpdateData
 0001:0000D7F0       ovcdbae.TOvcBaseDbArrayEditor.aeUpdateNumRows
 0001:0000D850       ovcdbae.TOvcBaseDbArrayEditor.aeUpdateScrollBar
 0001:0000D9B8       ovcdbae.TOvcBaseDbArrayEditor.aeWriteRangeHi
 0001:0000D9CC       ovcdbae.TOvcBaseDbArrayEditor.aeWriteRangeLo
 0001:0000D9E0       ovcdbae.TOvcBaseDbArrayEditor.ChangeScale
 0001:0000DA18       ovcdbae.TOvcBaseDbArrayEditor.CMCtl3DChanged
 0001:0000DA58       ovcdbae.TOvcBaseDbArrayEditor.CMFontChanged
 0001:0000DA84       ovcdbae.TOvcBaseDbArrayEditor.Create
 0001:0000DD2C       ovcdbae.TOvcBaseDbArrayEditor.CreateParams
 0001:0000DD8C       ovcdbae.TOvcBaseDbArrayEditor.CreateWnd
 0001:0000DDEC       ovcdbae.TOvcBaseDbArrayEditor.DefineProperties
 0001:0000DE5C       ovcdbae.TOvcBaseDbArrayEditor.Destroy
 0001:0000DEBC       ovcdbae.TOvcBaseDbArrayEditor.DoGetItemColor
 0001:0000DEEC       ovcdbae.TOvcBaseDbArrayEditor.DoOnIndicatorClick
 0001:0000DF14       ovcdbae.TOvcBaseDbArrayEditor.GetDataLink
 0001:0000DF74       ovcdbae.TOvcBaseDbArrayEditor.GetField
 0001:0000DFE0       ovcdbae.TOvcBaseDbArrayEditor.GetRangeHi
 0001:0000DFFC       ovcdbae.TOvcBaseDbArrayEditor.GetRangeLo
 0001:0000E018       ovcdbae.TOvcBaseDbArrayEditor.Paint
 0001:0000E828       ovcdbae.TOvcBaseDbArrayEditor.Reset
 0001:0000E854       ovcdbae.TOvcBaseDbArrayEditor.Scroll
 0001:0000E888       ovcdbae.TOvcBaseDbArrayEditor.SetActiveRow
 0001:0000E8E0       ovcdbae.TOvcBaseDbArrayEditor.SetAutoRowHeight
 0001:0000E8FC       ovcdbae.TOvcBaseDbArrayEditor.SetBorderStyle
 0001:0000E910       ovcdbae.TOvcBaseDbArrayEditor.SetDataField
 0001:0000E93C       ovcdbae.TOvcBaseDbArrayEditor.SetDataSource
 0001:0000E948       ovcdbae.TOvcBaseDbArrayEditor.SetDateOrTime
 0001:0000E984       ovcdbae.TOvcBaseDbArrayEditor.SetDecimalPlaces
 0001:0000E9C4       ovcdbae.TOvcBaseDbArrayEditor.SetEpoch
 0001:0000EA00       ovcdbae.TOvcBaseDbArrayEditor.SetFieldType
 0001:0000EA0C       ovcdbae.TOvcBaseDbArrayEditor.SetFocus
 0001:0000EA38       ovcdbae.TOvcBaseDbArrayEditor.SetLineColor
 0001:0000EA4C       ovcdbae.TOvcBaseDbArrayEditor.SetMaxLength
 0001:0000EA94       ovcdbae.TOvcBaseDbArrayEditor.SetOptions
 0001:0000EB04       ovcdbae.TOvcBaseDbArrayEditor.SetPadChar
 0001:0000EB3C       ovcdbae.TOvcBaseDbArrayEditor.SetPictureMask
 0001:0000EC48       ovcdbae.TOvcBaseDbArrayEditor.SetRangeHi
 0001:0000EC88       ovcdbae.TOvcBaseDbArrayEditor.SetRangeLo
 0001:0000ECC8       ovcdbae.TOvcBaseDbArrayEditor.SetRowHeight
 0001:0000ECF0       ovcdbae.TOvcBaseDbArrayEditor.SetRowIndicatorWidth
 0001:0000ED68       ovcdbae.TOvcBaseDbArrayEditor.SetShowIndicator
 0001:0000EE04       ovcdbae.TOvcBaseDbArrayEditor.SetTextMargin
 0001:0000EE60       ovcdbae.TOvcBaseDbArrayEditor.SetUseScrollBar
 0001:0000EE74       ovcdbae.TOvcBaseDbArrayEditor.SetZeroAsNull
 0001:0000EE34       ovcdbae.TOvcBaseDbArrayEditor.UpdateRecord
 0001:0000EF00       ovcdbae.TOvcBaseDbArrayEditor.WMEraseBkGnd
 0001:0000EEEC       ovcdbae.TOvcBaseDbArrayEditor.WMGetMinMaxInfo
 0001:0000EF08       ovcdbae.TOvcBaseDbArrayEditor.WMLButtonDown
 0001:0000F060       ovcdbae.TOvcBaseDbArrayEditor.WMMouseActivate
 0001:0000F06C       ovcdbae.TOvcBaseDbArrayEditor.WMNCHitTest
 0001:0000F088       ovcdbae.TOvcBaseDbArrayEditor.WMSetFocus
 0001:0000F0E4       ovcdbae.TOvcBaseDbArrayEditor.WMSize
 0001:0000F170       ovcdbae.TOvcBaseDbArrayEditor.WMVScroll
 0001:0000FEDC       ovcdbae.TOvcDbNumericArrayEditor.aeCreateEditCell
 0001:000102FC       ovcdbae.TOvcDbNumericArrayEditor.aeGetCellProperties
 0001:000103B4       ovcdbae.TOvcDbNumericArrayEditor.Create
 0001:00010AC0       ovcdbae.TOvcDbNumericCell.Create
 0001:00010B2C       ovcdbae.TOvcDbNumericCell.CreateWnd
 0001:00010CC8       ovcdbae.TOvcDbNumericCell.WMKeyDown
 0001:0000F920       ovcdbae.TOvcDbPictureArrayEditor.aeCreateEditCell
 0001:0000FDB0       ovcdbae.TOvcDbPictureArrayEditor.aeGetCellProperties
 0001:0000FE68       ovcdbae.TOvcDbPictureArrayEditor.Create
 0001:00010770       ovcdbae.TOvcDbPictureCell.Create
 0001:000107DC       ovcdbae.TOvcDbPictureCell.CreateWnd
 0001:00010978       ovcdbae.TOvcDbPictureCell.WMKeyDown
 0001:0000F3A0       ovcdbae.TOvcDbSimpleArrayEditor.aeCreateEditCell
 0001:0000F804       ovcdbae.TOvcDbSimpleArrayEditor.aeGetCellProperties
 0001:0000F8BC       ovcdbae.TOvcDbSimpleArrayEditor.Create
 0001:00010420       ovcdbae.TOvcDbSimpleCell.Create
 0001:0001048C       ovcdbae.TOvcDbSimpleCell.CreateWnd
 0001:00010628       ovcdbae.TOvcDbSimpleCell.WMKeyDown
 0004:00000034       ovcdbcal..2
 0001:00010ED8       ovcdbcal..TOvcDbCalendar
 0001:00011E5C       ovcdbcal.Finalization
 0002:000001BC       ovcdbcal.ovcdbcal
 0003:00000050       ovcdbcal.SupportedFieldTypes
 0001:00011770       ovcdbcal.TOvcDbCalendar.calDataChange
 0001:000117F8       ovcdbcal.TOvcDbCalendar.calUpdateData
 0001:00011918       ovcdbcal.TOvcDbCalendar.CMExit
 0001:0001197C       ovcdbcal.TOvcDbCalendar.CMGetDataLink
 0001:00011988       ovcdbcal.TOvcDbCalendar.Create
 0001:00011A04       ovcdbcal.TOvcDbCalendar.Destroy
 0001:00011A3C       ovcdbcal.TOvcDbCalendar.DoOnChange
 0001:00011DE4       ovcdbcal.TOvcDbCalendar.ExecuteAction
 0001:00011A60       ovcdbcal.TOvcDbCalendar.GetDataField
 0001:00011A7C       ovcdbcal.TOvcDbCalendar.GetDataSource
 0001:00011A90       ovcdbcal.TOvcDbCalendar.GetField
 0001:00011A9C       ovcdbcal.TOvcDbCalendar.IsReadOnly
 0001:00011DB0       ovcdbcal.TOvcDbCalendar.KeyPress
 0001:00011AD0       ovcdbcal.TOvcDbCalendar.Notification
 0001:00011B14       ovcdbcal.TOvcDbCalendar.SetCalendarDate
 0001:00011B88       ovcdbcal.TOvcDbCalendar.SetDataField
 0001:00011CFC       ovcdbcal.TOvcDbCalendar.SetDataSource
 0001:00011E20       ovcdbcal.TOvcDbCalendar.UpdateAction
 0001:00011D6C       ovcdbcal.TOvcDbCalendar.WMKeyDown
 0001:00011D28       ovcdbcal.TOvcDbCalendar.WMLButtonDown
 0004:00000038       ovcdbccb..2
 0001:00011EBC       ovcdbccb..TOvcDbColorComboBox
 0001:00012C30       ovcdbccb.Finalization
 0002:000001C4       ovcdbccb.ovcdbccb
 0003:00000058       ovcdbccb.SupportedFieldTypes
 0001:0001277C       ovcdbccb.TOvcDbColorComboBox.ccbDataChange
 0001:000127BC       ovcdbccb.TOvcDbColorComboBox.ccbUpdateData
 0001:000127F4       ovcdbccb.TOvcDbColorComboBox.Change
 0001:000128E0       ovcdbccb.TOvcDbColorComboBox.CMGetDataLink
 0001:000128EC       ovcdbccb.TOvcDbColorComboBox.Create
 0001:00012960       ovcdbccb.TOvcDbColorComboBox.Destroy
 0001:00012BB8       ovcdbccb.TOvcDbColorComboBox.ExecuteAction
 0001:00012998       ovcdbccb.TOvcDbColorComboBox.GetDataField
 0001:000129B4       ovcdbccb.TOvcDbColorComboBox.GetDataSource
 0001:000129C8       ovcdbccb.TOvcDbColorComboBox.GetField
 0001:000129D4       ovcdbccb.TOvcDbColorComboBox.Notification
 0001:00012A18       ovcdbccb.TOvcDbColorComboBox.SetDataField
 0001:00012B8C       ovcdbccb.TOvcDbColorComboBox.SetDataSource
 0001:00012BF4       ovcdbccb.TOvcDbColorComboBox.UpdateAction
 0004:0000003C       ovcdbcl..2
 0001:00012CE4       ovcdbcl..TOvcDbColumnList
 0001:000156D4       ovcdbcl.Finalization
 0001:00014F08       ovcdbcl.HScrollPrim
 0002:000001CC       ovcdbcl.ovcdbcl
 0001:000136E8       ovcdbcl.TOvcDbColumnList.ChangeScale
 0001:00013720       ovcdbcl.TOvcDbColumnList.clActiveChange
 0001:0001373C       ovcdbcl.TOvcDbColumnList.clAdjustIntegralHeight
 0001:00013788       ovcdbcl.TOvcDbColumnList.clAdjustRowHeight
 0001:00013874       ovcdbcl.TOvcDbColumnList.clCalcNumRows
 0001:000138B4       ovcdbcl.TOvcDbColumnList.clColorChanged
 0001:000138BC       ovcdbcl.TOvcDbColumnList.clDataChange
 0001:000138EC       ovcdbcl.TOvcDbColumnList.clDrawHeader
 0001:00013C2C       ovcdbcl.TOvcDbColumnList.clEditingChange
 0001:00013C40       ovcdbcl.TOvcDbColumnList.clInitScrollBarInfo
 0001:00013C6C       ovcdbcl.TOvcDbColumnList.clSetHScrollPos
 0001:00013C98       ovcdbcl.TOvcDbColumnList.clSetHScrollRange
 0001:00013CF0       ovcdbcl.TOvcDbColumnList.clSetVScrollPos
 0001:00013E4C       ovcdbcl.TOvcDbColumnList.clSetVScrollRange
 0001:00013E54       ovcdbcl.TOvcDbColumnList.clUpdateActive
 0001:00013E80       ovcdbcl.TOvcDbColumnList.clUpdateData
 0001:00013E84       ovcdbcl.TOvcDbColumnList.clUpdateNumRows
 0001:00013EF4       ovcdbcl.TOvcDbColumnList.CMCtl3DChanged
 0001:00013F34       ovcdbcl.TOvcDbColumnList.CMFontChanged
 0001:00013F80       ovcdbcl.TOvcDbColumnList.CMGetDataLink
 0001:00013F8C       ovcdbcl.TOvcDbColumnList.Create
 0001:00014298       ovcdbcl.TOvcDbColumnList.CreateParams
 0001:000142FC       ovcdbcl.TOvcDbColumnList.CreateWnd
 0001:0001433C       ovcdbcl.TOvcDbColumnList.Destroy
 0001:000143B0       ovcdbcl.TOvcDbColumnList.DoOnClickHeader
 0001:000143E0       ovcdbcl.TOvcDbColumnList.DoOnIndicatorClick
 0001:00014408       ovcdbcl.TOvcDbColumnList.DoOnUserCommand
 0001:0001565C       ovcdbcl.TOvcDbColumnList.ExecuteAction
 0001:0001448C       ovcdbcl.TOvcDbColumnList.GetDataField
 0001:000144A8       ovcdbcl.TOvcDbColumnList.GetDataSource
 0001:00014428       ovcdbcl.TOvcDbColumnList.GetField
 0001:000144BC       ovcdbcl.TOvcDbColumnList.InvalidateItem
 0001:00014520       ovcdbcl.TOvcDbColumnList.Notification
 0001:0001455C       ovcdbcl.TOvcDbColumnList.Paint
 0001:00014C58       ovcdbcl.TOvcDbColumnList.SetActiveRow
 0001:00014CA4       ovcdbcl.TOvcDbColumnList.SetAutoRowHeight
 0001:00014CC0       ovcdbcl.TOvcDbColumnList.SetBorderStyle
 0001:00014CD4       ovcdbcl.TOvcDbColumnList.SetDataField
 0001:00014D84       ovcdbcl.TOvcDbColumnList.SetDataSource
 0001:00014DB0       ovcdbcl.TOvcDbColumnList.SetHeader
 0001:00014DE0       ovcdbcl.TOvcDbColumnList.SetIntegralHeight
 0001:00014DF4       ovcdbcl.TOvcDbColumnList.SetLineColor
 0001:00014E08       ovcdbcl.TOvcDbColumnList.SetRowHeight
 0001:00014E8C       ovcdbcl.TOvcDbColumnList.SetRowIndicatorWidth
 0001:00014E30       ovcdbcl.TOvcDbColumnList.SetScrollBars
 0001:00014E44       ovcdbcl.TOvcDbColumnList.SetShowHeader
 0001:00014E58       ovcdbcl.TOvcDbColumnList.SetShowIndicator
 0001:00014EC4       ovcdbcl.TOvcDbColumnList.SetTextMargin
 0001:00015698       ovcdbcl.TOvcDbColumnList.UpdateAction
 0001:00014EDC       ovcdbcl.TOvcDbColumnList.WMEraseBkgnd
 0001:00014EE4       ovcdbcl.TOvcDbColumnList.WMGetDlgCode
 0001:00014EF4       ovcdbcl.TOvcDbColumnList.WMGetMinMaxInfo
 0001:00014FBC       ovcdbcl.TOvcDbColumnList.WMHScroll
 0001:00015060       ovcdbcl.TOvcDbColumnList.WMKeyDown
 0001:00015254       ovcdbcl.TOvcDbColumnList.WMKillFocus
 0001:00015270       ovcdbcl.TOvcDbColumnList.WMLButtonDown
 0001:00015388       ovcdbcl.TOvcDbColumnList.WMMouseActivate
 0001:000153D4       ovcdbcl.TOvcDbColumnList.WMNCHitTest
 0001:000153F0       ovcdbcl.TOvcDbColumnList.WMSetFocus
 0001:0001540C       ovcdbcl.TOvcDbColumnList.WMSize
 0001:0001543C       ovcdbcl.TOvcDbColumnList.WMVScroll
 0004:00000040       ovcdbclk..2
 0001:00015754       ovcdbclk..TOvcDbClock
 0001:000160A4       ovcdbclk.Finalization
 0002:000001D4       ovcdbclk.ovcdbclk
 0003:00000060       ovcdbclk.SupportedFieldTypes
 0001:00015CC8       ovcdbclk.TOvcDbClock.clkDataChange
 0001:00015D5C       ovcdbclk.TOvcDbClock.CMGetDataLink
 0001:00015D68       ovcdbclk.TOvcDbClock.Create
 0001:00015DD4       ovcdbclk.TOvcDbClock.Destroy
 0001:0001602C       ovcdbclk.TOvcDbClock.ExecuteAction
 0001:00015E0C       ovcdbclk.TOvcDbClock.GetDataField
 0001:00015E28       ovcdbclk.TOvcDbClock.GetDataSource
 0001:00015E3C       ovcdbclk.TOvcDbClock.GetField
 0001:00015E48       ovcdbclk.TOvcDbClock.Notification
 0001:00015E8C       ovcdbclk.TOvcDbClock.SetDataField
 0001:00016000       ovcdbclk.TOvcDbClock.SetDataSource
 0001:00016068       ovcdbclk.TOvcDbClock.UpdateAction
 0004:00000044       ovcdbdat..3
 0001:000161A4       ovcdbdat..TOvcCustomDbDateEdit
 0001:00016384       ovcdbdat..TOvcDbDateEdit
 0003:00000068       ovcdbdat.DateFieldTypes
 0001:00017BE4       ovcdbdat.Finalization
 0002:000001DC       ovcdbdat.ovcdbdat
 0001:00016EBC       ovcdbdat.TOvcCustomDbDateEdit.Change
 0001:00016ED4       ovcdbdat.TOvcCustomDbDateEdit.CMEnter
 0001:00016EF0       ovcdbdat.TOvcCustomDbDateEdit.CMExit
 0001:00016F84       ovcdbdat.TOvcCustomDbDateEdit.CMGetDataLink
 0001:00016F90       ovcdbdat.TOvcCustomDbDateEdit.Create
 0001:00017024       ovcdbdat.TOvcCustomDbDateEdit.DataChange
 0001:0001721C       ovcdbdat.TOvcCustomDbDateEdit.Destroy
 0001:00017268       ovcdbdat.TOvcCustomDbDateEdit.EditingChange
 0001:00017B6C       ovcdbdat.TOvcCustomDbDateEdit.ExecuteAction
 0001:0001729C       ovcdbdat.TOvcCustomDbDateEdit.GetButtonEnabled
 0001:000172D0       ovcdbdat.TOvcCustomDbDateEdit.GetDataField
 0001:000172EC       ovcdbdat.TOvcCustomDbDateEdit.GetDataSource
 0001:000172F8       ovcdbdat.TOvcCustomDbDateEdit.GetField
 0001:00017304       ovcdbdat.TOvcCustomDbDateEdit.GetReadOnly
 0001:00017344       ovcdbdat.TOvcCustomDbDateEdit.GetTextMargins
 0001:0001740C       ovcdbdat.TOvcCustomDbDateEdit.KeyDown
 0001:00017444       ovcdbdat.TOvcCustomDbDateEdit.KeyPress
 0001:00017520       ovcdbdat.TOvcCustomDbDateEdit.Notification
 0001:0001755C       ovcdbdat.TOvcCustomDbDateEdit.PopupClose
 0001:0001758C       ovcdbdat.TOvcCustomDbDateEdit.PopupOpen
 0001:000175A4       ovcdbdat.TOvcCustomDbDateEdit.SetDataField
 0001:0001763C       ovcdbdat.TOvcCustomDbDateEdit.SetDataSource
 0001:00017660       ovcdbdat.TOvcCustomDbDateEdit.SetFocused
 0001:00017694       ovcdbdat.TOvcCustomDbDateEdit.SetReadOnly
 0001:00017BA8       ovcdbdat.TOvcCustomDbDateEdit.UpdateAction
 0001:000176A0       ovcdbdat.TOvcCustomDbDateEdit.UpdateData
 0001:000178B0       ovcdbdat.TOvcCustomDbDateEdit.WMCut
 0001:000178D0       ovcdbdat.TOvcCustomDbDateEdit.WMPaint
 0001:00017B4C       ovcdbdat.TOvcCustomDbDateEdit.WMPaste
 0004:00000048       ovcdbdLb..2
 0001:00017C84       ovcdbdLb..TOvcDbDisplayLabel
 0001:00018524       ovcdbdLb.Finalization
 0002:000001E4       ovcdbdLb.ovcdbdLb
 0001:0001825C       ovcdbdLb.TOvcDbDisplayLabel.CMGetDataLink
 0001:00018268       ovcdbdLb.TOvcDbDisplayLabel.Create
 0001:000182C4       ovcdbdLb.TOvcDbDisplayLabel.Destroy
 0001:000182FC       ovcdbdLb.TOvcDbDisplayLabel.dlDataChange
 0001:00018348       ovcdbdLb.TOvcDbDisplayLabel.dlGetDisplayLabel
 0001:000184AC       ovcdbdLb.TOvcDbDisplayLabel.ExecuteAction
 0001:000183C4       ovcdbdLb.TOvcDbDisplayLabel.GetDataField
 0001:000183E0       ovcdbdLb.TOvcDbDisplayLabel.GetDataSource
 0001:000183EC       ovcdbdLb.TOvcDbDisplayLabel.GetField
 0001:000183F8       ovcdbdLb.TOvcDbDisplayLabel.Notification
 0001:00018434       ovcdbdLb.TOvcDbDisplayLabel.SetDataField
 0001:00018488       ovcdbdLb.TOvcDbDisplayLabel.SetDataSource
 0001:000184E8       ovcdbdLb.TOvcDbDisplayLabel.UpdateAction
 0004:0000004C       ovcdbed..2
 0001:00018774       ovcdbed..TOvcDbEditor
 0001:00019E14       ovcdbed.DoChange
 0001:00019FC0       ovcdbed.Finalization
 0002:000001F4       ovcdbed.ovcdbed
 0001:00019390       ovcdbed.TOvcDbEditor.CMEnter
 0001:000193B0       ovcdbed.TOvcDbEditor.CMExit
 0001:00019424       ovcdbed.TOvcDbEditor.CMGetDataLink
 0001:00019430       ovcdbed.TOvcDbEditor.Create
 0001:000194AC       ovcdbed.TOvcDbEditor.CreateWnd
 0001:000194CC       ovcdbed.TOvcDbEditor.CutToClipboard
 0001:00019550       ovcdbed.TOvcDbEditor.Destroy
 0001:00019588       ovcdbed.TOvcDbEditor.edAddSampleParas
 0001:0001958C       ovcdbed.TOvcDbEditor.eddbDataChange
 0001:0001959C       ovcdbed.TOvcDbEditor.eddbEditingChange
 0001:000195A0       ovcdbed.TOvcDbEditor.eddbGetEditorValue
 0001:000196A4       ovcdbed.TOvcDbEditor.eddbSetEditorValue
 0001:00019A1C       ovcdbed.TOvcDbEditor.eddbUpdateData
 0001:00019F48       ovcdbed.TOvcDbEditor.ExecuteAction
 0001:00019AC0       ovcdbed.TOvcDbEditor.GetDataField
 0001:00019ADC       ovcdbed.TOvcDbEditor.GetDataSource
 0001:00019AB4       ovcdbed.TOvcDbEditor.GetField
 0001:00019A24       ovcdbed.TOvcDbEditor.GetReadOnly
 0001:00019AF0       ovcdbed.TOvcDbEditor.Notification
 0001:00019B28       ovcdbed.TOvcDbEditor.PasteFromClipboard
 0001:00019BAC       ovcdbed.TOvcDbEditor.Redo
 0001:00019C30       ovcdbed.TOvcDbEditor.Replace
 0001:00019CCC       ovcdbed.TOvcDbEditor.SetDataField
 0001:00019D28       ovcdbed.TOvcDbEditor.SetDataSource
 0001:00019D40       ovcdbed.TOvcDbEditor.Undo
 0001:00019F84       ovcdbed.TOvcDbEditor.UpdateAction
 0001:00019DC4       ovcdbed.TOvcDbEditor.WMChar
 0001:00019E8C       ovcdbed.TOvcDbEditor.WMKeyDown
 0004:00000050       ovcdbfcb..2
 0001:0001A00C       ovcdbfcb..TOvcDbFieldComboBox
 0001:0001AEB4       ovcdbfcb.Finalization
 0002:000001FC       ovcdbfcb.ovcdbfcb
 0001:0001A928       ovcdbfcb.TOvcDbFieldComboBox.ActiveChanged
 0001:0001A930       ovcdbfcb.TOvcDbFieldComboBox.Create
 0001:0001A9B8       ovcdbfcb.TOvcDbFieldComboBox.Destroy
 0001:0001A9F0       ovcdbfcb.TOvcDbFieldComboBox.DrawItem
 0001:0001AE3C       ovcdbfcb.TOvcDbFieldComboBox.ExecuteAction
 0001:0001AB90       ovcdbfcb.TOvcDbFieldComboBox.GetDataSource
 0001:0001AB9C       ovcdbfcb.TOvcDbFieldComboBox.GetFieldName
 0001:0001AC88       ovcdbfcb.TOvcDbFieldComboBox.Loaded
 0001:0001AC9C       ovcdbfcb.TOvcDbFieldComboBox.Populate
 0001:0001ADC4       ovcdbfcb.TOvcDbFieldComboBox.SetDataSource
 0001:0001ADDC       ovcdbfcb.TOvcDbFieldComboBox.SetOmitFields
 0001:0001AE20       ovcdbfcb.TOvcDbFieldComboBox.SetShowHiddenFields
 0001:0001AE78       ovcdbfcb.TOvcDbFieldComboBox.UpdateAction
 0004:00000014       ovcdbhll..2
 0001:000018B4       ovcdbhll..TOvcDbEngineHelperBase
 0001:00001C2C       ovcdbhll.Finalization
 0002:0000013C       ovcdbhll.ovcdbhll
 0001:00001A90       ovcdbhll.OvcFindNearestKey
 0001:00001AA8       ovcdbhll.OvcGetAliasDriverName
 0001:00001AC4       ovcdbhll.OvcGetAliasNames
 0001:00001B18       ovcdbhll.OvcGetAliasPath
 0001:00001B34       ovcdbhll.OvcGetIndexDefs
 0001:00001B44       ovcdbhll.OvcGetIndexField
 0001:00001B54       ovcdbhll.OvcGetIndexFieldCount
 0001:00001B64       ovcdbhll.OvcGetIndexFieldNames
 0001:00001B80       ovcdbhll.OvcGetIndexName
 0001:00001BD4       ovcdbhll.OvcGetTableNames
 0001:00001B9C       ovcdbhll.OvcIsChildDataSet
 0001:00001BAC       ovcdbhll.OvcSetIndexFieldNames
 0001:00001BC0       ovcdbhll.OvcSetIndexName
 0001:000019B0       ovcdbhll.TOvcDbEngineHelperBase.FindNearestKey
 0001:00001A0C       ovcdbhll.TOvcDbEngineHelperBase.GetAliasDriverName
 0001:000019B8       ovcdbhll.TOvcDbEngineHelperBase.GetAliasNames
 0001:00001A00       ovcdbhll.TOvcDbEngineHelperBase.GetAliasPath
 0001:00001A60       ovcdbhll.TOvcDbEngineHelperBase.GetIndexDefs
 0001:00001A64       ovcdbhll.TOvcDbEngineHelperBase.GetIndexField
 0001:00001A68       ovcdbhll.TOvcDbEngineHelperBase.GetIndexFieldCount
 0001:00001A6C       ovcdbhll.TOvcDbEngineHelperBase.GetIndexFieldNames
 0001:00001A78       ovcdbhll.TOvcDbEngineHelperBase.GetIndexName
 0001:00001A18       ovcdbhll.TOvcDbEngineHelperBase.GetTableNames
 0001:00001A84       ovcdbhll.TOvcDbEngineHelperBase.IsChildDataSet
 0001:00001A88       ovcdbhll.TOvcDbEngineHelperBase.SetIndexFieldNames
 0001:00001A8C       ovcdbhll.TOvcDbEngineHelperBase.SetIndexName
 0004:00000054       ovcdbidx..4
 0001:0001B188       ovcdbidx..TOvcDbIndexSelect
 0001:0001AFF4       ovcdbidx..TOvcIndexInfo
 0001:0001B09C       ovcdbidx..TOvcIndexSelectDataLink
 0003:00000070       ovcdbidx.DX
 0003:00000074       ovcdbidx.DY
 0001:0001CB28       ovcdbidx.Finalization
 0002:00000204       ovcdbidx.ovcdbidx
 0001:0001BE58       ovcdbidx.TOvcDbIndexSelect.Change
 0001:0001BED8       ovcdbidx.TOvcDbIndexSelect.ClearObjects
 0001:0001BF48       ovcdbidx.TOvcDbIndexSelect.CMVisibleChanged
 0001:0001BF78       ovcdbidx.TOvcDbIndexSelect.Create
 0001:0001C01C       ovcdbidx.TOvcDbIndexSelect.CreateWnd
 0001:0001C030       ovcdbidx.TOvcDbIndexSelect.Destroy
 0001:0001C094       ovcdbidx.TOvcDbIndexSelect.DestroyWnd
 0001:0001C0AC       ovcdbidx.TOvcDbIndexSelect.DropDown
 0001:0001C148       ovcdbidx.TOvcDbIndexSelect.GetAbout
 0001:0001C0C8       ovcdbidx.TOvcDbIndexSelect.GetAttachedLabel
 0001:0001C134       ovcdbidx.TOvcDbIndexSelect.GetDataSource
 0001:0001C178       ovcdbidx.TOvcDbIndexSelect.GetIndexFieldNames
 0001:0001C16C       ovcdbidx.TOvcDbIndexSelect.GetIndexName
 0001:0001C184       ovcdbidx.TOvcDbIndexSelect.isFindIndex
 0001:0001C2D0       ovcdbidx.TOvcDbIndexSelect.LabelAttach
 0001:0001C410       ovcdbidx.TOvcDbIndexSelect.LabelChange
 0001:0001C41C       ovcdbidx.TOvcDbIndexSelect.Notification
 0001:0001C480       ovcdbidx.TOvcDbIndexSelect.OMAssignLabel
 0001:0001C490       ovcdbidx.TOvcDbIndexSelect.OMPositionLabel
 0001:0001C538       ovcdbidx.TOvcDbIndexSelect.OMRecordLabelPosition
 0001:0001C59C       ovcdbidx.TOvcDbIndexSelect.PositionLabel
 0001:0001C634       ovcdbidx.TOvcDbIndexSelect.RefreshList
 0001:0001CA10       ovcdbidx.TOvcDbIndexSelect.RefreshNow
 0001:0001CAF8       ovcdbidx.TOvcDbIndexSelect.SetAbout
 0001:0001CA24       ovcdbidx.TOvcDbIndexSelect.SetBounds
 0001:0001CA60       ovcdbidx.TOvcDbIndexSelect.SetDataSource
 0001:0001CA90       ovcdbidx.TOvcDbIndexSelect.SetDisplayMode
 0001:0001CAAC       ovcdbidx.TOvcDbIndexSelect.SetMonitorIdx
 0001:0001CAD4       ovcdbidx.TOvcDbIndexSelect.SetRefreshPendingFlag
 0001:0001CADC       ovcdbidx.TOvcDbIndexSelect.SetShowHidden
 0001:0001CAFC       ovcdbidx.TOvcDbIndexSelect.WMDestroy
 0001:0001CB04       ovcdbidx.TOvcDbIndexSelect.WMPaint
 0001:0001B924       ovcdbidx.TOvcIndexInfo.Create
 0001:0001B998       ovcdbidx.TOvcIndexInfo.Destroy
 0001:0001B9CC       ovcdbidx.TOvcIndexInfo.RefreshIndexInfo
 0001:0001BD9C       ovcdbidx.TOvcIndexInfo.SetDisplayName
 0001:0001BDD0       ovcdbidx.TOvcIndexSelectDataLink.ActiveChanged
 0001:0001BDEC       ovcdbidx.TOvcIndexSelectDataLink.Create
 0001:0001BE28       ovcdbidx.TOvcIndexSelectDataLink.DataSetChanged
 0001:0001BE3C       ovcdbidx.TOvcIndexSelectDataLink.LayoutChanged
 0004:00000058       ovcdbise..2
 0001:0001CB80       ovcdbise..TOvcDbSearchEdit
 0003:00000078       ovcdbise.DX
 0003:0000007C       ovcdbise.DY
 0001:0001DCC4       ovcdbise.Finalization
 0002:0000020C       ovcdbise.ovcdbise
 0001:0001D450       ovcdbise.TOvcDbSearchEdit.CMVisibleChanged
 0001:0001D480       ovcdbise.TOvcDbSearchEdit.Create
 0001:0001D500       ovcdbise.TOvcDbSearchEdit.Destroy
 0001:0001D5D8       ovcdbise.TOvcDbSearchEdit.GetAbout
 0001:0001D558       ovcdbise.TOvcDbSearchEdit.GetAttachedLabel
 0001:0001D5C4       ovcdbise.TOvcDbSearchEdit.GetDataSource
 0001:0001D5FC       ovcdbise.TOvcDbSearchEdit.LabelAttach
 0001:0001D73C       ovcdbise.TOvcDbSearchEdit.LabelChange
 0001:0001D748       ovcdbise.TOvcDbSearchEdit.Notification
 0001:0001D7AC       ovcdbise.TOvcDbSearchEdit.OMAssignLabel
 0001:0001D7BC       ovcdbise.TOvcDbSearchEdit.OMPositionLabel
 0001:0001D864       ovcdbise.TOvcDbSearchEdit.OMRecordLabelPosition
 0001:0001D8C8       ovcdbise.TOvcDbSearchEdit.PerformSearch
 0001:0001DBC8       ovcdbise.TOvcDbSearchEdit.PositionLabel
 0001:0001DCC0       ovcdbise.TOvcDbSearchEdit.SetAbout
 0001:0001DC60       ovcdbise.TOvcDbSearchEdit.SetBounds
 0001:0001DC9C       ovcdbise.TOvcDbSearchEdit.SetDataSource
 0004:0000005C       ovcdbmdg..3
 0001:0001DF04       ovcdbmdg..TOvcDbMemoDialog
 0001:0001DCF4       ovcdbmdg..TOvcfrmDbMemoDlg
 0001:0001E5F4       ovcdbmdg.Finalization
 0002:00000214       ovcdbmdg.ovcdbmdg
 0001:0001E150       ovcdbmdg.TOvcDbMemoDialog.Create
 0001:0001E1AC       ovcdbmdg.TOvcDbMemoDialog.Destroy
 0001:0001E1EC       ovcdbmdg.TOvcDbMemoDialog.Execute
 0001:0001E500       ovcdbmdg.TOvcDbMemoDialog.ExecuteAction
 0001:0001E474       ovcdbmdg.TOvcDbMemoDialog.GetDataField
 0001:0001E48C       ovcdbmdg.TOvcDbMemoDialog.GetDataSource
 0001:0001E494       ovcdbmdg.TOvcDbMemoDialog.SetDataField
 0001:0001E4E4       ovcdbmdg.TOvcDbMemoDialog.SetDataSource
 0001:0001E4F0       ovcdbmdg.TOvcDbMemoDialog.SetMemoFont
 0001:0001E538       ovcdbmdg.TOvcDbMemoDialog.UpdateAction
 0001:0001E570       ovcdbmdg.TOvcfrmDbMemoDlg.FormCloseQuery
 0004:00000024       ovcdbnf..2
 0001:00003FC0       ovcdbnf..TOvcDbNumericField
 0001:0000506C       ovcdbnf.FieldIsZero
 0001:00005F20       ovcdbnf.Finalization
 0002:0000019C       ovcdbnf.ovcdbnf
 0003:00000030       ovcdbnf.SupportedFieldTypes
 0001:00004A48       ovcdbnf.TOvcDbNumericField.CMEnter
 0001:00004A64       ovcdbnf.TOvcDbNumericField.CMExit
 0001:00004A6C       ovcdbnf.TOvcDbNumericField.CMGetDataLink
 0001:00004A78       ovcdbnf.TOvcDbNumericField.Create
 0001:00004B18       ovcdbnf.TOvcDbNumericField.CreateWnd
 0001:00004B48       ovcdbnf.TOvcDbNumericField.CutToClipboard
 0001:00004BC8       ovcdbnf.TOvcDbNumericField.Destroy
 0001:00004C14       ovcdbnf.TOvcDbNumericField.DoOnChange
 0001:00004C40       ovcdbnf.TOvcDbNumericField.efEdit
 0001:00004CBC       ovcdbnf.TOvcDbNumericField.efGetSampleDisplayData
 0001:00004E38       ovcdbnf.TOvcDbNumericField.efIncDecValue
 0001:00004EB0       ovcdbnf.TOvcDbNumericField.efIsReadOnly
 0001:00005EA8       ovcdbnf.TOvcDbNumericField.ExecuteAction
 0001:00004F34       ovcdbnf.TOvcDbNumericField.GetDataField
 0001:00004F50       ovcdbnf.TOvcDbNumericField.GetDataSource
 0001:00004F64       ovcdbnf.TOvcDbNumericField.GetField
 0001:00004FE4       ovcdbnf.TOvcDbNumericField.nfdbDataChange
 0001:00005048       ovcdbnf.TOvcDbNumericField.nfdbEditingChange
 0001:00005120       ovcdbnf.TOvcDbNumericField.nfdbGetFieldValue
 0001:0000528C       ovcdbnf.TOvcDbNumericField.nfdbSetFieldProperties
 0001:00005348       ovcdbnf.TOvcDbNumericField.nfdbSetFieldValue
 0001:000055B8       ovcdbnf.TOvcDbNumericField.nfdbUpdateData
 0001:00005688       ovcdbnf.TOvcDbNumericField.nfSetPictureMask
 0001:000056A4       ovcdbnf.TOvcDbNumericField.Notification
 0001:000056EC       ovcdbnf.TOvcDbNumericField.PasteFromClipboard
 0001:0000576C       ovcdbnf.TOvcDbNumericField.Restore
 0001:0000578C       ovcdbnf.TOvcDbNumericField.SetDataField
 0001:00005844       ovcdbnf.TOvcDbNumericField.SetDataSource
 0001:00005878       ovcdbnf.TOvcDbNumericField.SetFieldType
 0001:00005918       ovcdbnf.TOvcDbNumericField.SetUseTFieldMask
 0001:00005930       ovcdbnf.TOvcDbNumericField.SetZeroAsNull
 0001:00005EE4       ovcdbnf.TOvcDbNumericField.UpdateAction
 0001:00005940       ovcdbnf.TOvcDbNumericField.WMKeyDown
 0001:00005A44       ovcdbnf.TOvcDbNumericField.WMKillFocus
 0001:00005AAC       ovcdbnf.TOvcDbNumericField.WMLButtonDblClk
 0001:00005AC0       ovcdbnf.TOvcDbNumericField.WMLButtonDown
 0001:00005AD4       ovcdbnf.TOvcDbNumericField.WMLButtonUp
 0001:00005AF4       ovcdbnf.TOvcDbNumericField.WMPaint
 0001:00005E7C       ovcdbnf.TOvcDbNumericField.WMSetFocus
 0004:00000060       ovcdbnum..3
 0001:0001E624       ovcdbnum..TOvcCustomDbNumberEdit
 0001:0001E80C       ovcdbnum..TOvcDbNumberEdit
 0001:0001FC18       ovcdbnum.Finalization
 0003:00000080       ovcdbnum.NumFieldTypes
 0002:0000021C       ovcdbnum.ovcdbnum
 0001:0001F12C       ovcdbnum.TOvcCustomDbNumberEdit.Change
 0001:0001F144       ovcdbnum.TOvcCustomDbNumberEdit.CMEnter
 0001:0001F160       ovcdbnum.TOvcCustomDbNumberEdit.CMExit
 0001:0001F1F4       ovcdbnum.TOvcCustomDbNumberEdit.CMGetDataLink
 0001:0001F200       ovcdbnum.TOvcCustomDbNumberEdit.Create
 0001:0001F294       ovcdbnum.TOvcCustomDbNumberEdit.DataChange
 0001:0001F44C       ovcdbnum.TOvcCustomDbNumberEdit.Destroy
 0001:0001F498       ovcdbnum.TOvcCustomDbNumberEdit.EditingChange
 0001:0001FBA0       ovcdbnum.TOvcCustomDbNumberEdit.ExecuteAction
 0001:0001F4CC       ovcdbnum.TOvcCustomDbNumberEdit.GetButtonEnabled
 0001:0001F500       ovcdbnum.TOvcCustomDbNumberEdit.GetDataField
 0001:0001F51C       ovcdbnum.TOvcCustomDbNumberEdit.GetDataSource
 0001:0001F528       ovcdbnum.TOvcCustomDbNumberEdit.GetField
 0001:0001F534       ovcdbnum.TOvcCustomDbNumberEdit.GetReadOnly
 0001:0001F560       ovcdbnum.TOvcCustomDbNumberEdit.GetTextMargins
 0001:0001F628       ovcdbnum.TOvcCustomDbNumberEdit.KeyDown
 0001:0001F660       ovcdbnum.TOvcCustomDbNumberEdit.KeyPress
 0001:0001F710       ovcdbnum.TOvcCustomDbNumberEdit.Notification
 0001:0001F74C       ovcdbnum.TOvcCustomDbNumberEdit.PopupClose
 0001:0001F77C       ovcdbnum.TOvcCustomDbNumberEdit.PopupOpen
 0001:0001F794       ovcdbnum.TOvcCustomDbNumberEdit.SetDataField
 0001:0001F82C       ovcdbnum.TOvcCustomDbNumberEdit.SetDataSource
 0001:0001F850       ovcdbnum.TOvcCustomDbNumberEdit.SetFocused
 0001:0001F884       ovcdbnum.TOvcCustomDbNumberEdit.SetReadOnly
 0001:0001FBDC       ovcdbnum.TOvcCustomDbNumberEdit.UpdateAction
 0001:0001F890       ovcdbnum.TOvcCustomDbNumberEdit.UpdateData
 0001:0001F8E4       ovcdbnum.TOvcCustomDbNumberEdit.WMCut
 0001:0001F904       ovcdbnum.TOvcCustomDbNumberEdit.WMPaint
 0001:0001FB80       ovcdbnum.TOvcCustomDbNumberEdit.WMPaste
 0004:00000028       ovcdbpf..2
 0001:00006008       ovcdbpf..TOvcDbPictureField
 0001:00007268       ovcdbpf.FieldIsZero
 0001:00008A48       ovcdbpf.Finalization
 0002:000001A4       ovcdbpf.ovcdbpf
 0003:00000038       ovcdbpf.SupportedFieldTypes
 0001:00006B74       ovcdbpf.TOvcDbPictureField.CMEnter
 0001:00006B90       ovcdbpf.TOvcDbPictureField.CMExit
 0001:00006B98       ovcdbpf.TOvcDbPictureField.CMGetDataLink
 0001:00006BA4       ovcdbpf.TOvcDbPictureField.Create
 0001:00006C4C       ovcdbpf.TOvcDbPictureField.CreateWnd
 0001:00006C7C       ovcdbpf.TOvcDbPictureField.CutToClipboard
 0001:00006CFC       ovcdbpf.TOvcDbPictureField.Destroy
 0001:00006D48       ovcdbpf.TOvcDbPictureField.DoOnChange
 0001:00006D74       ovcdbpf.TOvcDbPictureField.efEdit
 0001:00006DF0       ovcdbpf.TOvcDbPictureField.efGetSampleDisplayData
 0001:00006F6C       ovcdbpf.TOvcDbPictureField.efIncDecValue
 0001:00006FE4       ovcdbpf.TOvcDbPictureField.efIsReadOnly
 0001:000089D0       ovcdbpf.TOvcDbPictureField.ExecuteAction
 0001:00007068       ovcdbpf.TOvcDbPictureField.GetDataField
 0001:00007084       ovcdbpf.TOvcDbPictureField.GetDataSource
 0001:00007098       ovcdbpf.TOvcDbPictureField.GetField
 0001:00007118       ovcdbpf.TOvcDbPictureField.Notification
 0001:00007160       ovcdbpf.TOvcDbPictureField.PasteFromClipboard
 0001:000071E0       ovcdbpf.TOvcDbPictureField.pfdbDataChange
 0001:00007244       ovcdbpf.TOvcDbPictureField.pfdbEditingChange
 0001:00007330       ovcdbpf.TOvcDbPictureField.pfdbGetFieldValue
 0001:000076E8       ovcdbpf.TOvcDbPictureField.pfdbSetFieldProperties
 0001:00007920       ovcdbpf.TOvcDbPictureField.pfdbSetFieldValue
 0001:0000808C       ovcdbpf.TOvcDbPictureField.pfdbUpdateData
 0001:0000815C       ovcdbpf.TOvcDbPictureField.pfSetPictureMask
 0001:00008178       ovcdbpf.TOvcDbPictureField.Restore
 0001:00008198       ovcdbpf.TOvcDbPictureField.SetDataField
 0001:00008250       ovcdbpf.TOvcDbPictureField.SetDataSource
 0001:00008284       ovcdbpf.TOvcDbPictureField.SetDateOrTime
 0001:000082B0       ovcdbpf.TOvcDbPictureField.SetFieldType
 0001:00008350       ovcdbpf.TOvcDbPictureField.SetUseTFieldMask
 0001:00008368       ovcdbpf.TOvcDbPictureField.SetZeroAsNull
 0001:00008A0C       ovcdbpf.TOvcDbPictureField.UpdateAction
 0001:00008378       ovcdbpf.TOvcDbPictureField.WMKeyDown
 0001:0000847C       ovcdbpf.TOvcDbPictureField.WMKillFocus
 0001:000084E4       ovcdbpf.TOvcDbPictureField.WMLButtonDblClk
 0001:000084F8       ovcdbpf.TOvcDbPictureField.WMLButtonDown
 0001:0000850C       ovcdbpf.TOvcDbPictureField.WMLButtonUp
 0001:0000852C       ovcdbpf.TOvcDbPictureField.WMPaint
 0001:000089A4       ovcdbpf.TOvcDbPictureField.WMSetFocus
 0004:00000064       ovcdbplb..2
 0001:0001FCFC       ovcdbplb..TOvcDbPictureLabel
 0001:000208E0       ovcdbplb.Finalization
 0002:00000224       ovcdbplb.ovcdbplb
 0001:00020378       ovcdbplb.TOvcDbPictureLabel.CMGetDataLink
 0001:00020384       ovcdbplb.TOvcDbPictureLabel.Create
 0001:000203F8       ovcdbplb.TOvcDbPictureLabel.Destroy
 0001:00020868       ovcdbplb.TOvcDbPictureLabel.ExecuteAction
 0001:00020430       ovcdbplb.TOvcDbPictureLabel.GetDataField
 0001:0002044C       ovcdbplb.TOvcDbPictureLabel.GetDataSource
 0001:00020460       ovcdbplb.TOvcDbPictureLabel.GetField
 0001:0002046C       ovcdbplb.TOvcDbPictureLabel.Notification
 0001:000204A8       ovcdbplb.TOvcDbPictureLabel.Paint
 0001:000205CC       ovcdbplb.TOvcDbPictureLabel.plDataChange
 0001:000205D4       ovcdbplb.TOvcDbPictureLabel.plGetFieldValue
 0001:00020794       ovcdbplb.TOvcDbPictureLabel.plGetSampleDisplayData
 0001:000207CC       ovcdbplb.TOvcDbPictureLabel.SetDataField
 0001:00020820       ovcdbplb.TOvcDbPictureLabel.SetDataSource
 0001:00020844       ovcdbplb.TOvcDbPictureLabel.SetShowDateOrTime
 0001:000208A4       ovcdbplb.TOvcDbPictureLabel.UpdateAction
 0004:00000068       ovcdbrpv..4
 0001:00020F70       ovcdbrpv..TOvcDbReportView
 0001:00020CB8       ovcdbrpv..TOvcDbRvDataLink
 0001:00020D98       ovcdbrpv..TOvcDbRvField
 0001:00021AD8       ovcdbrpv..TOvcDbRVListBox
 0001:00023764       ovcdbrpv.Finalization
 0003:00000088       ovcdbrpv.InReload
 0002:0000023C       ovcdbrpv.ovcdbrpv
 0001:00021D00       ovcdbrpv.TOvcDbReportView.ActiveChanged
 0001:00021D48       ovcdbrpv.TOvcDbReportView.AssignStructure
 0001:00021E30       ovcdbrpv.TOvcDbReportView.BindViews
 0001:00021F58       ovcdbrpv.TOvcDbReportView.BuildFieldTable
 0001:0002230C       ovcdbrpv.TOvcDbReportView.ClearAll
 0001:00022378       ovcdbrpv.TOvcDbReportView.ClearBindings
 0001:000223E4       ovcdbrpv.TOvcDbReportView.ClearDataList
 0001:00021F18       ovcdbrpv.TOvcDbReportView.ClearTableFields
 0001:000224A0       ovcdbrpv.TOvcDbReportView.Click
 0001:000224D0       ovcdbrpv.TOvcDbReportView.Create
 0001:000236F4       ovcdbrpv.TOvcDbReportView.CreateListBox
 0001:000225E4       ovcdbrpv.TOvcDbReportView.CreateValidFieldName
 0001:00023578       ovcdbrpv.TOvcDbReportView.DataSetChanged
 0001:000235B0       ovcdbrpv.TOvcDbReportView.DataSetScrolled
 0001:0002278C       ovcdbrpv.TOvcDbReportView.DblClick
 0001:00022708       ovcdbrpv.TOvcDbReportView.Destroy
 0001:000227BC       ovcdbrpv.TOvcDbReportView.DoBusy
 0001:00022810       ovcdbrpv.TOvcDbReportView.DoCompareFields
 0001:00023748       ovcdbrpv.TOvcDbReportView.DoDetail
 0001:0002368C       ovcdbrpv.TOvcDbReportView.DoDrawViewField
 0001:00022B8C       ovcdbrpv.TOvcDbReportView.DoEnumEvent
 0001:00022BC8       ovcdbrpv.TOvcDbReportView.DoGetFieldAsFloat
 0001:00022C50       ovcdbrpv.TOvcDbReportView.DoGetFieldAsString
 0001:00022CDC       ovcdbrpv.TOvcDbReportView.DoGetFieldValue
 0001:00022D3C       ovcdbrpv.TOvcDbReportView.DoGetGroupString
 0001:00022E84       ovcdbrpv.TOvcDbReportView.DoKeySearch
 0001:00022F14       ovcdbrpv.TOvcDbReportView.Enumerate
 0001:00022FA8       ovcdbrpv.TOvcDbReportView.EnumerateEx
 0001:00022F3C       ovcdbrpv.TOvcDbReportView.EnumerateSelected
 0001:00023500       ovcdbrpv.TOvcDbReportView.ExecuteAction
 0001:0002301C       ovcdbrpv.TOvcDbReportView.GetDataSource
 0001:00023030       ovcdbrpv.TOvcDbReportView.GetFieldClassType
 0001:00023038       ovcdbrpv.TOvcDbReportView.InternalRecordCount
 0001:000235E0       ovcdbrpv.TOvcDbReportView.Loaded
 0001:000223F0       ovcdbrpv.TOvcDbReportView.MoveDataPointer
 0001:000235F4       ovcdbrpv.TOvcDbReportView.Notification
 0001:00023144       ovcdbrpv.TOvcDbReportView.RecordChanged
 0001:0002314C       ovcdbrpv.TOvcDbReportView.ReloadData
 0001:000232D0       ovcdbrpv.TOvcDbReportView.SetDataSource
 0001:0002331C       ovcdbrpv.TOvcDbReportView.SetName
 0001:0002353C       ovcdbrpv.TOvcDbReportView.UpdateAction
 0001:00022440       ovcdbrpv.TOvcDbReportView.UpdateCurrentSelection
 0001:00021CB4       ovcdbrpv.TOvcDbRvDataLink.ActiveChanged
 0001:00021C78       ovcdbrpv.TOvcDbRvDataLink.Create
 0001:00021CCC       ovcdbrpv.TOvcDbRvDataLink.DataSetChanged
 0001:00021CD8       ovcdbrpv.TOvcDbRvDataLink.DataSetScrolled
 0001:00021CE8       ovcdbrpv.TOvcDbRvDataLink.LayoutChanged
 0001:00021CE4       ovcdbrpv.TOvcDbRvDataLink.RecordChanged
 0001:00021CC0       ovcdbrpv.TOvcDbRvDataLink.UpdateData
 0001:00023704       ovcdbrpv.TOvcDbRVListBox.Paint
 0004:0000006C       ovcdbsed..3
 0001:0002389C       ovcdbsed..TOvcCustomDbSliderEdit
 0001:00023A84       ovcdbsed..TOvcDbSliderEdit
 0001:00024ECC       ovcdbsed.Finalization
 0002:00000244       ovcdbsed.ovcdbsed
 0003:0000008C       ovcdbsed.SupportedFieldTypes
 0001:000243A0       ovcdbsed.TOvcCustomDbSliderEdit.Change
 0001:000243B8       ovcdbsed.TOvcCustomDbSliderEdit.CMEnter
 0001:000243D4       ovcdbsed.TOvcCustomDbSliderEdit.CMExit
 0001:0002445C       ovcdbsed.TOvcCustomDbSliderEdit.CMGetDataLink
 0001:00024468       ovcdbsed.TOvcCustomDbSliderEdit.Create
 0001:000244FC       ovcdbsed.TOvcCustomDbSliderEdit.DataChange
 0001:000246B4       ovcdbsed.TOvcCustomDbSliderEdit.Destroy
 0001:00024700       ovcdbsed.TOvcCustomDbSliderEdit.EditingChange
 0001:00024E54       ovcdbsed.TOvcCustomDbSliderEdit.ExecuteAction
 0001:00024734       ovcdbsed.TOvcCustomDbSliderEdit.GetButtonEnabled
 0001:00024768       ovcdbsed.TOvcCustomDbSliderEdit.GetDataField
 0001:00024784       ovcdbsed.TOvcCustomDbSliderEdit.GetDataSource
 0001:00024790       ovcdbsed.TOvcCustomDbSliderEdit.GetField
 0001:0002479C       ovcdbsed.TOvcCustomDbSliderEdit.GetReadOnly
 0001:000247C8       ovcdbsed.TOvcCustomDbSliderEdit.GetTextMargins
 0001:00024890       ovcdbsed.TOvcCustomDbSliderEdit.KeyDown
 0001:000248C8       ovcdbsed.TOvcCustomDbSliderEdit.KeyPress
 0001:00024978       ovcdbsed.TOvcCustomDbSliderEdit.Notification
 0001:000249B4       ovcdbsed.TOvcCustomDbSliderEdit.PopupClose
 0001:000249E4       ovcdbsed.TOvcCustomDbSliderEdit.PopupOpen
 0001:000249FC       ovcdbsed.TOvcCustomDbSliderEdit.SetDataField
 0001:00024A94       ovcdbsed.TOvcCustomDbSliderEdit.SetDataSource
 0001:00024AB8       ovcdbsed.TOvcCustomDbSliderEdit.SetFocused
 0001:00024AEC       ovcdbsed.TOvcCustomDbSliderEdit.SetReadOnly
 0001:00024E90       ovcdbsed.TOvcCustomDbSliderEdit.UpdateAction
 0001:00024AF8       ovcdbsed.TOvcCustomDbSliderEdit.UpdateData
 0001:00024B98       ovcdbsed.TOvcCustomDbSliderEdit.WMCut
 0001:00024BB8       ovcdbsed.TOvcCustomDbSliderEdit.WMPaint
 0001:00024E34       ovcdbsed.TOvcCustomDbSliderEdit.WMPaste
 0004:0000002C       ovcdbsf..2
 0001:00008AC8       ovcdbsf..TOvcDbSimpleField
 0001:00009EA4       ovcdbsf.FieldIsZero
 0001:0000ADD0       ovcdbsf.Finalization
 0002:000001AC       ovcdbsf.ovcdbsf
 0003:00000040       ovcdbsf.SupportedFieldTypes
 0001:000095E4       ovcdbsf.TOvcDbSimpleField.CMEnter
 0001:00009600       ovcdbsf.TOvcDbSimpleField.CMExit
 0001:00009608       ovcdbsf.TOvcDbSimpleField.CMGetDataLink
 0001:00009614       ovcdbsf.TOvcDbSimpleField.Create
 0001:000096B4       ovcdbsf.TOvcDbSimpleField.CreateWnd
 0001:000096E4       ovcdbsf.TOvcDbSimpleField.CutToClipboard
 0001:00009764       ovcdbsf.TOvcDbSimpleField.Destroy
 0001:000097B0       ovcdbsf.TOvcDbSimpleField.DoOnChange
 0001:000097DC       ovcdbsf.TOvcDbSimpleField.efEdit
 0001:00009858       ovcdbsf.TOvcDbSimpleField.efGetSampleDisplayData
 0001:000099D4       ovcdbsf.TOvcDbSimpleField.efIncDecValue
 0001:00009A4C       ovcdbsf.TOvcDbSimpleField.efIsReadOnly
 0001:0000AD58       ovcdbsf.TOvcDbSimpleField.ExecuteAction
 0001:00009AD0       ovcdbsf.TOvcDbSimpleField.GetDataField
 0001:00009AEC       ovcdbsf.TOvcDbSimpleField.GetDataSource
 0001:00009B00       ovcdbsf.TOvcDbSimpleField.GetField
 0001:00009B80       ovcdbsf.TOvcDbSimpleField.Notification
 0001:00009BC8       ovcdbsf.TOvcDbSimpleField.PasteFromClipboard
 0001:00009C48       ovcdbsf.TOvcDbSimpleField.Restore
 0001:00009C68       ovcdbsf.TOvcDbSimpleField.SetDataField
 0001:00009D20       ovcdbsf.TOvcDbSimpleField.SetDataSource
 0001:00009D54       ovcdbsf.TOvcDbSimpleField.SetFieldType
 0001:00009DF4       ovcdbsf.TOvcDbSimpleField.SetUseTFieldMask
 0001:00009E0C       ovcdbsf.TOvcDbSimpleField.SetZeroAsNull
 0001:00009E1C       ovcdbsf.TOvcDbSimpleField.sfdbDataChange
 0001:00009E80       ovcdbsf.TOvcDbSimpleField.sfdbEditingChange
 0001:00009F6C       ovcdbsf.TOvcDbSimpleField.sfdbGetFieldValue
 0001:0000A1CC       ovcdbsf.TOvcDbSimpleField.sfdbSetFieldProperties
 0001:0000A2FC       ovcdbsf.TOvcDbSimpleField.sfdbSetFieldValue
 0001:0000A704       ovcdbsf.TOvcDbSimpleField.sfdbUpdateData
 0001:0000AD94       ovcdbsf.TOvcDbSimpleField.UpdateAction
 0001:0000A7D4       ovcdbsf.TOvcDbSimpleField.WMKeyDown
 0001:0000A8D8       ovcdbsf.TOvcDbSimpleField.WMKillFocus
 0001:0000A940       ovcdbsf.TOvcDbSimpleField.WMLButtonDblClk
 0001:0000A954       ovcdbsf.TOvcDbSimpleField.WMLButtonDown
 0001:0000A970       ovcdbsf.TOvcDbSimpleField.WMLButtonUp
 0001:0000A990       ovcdbsf.TOvcDbSimpleField.WMPaint
 0001:0000AD2C       ovcdbsf.TOvcDbSimpleField.WMSetFocus
 0004:00000070       ovcdbsld..2
 0001:00024EFC       ovcdbsld..TOvcDbSlider
 0001:00025AF8       ovcdbsld.Finalization
 0002:0000024C       ovcdbsld.ovcdbsld
 0003:00000094       ovcdbsld.SupportedFieldTypes
 0001:0002562C       ovcdbsld.TOvcDbSlider.CMExit
 0001:00025690       ovcdbsld.TOvcDbSlider.CMGetDataLink
 0001:0002569C       ovcdbsld.TOvcDbSlider.Create
 0001:00025710       ovcdbsld.TOvcDbSlider.Destroy
 0001:00025748       ovcdbsld.TOvcDbSlider.DoOnChange
 0001:00025A80       ovcdbsld.TOvcDbSlider.ExecuteAction
 0001:00025760       ovcdbsld.TOvcDbSlider.GetDataField
 0001:0002577C       ovcdbsld.TOvcDbSlider.GetDataSource
 0001:00025790       ovcdbsld.TOvcDbSlider.GetField
 0001:0002579C       ovcdbsld.TOvcDbSlider.Notification
 0001:000257E0       ovcdbsld.TOvcDbSlider.SetDataField
 0001:00025954       ovcdbsld.TOvcDbSlider.SetDataSource
 0001:00025980       ovcdbsld.TOvcDbSlider.slDataChange
 0001:000259C0       ovcdbsld.TOvcDbSlider.slUpdateData
 0001:00025ABC       ovcdbsld.TOvcDbSlider.UpdateAction
 0001:00025A3C       ovcdbsld.TOvcDbSlider.WMKeyDown
 0001:000259F8       ovcdbsld.TOvcDbSlider.WMLButtonDown
 0004:00000074       ovcdbtbl..6
 0001:00026174       ovcdbtbl..TOvcCustomDbTable
 0001:00026400       ovcdbtbl..TOvcDbTable
 0001:00025F90       ovcdbtbl..TOvcDbTableColumn
 0001:00025EAC       ovcdbtbl..TOvcDbTableDataLink
 0001:00026088       ovcdbtbl..TOvcVisibleColumns
 0001:00028FA8       ovcdbtbl.DrawEffects
 0001:00030858       ovcdbtbl.Finalization
 0001:0002E5AC       ovcdbtbl.GetColumnWidth
 0002:0000025C       ovcdbtbl.ovcdbtbl
 0001:000290A4       ovcdbtbl.PaintString
 0003:0000009C       ovcdbtbl.SupportedFieldTypes
 0001:00027578       ovcdbtbl.TOvcCustomDbTable.CalcRowCol
 0001:000277A0       ovcdbtbl.TOvcCustomDbTable.ChangeScale
 0001:00027810       ovcdbtbl.TOvcCustomDbTable.CMColorChanged
 0001:00027824       ovcdbtbl.TOvcCustomDbTable.CMCtl3DChanged
 0001:00027864       ovcdbtbl.TOvcCustomDbTable.CMDesignHitTest
 0001:000278D0       ovcdbtbl.TOvcCustomDbTable.CMFontChanged
 0001:000278F4       ovcdbtbl.TOvcCustomDbTable.Create
 0001:00027CCC       ovcdbtbl.TOvcCustomDbTable.CreateParams
 0001:00027D30       ovcdbtbl.TOvcCustomDbTable.CreateWnd
 0001:00027DE4       ovcdbtbl.TOvcCustomDbTable.ctimKillFocus
 0001:00027ED4       ovcdbtbl.TOvcCustomDbTable.ctimQueryActiveCol
 0001:00027EE0       ovcdbtbl.TOvcCustomDbTable.ctimQueryActiveRow
 0001:00027EB0       ovcdbtbl.TOvcCustomDbTable.ctimQueryColor
 0001:00027EB8       ovcdbtbl.TOvcCustomDbTable.ctimQueryFont
 0001:00027EC0       ovcdbtbl.TOvcCustomDbTable.ctimQueryLockedCols
 0001:00027ECC       ovcdbtbl.TOvcCustomDbTable.ctimQueryLockedRows
 0001:00027E44       ovcdbtbl.TOvcCustomDbTable.ctimQueryOptions
 0001:00027EEC       ovcdbtbl.TOvcCustomDbTable.ctimRemoveCell
 0001:00027F04       ovcdbtbl.TOvcCustomDbTable.ctimSetFocus
 0001:00027F14       ovcdbtbl.TOvcCustomDbTable.ctimStartEdit
 0001:00027FF4       ovcdbtbl.TOvcCustomDbTable.ctimStartEditKey
 0001:00027F38       ovcdbtbl.TOvcCustomDbTable.ctimStartEditMouse
 0001:0002804C       ovcdbtbl.TOvcCustomDbTable.DefineProperties
 0001:00028088       ovcdbtbl.TOvcCustomDbTable.Destroy
 0001:00028158       ovcdbtbl.TOvcCustomDbTable.DoOnActiveCellChanged
 0001:000281A0       ovcdbtbl.TOvcCustomDbTable.DoOnColumnMoved
 0001:000281E8       ovcdbtbl.TOvcCustomDbTable.DoOnGetCellAttributes
 0001:0002823C       ovcdbtbl.TOvcCustomDbTable.DoOnIndicatorClick
 0001:00028264       ovcdbtbl.TOvcCustomDbTable.DoOnLeftColumnChanged
 0001:000282A0       ovcdbtbl.TOvcCustomDbTable.DoOnLockedCellClick
 0001:000282E8       ovcdbtbl.TOvcCustomDbTable.DoOnMouseWheel
 0001:00028330       ovcdbtbl.TOvcCustomDbTable.DoOnPaintUnusedArea
 0001:00028378       ovcdbtbl.TOvcCustomDbTable.DoOnUnusedAreaClick
 0001:000283C0       ovcdbtbl.TOvcCustomDbTable.DoOnUserCommand
 0001:00028404       ovcdbtbl.TOvcCustomDbTable.FilterKey
 0001:000284D4       ovcdbtbl.TOvcCustomDbTable.GetColumnCount
 0001:0002851C       ovcdbtbl.TOvcCustomDbTable.GetColumnOrder
 0001:000284E0       ovcdbtbl.TOvcCustomDbTable.GetColumnOrderStrings
 0001:000285F0       ovcdbtbl.TOvcCustomDbTable.GetColumnWidths
 0001:00028570       ovcdbtbl.TOvcCustomDbTable.GetColumnWidthsStrings
 0001:0002863C       ovcdbtbl.TOvcCustomDbTable.GetDataSource
 0001:00028650       ovcdbtbl.TOvcCustomDbTable.GetFieldCount
 0001:0002865C       ovcdbtbl.TOvcCustomDbTable.GetFields
 0001:00028668       ovcdbtbl.TOvcCustomDbTable.GetSelectedField
 0001:0002868C       ovcdbtbl.TOvcCustomDbTable.GetVisibleColumnCount
 0001:00028698       ovcdbtbl.TOvcCustomDbTable.IncCol
 0001:00028730       ovcdbtbl.TOvcCustomDbTable.IncRow
 0001:00028750       ovcdbtbl.TOvcCustomDbTable.InEditingState
 0001:0002875C       ovcdbtbl.TOvcCustomDbTable.InvalidateCell
 0001:000287A4       ovcdbtbl.TOvcCustomDbTable.InvalidateColumn
 0001:000287D4       ovcdbtbl.TOvcCustomDbTable.InvalidateHeader
 0001:00028828       ovcdbtbl.TOvcCustomDbTable.InvalidateIndicators
 0001:00028878       ovcdbtbl.TOvcCustomDbTable.InvalidateNotLocked
 0001:000288F8       ovcdbtbl.TOvcCustomDbTable.InvalidateRow
 0001:00028934       ovcdbtbl.TOvcCustomDbTable.InvalidateUnusedArea
 0001:000289B8       ovcdbtbl.TOvcCustomDbTable.Loaded
 0001:00028A2C       ovcdbtbl.TOvcCustomDbTable.MakeColumnVisible
 0001:00028B14       ovcdbtbl.TOvcCustomDbTable.MoveActiveCell
 0001:00028E34       ovcdbtbl.TOvcCustomDbTable.Notification
 0001:0002914C       ovcdbtbl.TOvcCustomDbTable.Paint
 0001:0002A16C       ovcdbtbl.TOvcCustomDbTable.ResolveCellAttributes
 0001:0002A2C8       ovcdbtbl.TOvcCustomDbTable.SaveEditedData
 0001:0002A3C0       ovcdbtbl.TOvcCustomDbTable.Scroll
 0001:0002A3E8       ovcdbtbl.TOvcCustomDbTable.SetAccess
 0001:0002A420       ovcdbtbl.TOvcCustomDbTable.SetActiveCell
 0001:0002A5E8       ovcdbtbl.TOvcCustomDbTable.SetActiveColumn
 0001:0002A5F8       ovcdbtbl.TOvcCustomDbTable.SetActiveRow
 0001:0002A604       ovcdbtbl.TOvcCustomDbTable.SetAdjust
 0001:0002A630       ovcdbtbl.TOvcCustomDbTable.SetBorderStyle
 0001:0002A644       ovcdbtbl.TOvcCustomDbTable.SetBounds
 0001:0002A6E0       ovcdbtbl.TOvcCustomDbTable.SetCellProperties
 0001:0002AF9C       ovcdbtbl.TOvcCustomDbTable.SetColors
 0001:0002AFAC       ovcdbtbl.TOvcCustomDbTable.SetColorUnused
 0001:0002ABF8       ovcdbtbl.TOvcCustomDbTable.SetColumnCount
 0001:0002AD88       ovcdbtbl.TOvcCustomDbTable.SetColumnOrder
 0001:0002AC2C       ovcdbtbl.TOvcCustomDbTable.SetColumnOrderStrings
 0001:0002AFC4       ovcdbtbl.TOvcCustomDbTable.SetColumns
 0001:0002AF44       ovcdbtbl.TOvcCustomDbTable.SetColumnWidths
 0001:0002AE80       ovcdbtbl.TOvcCustomDbTable.SetColumnWidthsStrings
 0001:0002AFE4       ovcdbtbl.TOvcCustomDbTable.SetDataSource
 0001:0002B0D0       ovcdbtbl.TOvcCustomDbTable.SetDefaultMargin
 0001:0002B1DC       ovcdbtbl.TOvcCustomDbTable.SetHeaderCell
 0001:0002B328       ovcdbtbl.TOvcCustomDbTable.SetHeaderHeight
 0001:0002B38C       ovcdbtbl.TOvcCustomDbTable.SetHeaderOptions
 0001:0002B4EC       ovcdbtbl.TOvcCustomDbTable.SetLeftColumn
 0001:0002B0EC       ovcdbtbl.TOvcCustomDbTable.SetLinkActive
 0001:0002B534       ovcdbtbl.TOvcCustomDbTable.SetLockedColumns
 0001:0002B5CC       ovcdbtbl.TOvcCustomDbTable.SetOptions
 0001:0002B788       ovcdbtbl.TOvcCustomDbTable.SetRowHeight
 0001:0002B7D4       ovcdbtbl.TOvcCustomDbTable.SetRowIndicatorWidth
 0001:0002B860       ovcdbtbl.TOvcCustomDbTable.SetScrollBars
 0001:0002B874       ovcdbtbl.TOvcCustomDbTable.SetSelectedField
 0001:0002B8B0       ovcdbtbl.TOvcCustomDbTable.SetTextStyle
 0001:0002B8C8       ovcdbtbl.TOvcCustomDbTable.StartEditing
 0001:0002BC5C       ovcdbtbl.TOvcCustomDbTable.StopEditing
 0001:0002BE38       ovcdbtbl.TOvcCustomDbTable.tbAdjustIntegralHeight
 0001:0002BEA0       ovcdbtbl.TOvcCustomDbTable.tbCalcActiveCellRect
 0001:0002BF20       ovcdbtbl.TOvcCustomDbTable.tbCalcCellRect
 0001:0002BFBC       ovcdbtbl.TOvcCustomDbTable.tbCalcColumnRect
 0001:0002C038       ovcdbtbl.TOvcCustomDbTable.tbCalcColumnsOnLastPage
 0001:0002C26C       ovcdbtbl.TOvcCustomDbTable.tbCalcRowBottom
 0001:0002C0E0       ovcdbtbl.TOvcCustomDbTable.tbCalcRowColData
 0001:0002C204       ovcdbtbl.TOvcCustomDbTable.tbCalcRowRect
 0001:0002C240       ovcdbtbl.TOvcCustomDbTable.tbCalcRowTop
 0001:0002C284       ovcdbtbl.TOvcCustomDbTable.tbCalcVisibleRows
 0001:0002C2C8       ovcdbtbl.TOvcCustomDbTable.tbCanModify
 0001:0002C458       ovcdbtbl.TOvcCustomDbTable.tbCellChanged
 0001:0002C488       ovcdbtbl.TOvcCustomDbTable.tbCellModified
 0001:0002C534       ovcdbtbl.TOvcCustomDbTable.tbColorsChanged
 0001:0002C564       ovcdbtbl.TOvcCustomDbTable.tbColumnAtRight
 0001:0002C588       ovcdbtbl.TOvcCustomDbTable.tbColumnChanged
 0001:0002C854       ovcdbtbl.TOvcCustomDbTable.tbDataChanged
 0001:0002C8DC       ovcdbtbl.TOvcCustomDbTable.tbDefineFieldMap
 0001:0002C9FC       ovcdbtbl.TOvcCustomDbTable.tbDrawActiveCell
 0001:0002CEBC       ovcdbtbl.TOvcCustomDbTable.tbDrawMoveLine
 0001:0002D00C       ovcdbtbl.TOvcCustomDbTable.tbDrawSizeLine
 0001:0002D0E4       ovcdbtbl.TOvcCustomDbTable.tbDrawUnusedArea
 0001:0002D1D4       ovcdbtbl.TOvcCustomDbTable.tbEditCellHasFocus
 0001:0002D240       ovcdbtbl.TOvcCustomDbTable.tbEditingChanged
 0001:0002D2B4       ovcdbtbl.TOvcCustomDbTable.tbFindCell
 0001:0002D2E4       ovcdbtbl.TOvcCustomDbTable.tbGetDataSize
 0001:0002D3E8       ovcdbtbl.TOvcCustomDbTable.tbGetFieldColumn
 0001:0002D428       ovcdbtbl.TOvcCustomDbTable.tbGetFieldValue
 0001:0002D924       ovcdbtbl.TOvcCustomDbTable.tbGridPenChanged
 0001:0002DA1C       ovcdbtbl.TOvcCustomDbTable.tbIsColumnHidden
 0001:0002D9F0       ovcdbtbl.TOvcCustomDbTable.tbIsDbActive
 0001:0002DA84       ovcdbtbl.TOvcCustomDbTable.tbIsInMoveArea
 0001:0002D954       ovcdbtbl.TOvcCustomDbTable.tbIsOnGridLine
 0001:0002DBC0       ovcdbtbl.TOvcCustomDbTable.tbIsSibling
 0001:0002DB10       ovcdbtbl.TOvcCustomDbTable.tbLayoutChanged
 0001:0002DC0C       ovcdbtbl.TOvcCustomDbTable.tbLoading
 0001:0002DC44       ovcdbtbl.TOvcCustomDbTable.tbMoveActCellPageLeft
 0001:0002DD10       ovcdbtbl.TOvcCustomDbTable.tbMoveActCellPageRight
 0001:0002DDE4       ovcdbtbl.TOvcCustomDbTable.tbPaintBitmapCell
 0001:0002E048       ovcdbtbl.TOvcCustomDbTable.tbPaintString
 0001:0002E35C       ovcdbtbl.TOvcCustomDbTable.tbQueryColData
 0001:0002E3E4       ovcdbtbl.TOvcCustomDbTable.tbReadColData
 0001:0002E73C       ovcdbtbl.TOvcCustomDbTable.tbRebuildColumns
 0001:0002E4FC       ovcdbtbl.TOvcCustomDbTable.tbRecordChanged
 0001:0002E8B4       ovcdbtbl.TOvcCustomDbTable.tbScrollBarPageLeft
 0001:0002E948       ovcdbtbl.TOvcCustomDbTable.tbScrollBarPageRight
 0001:0002E998       ovcdbtbl.TOvcCustomDbTable.tbScrollNotification
 0001:0002EB28       ovcdbtbl.TOvcCustomDbTable.tbScrollTableLeft
 0001:0002EC60       ovcdbtbl.TOvcCustomDbTable.tbScrollTableRight
 0001:0002ED28       ovcdbtbl.TOvcCustomDbTable.tbSetFieldValue
 0001:0002F2F4       ovcdbtbl.TOvcCustomDbTable.tbSetFocus
 0001:0002F300       ovcdbtbl.TOvcCustomDbTable.tbUpdateActive
 0001:0002F324       ovcdbtbl.TOvcCustomDbTable.tbUpdateBufferLimit
 0001:0002F3EC       ovcdbtbl.TOvcCustomDbTable.tbUpdateHScrollBar
 0001:0002F480       ovcdbtbl.TOvcCustomDbTable.tbUpdateVScrollBar
 0001:0002F5EC       ovcdbtbl.TOvcCustomDbTable.tbWriteColData
 0001:0002F684       ovcdbtbl.TOvcCustomDbTable.UpdateData
 0001:0002F69C       ovcdbtbl.TOvcCustomDbTable.WMCommand
 0001:0002F7E0       ovcdbtbl.TOvcCustomDbTable.WMEraseBkGnd
 0001:0002F7E8       ovcdbtbl.TOvcCustomDbTable.WMGetDlgCode
 0001:0002F80C       ovcdbtbl.TOvcCustomDbTable.WMHScroll
 0001:0002F930       ovcdbtbl.TOvcCustomDbTable.WMKeyDown
 0001:0002FB54       ovcdbtbl.TOvcCustomDbTable.WMKillFocus
 0001:0002FB7C       ovcdbtbl.TOvcCustomDbTable.WMLButtonDblClk
 0001:0002FC18       ovcdbtbl.TOvcCustomDbTable.WMLButtonDown
 0001:00030014       ovcdbtbl.TOvcCustomDbTable.WMLButtonUp
 0001:000302A8       ovcdbtbl.TOvcCustomDbTable.WMMouseMove
 0001:0003036C       ovcdbtbl.TOvcCustomDbTable.WMNCHitTest
 0001:00030388       ovcdbtbl.TOvcCustomDbTable.WMSetCursor
 0001:00030534       ovcdbtbl.TOvcCustomDbTable.WMSetFocus
 0001:000305DC       ovcdbtbl.TOvcCustomDbTable.WMSize
 0001:000305F0       ovcdbtbl.TOvcCustomDbTable.WMVScroll
 0001:000271BC       ovcdbtbl.TOvcDbTableColumn.Assign
 0001:000271F8       ovcdbtbl.TOvcDbTableColumn.Create
 0001:00027234       ovcdbtbl.TOvcDbTableColumn.GetField
 0001:000272EC       ovcdbtbl.TOvcDbTableColumn.GetTable
 0001:000272F0       ovcdbtbl.TOvcDbTableColumn.SetDataField
 0001:000273A4       ovcdbtbl.TOvcDbTableColumn.SetDateOrTime
 0001:000273E8       ovcdbtbl.TOvcDbTableColumn.SetField
 0001:00026E50       ovcdbtbl.TOvcDbTableDataLink.ActiveChanged
 0001:00026E60       ovcdbtbl.TOvcDbTableDataLink.AddMapping
 0001:00026FA8       ovcdbtbl.TOvcDbTableDataLink.ClearFieldMappings
 0001:00026FD4       ovcdbtbl.TOvcDbTableDataLink.Create
 0001:000270E0       ovcdbtbl.TOvcDbTableDataLink.DataSetChanged
 0001:000270F4       ovcdbtbl.TOvcDbTableDataLink.DataSetScrolled
 0001:00027010       ovcdbtbl.TOvcDbTableDataLink.Destroy
 0001:00027100       ovcdbtbl.TOvcDbTableDataLink.EditingChanged
 0001:0002703C       ovcdbtbl.TOvcDbTableDataLink.GetDefaultFields
 0001:00027060       ovcdbtbl.TOvcDbTableDataLink.GetFields
 0001:0002710C       ovcdbtbl.TOvcDbTableDataLink.LayoutChanged
 0001:00027118       ovcdbtbl.TOvcDbTableDataLink.Modified
 0001:00027120       ovcdbtbl.TOvcDbTableDataLink.RecordChanged
 0001:0002713C       ovcdbtbl.TOvcDbTableDataLink.Reset
 0001:00027164       ovcdbtbl.TOvcDbTableDataLink.UpdateData
 0001:00027408       ovcdbtbl.TOvcVisibleColumns.Add
 0001:00027418       ovcdbtbl.TOvcVisibleColumns.Clear
 0001:00027424       ovcdbtbl.TOvcVisibleColumns.Create
 0001:00027470       ovcdbtbl.TOvcVisibleColumns.Delete
 0001:0002747C       ovcdbtbl.TOvcVisibleColumns.Destroy
 0001:000274B8       ovcdbtbl.TOvcVisibleColumns.Exchange
 0001:000274F8       ovcdbtbl.TOvcVisibleColumns.GetColumn
 0001:0002751C       ovcdbtbl.TOvcVisibleColumns.GetCount
 0001:000274C4       ovcdbtbl.TOvcVisibleColumns.IndexOf
 0001:00027524       ovcdbtbl.TOvcVisibleColumns.Insert
 0001:00027544       ovcdbtbl.TOvcVisibleColumns.Move
 0004:00000018       ovcdbtcb..2
 0001:00001C5C       ovcdbtcb..TOvcDbTableNameComboBox
 0001:0000263C       ovcdbtcb.Finalization
 0002:00000144       ovcdbtcb.ovcdbtcb
 0001:000025A0       ovcdbtcb.TOvcDbTableNameComboBox.GetTableName
 0001:00002560       ovcdbtcb.TOvcDbTableNameComboBox.Loaded
 0001:000025DC       ovcdbtcb.TOvcDbTableNameComboBox.Notification
 0001:0000257C       ovcdbtcb.TOvcDbTableNameComboBox.Populate
 0001:00002610       ovcdbtcb.TOvcDbTableNameComboBox.SetAliasName
 0004:00000078       ovcdbtim..3
 0001:000308C0       ovcdbtim..TOvcCustomDbTimeEdit
 0001:00030A90       ovcdbtim..TOvcDbTimeEdit
 0001:000320F8       ovcdbtim.Finalization
 0002:00000264       ovcdbtim.ovcdbtim
 0003:000000A4       ovcdbtim.TimeFieldTypes
 0001:000314CC       ovcdbtim.TOvcCustomDbTimeEdit.Change
 0001:000314E4       ovcdbtim.TOvcCustomDbTimeEdit.CMEnter
 0001:00031500       ovcdbtim.TOvcCustomDbTimeEdit.CMExit
 0001:00031588       ovcdbtim.TOvcCustomDbTimeEdit.CMGetDataLink
 0001:00031594       ovcdbtim.TOvcCustomDbTimeEdit.Create
 0001:00031628       ovcdbtim.TOvcCustomDbTimeEdit.DataChange
 0001:00031854       ovcdbtim.TOvcCustomDbTimeEdit.Destroy
 0001:000318A0       ovcdbtim.TOvcCustomDbTimeEdit.EditingChange
 0001:00032080       ovcdbtim.TOvcCustomDbTimeEdit.ExecuteAction
 0001:000318B4       ovcdbtim.TOvcCustomDbTimeEdit.GetDataField
 0001:000318D0       ovcdbtim.TOvcCustomDbTimeEdit.GetDataSource
 0001:000318DC       ovcdbtim.TOvcCustomDbTimeEdit.GetField
 0001:000318E8       ovcdbtim.TOvcCustomDbTimeEdit.GetReadOnly
 0001:00031928       ovcdbtim.TOvcCustomDbTimeEdit.GetTextMargins
 0001:000319F0       ovcdbtim.TOvcCustomDbTimeEdit.KeyDown
 0001:00031A28       ovcdbtim.TOvcCustomDbTimeEdit.KeyPress
 0001:00031ABC       ovcdbtim.TOvcCustomDbTimeEdit.Notification
 0001:00031AF8       ovcdbtim.TOvcCustomDbTimeEdit.SetDataField
 0001:00031B90       ovcdbtim.TOvcCustomDbTimeEdit.SetDataSource
 0001:00031BB4       ovcdbtim.TOvcCustomDbTimeEdit.SetFocused
 0001:00031BE8       ovcdbtim.TOvcCustomDbTimeEdit.SetReadOnly
 0001:000320BC       ovcdbtim.TOvcCustomDbTimeEdit.UpdateAction
 0001:00031BF4       ovcdbtim.TOvcCustomDbTimeEdit.UpdateData
 0001:00031DD4       ovcdbtim.TOvcCustomDbTimeEdit.WMCut
 0001:00031DF4       ovcdbtim.TOvcCustomDbTimeEdit.WMPaint
 0001:00032060       ovcdbtim.TOvcCustomDbTimeEdit.WMPaste
 0001:00000368       SysInit.@InitPkg
 0001:000003CC       SysInit.@PackageLoad
 0001:000003D8       SysInit.@PackageUnload
 0001:00000258       SysInit.AllocTlsBuffer
 0001:00000314       SysInit.ExitProcessTLS
 0001:000002DC       SysInit.ExitThreadTLS
 0001:00000220       SysInit.FreeLibrary
 0001:00000264       SysInit.GetTlsSize
 0004:00000004       SysInit.HInstance
 0001:00000338       SysInit.InitializeModule
 0001:000002B0       SysInit.InitProcessTLS
 0001:0000026C       SysInit.InitThreadTLS
 0001:00000228       SysInit.LocalAlloc
 0001:00000230       SysInit.LocalFree
 0003:00000008       SysInit.Module
 0004:00000000       SysInit.ModuleIsLib
 0004:00000001       SysInit.ModuleIsPackage
 0003:00000004       SysInit.PtrToNil
 0001:00000238       SysInit.TlsAlloc
 0004:00000008       SysInit.tlsBuffer
 0001:00000240       SysInit.TlsFree
 0001:00000248       SysInit.TlsGetValue
 0003:00000000       SysInit.TlsIndex
 0005:00000000       SysInit.TlsLast
 0003:00000020       SysInit.TlsProc
 0001:00000250       SysInit.TlsSetValue
 0001:00000344       SysInit.UninitializeModule
 0004:0000000C       Windows..3
 0001:0000045C       Windows.BeginPaint
 0001:000003F4       Windows.CreateRectRgn
 0001:000003FC       Windows.DeleteObject
 0001:00000464       Windows.DrawText
 0001:0000046C       Windows.EndPaint
 0001:00000404       Windows.ExcludeClipRect
 0001:0000040C       Windows.ExtTextOut
 0001:00000550       Windows.Finalization
 0001:000003E4       Windows.FreeLibrary
 0001:00000474       Windows.GetAsyncKeyState
 0001:00000414       Windows.GetBkMode
 0001:0000041C       Windows.GetClipBox
 0001:0000047C       Windows.GetCursorPos
 0001:00000484       Windows.GetDC
 0001:0000048C       Windows.GetFocus
 0001:00000494       Windows.GetParent
 0001:0000049C       Windows.GetScrollInfo
 0001:000004A4       Windows.GetSystemMetrics
 0001:00000424       Windows.GetTextExtentPoint32
 0001:0000042C       Windows.GetTextMetrics
 0001:000004AC       Windows.GetWindow
 0001:000004B4       Windows.GetWindowRect
 0004:00000010       Windows.HtmlHelpModule
 0001:000004BC       Windows.InflateRect
 0001:000004C4       Windows.IntersectRect
 0001:000004CC       Windows.InvalidateRect
 0001:00000544       Windows.MakeLong
 0001:000004D4       Windows.MessageBeep
 0001:000003EC       Windows.MulDiv
 0001:000004DC       Windows.OffsetRect
 0001:000004E4       Windows.PostMessage
 0001:000004EC       Windows.ReleaseDC
 0001:000004F4       Windows.ScrollWindow
 0001:00000434       Windows.SelectClipRgn
 0001:0000043C       Windows.SelectObject
 0001:000004FC       Windows.SendMessage
 0001:00000444       Windows.SetBkColor
 0001:0000044C       Windows.SetBkMode
 0001:00000504       Windows.SetCursor
 0001:0000050C       Windows.SetFocus
 0001:00000514       Windows.SetRect
 0001:0000051C       Windows.SetScrollInfo
 0001:00000524       Windows.SetScrollPos
 0001:0000052C       Windows.SetScrollRange
 0001:00000454       Windows.SetTextAlign
 0001:00000534       Windows.UpdateWindow
 0001:0000053C       Windows.ValidateRect
 0002:00000008       Windows.Windows


  Address             Publics by Value

 0001:00000220       SysInit.FreeLibrary
 0001:00000228       SysInit.LocalAlloc
 0001:00000230       SysInit.LocalFree
 0001:00000238       SysInit.TlsAlloc
 0001:00000240       SysInit.TlsFree
 0001:00000248       SysInit.TlsGetValue
 0001:00000250       SysInit.TlsSetValue
 0001:00000258       SysInit.AllocTlsBuffer
 0001:00000264       SysInit.GetTlsSize
 0001:0000026C       SysInit.InitThreadTLS
 0001:000002B0       SysInit.InitProcessTLS
 0001:000002DC       SysInit.ExitThreadTLS
 0001:00000314       SysInit.ExitProcessTLS
 0001:00000338       SysInit.InitializeModule
 0001:00000344       SysInit.UninitializeModule
 0001:00000368       SysInit.@InitPkg
 0001:000003CC       SysInit.@PackageLoad
 0001:000003D8       SysInit.@PackageUnload
 0001:000003E4       Windows.FreeLibrary
 0001:000003EC       Windows.MulDiv
 0001:000003F4       Windows.CreateRectRgn
 0001:000003FC       Windows.DeleteObject
 0001:00000404       Windows.ExcludeClipRect
 0001:0000040C       Windows.ExtTextOut
 0001:00000414       Windows.GetBkMode
 0001:0000041C       Windows.GetClipBox
 0001:00000424       Windows.GetTextExtentPoint32
 0001:0000042C       Windows.GetTextMetrics
 0001:00000434       Windows.SelectClipRgn
 0001:0000043C       Windows.SelectObject
 0001:00000444       Windows.SetBkColor
 0001:0000044C       Windows.SetBkMode
 0001:00000454       Windows.SetTextAlign
 0001:0000045C       Windows.BeginPaint
 0001:00000464       Windows.DrawText
 0001:0000046C       Windows.EndPaint
 0001:00000474       Windows.GetAsyncKeyState
 0001:0000047C       Windows.GetCursorPos
 0001:00000484       Windows.GetDC
 0001:0000048C       Windows.GetFocus
 0001:00000494       Windows.GetParent
 0001:0000049C       Windows.GetScrollInfo
 0001:000004A4       Windows.GetSystemMetrics
 0001:000004AC       Windows.GetWindow
 0001:000004B4       Windows.GetWindowRect
 0001:000004BC       Windows.InflateRect
 0001:000004C4       Windows.IntersectRect
 0001:000004CC       Windows.InvalidateRect
 0001:000004D4       Windows.MessageBeep
 0001:000004DC       Windows.OffsetRect
 0001:000004E4       Windows.PostMessage
 0001:000004EC       Windows.ReleaseDC
 0001:000004F4       Windows.ScrollWindow
 0001:000004FC       Windows.SendMessage
 0001:00000504       Windows.SetCursor
 0001:0000050C       Windows.SetFocus
 0001:00000514       Windows.SetRect
 0001:0000051C       Windows.SetScrollInfo
 0001:00000524       Windows.SetScrollPos
 0001:0000052C       Windows.SetScrollRange
 0001:00000534       Windows.UpdateWindow
 0001:0000053C       Windows.ValidateRect
 0001:00000544       Windows.MakeLong
 0001:00000550       Windows.Finalization
 0001:000018B4       ovcdbhll..TOvcDbEngineHelperBase
 0001:000019B0       ovcdbhll.TOvcDbEngineHelperBase.FindNearestKey
 0001:000019B8       ovcdbhll.TOvcDbEngineHelperBase.GetAliasNames
 0001:00001A00       ovcdbhll.TOvcDbEngineHelperBase.GetAliasPath
 0001:00001A0C       ovcdbhll.TOvcDbEngineHelperBase.GetAliasDriverName
 0001:00001A18       ovcdbhll.TOvcDbEngineHelperBase.GetTableNames
 0001:00001A60       ovcdbhll.TOvcDbEngineHelperBase.GetIndexDefs
 0001:00001A64       ovcdbhll.TOvcDbEngineHelperBase.GetIndexField
 0001:00001A68       ovcdbhll.TOvcDbEngineHelperBase.GetIndexFieldCount
 0001:00001A6C       ovcdbhll.TOvcDbEngineHelperBase.GetIndexFieldNames
 0001:00001A78       ovcdbhll.TOvcDbEngineHelperBase.GetIndexName
 0001:00001A84       ovcdbhll.TOvcDbEngineHelperBase.IsChildDataSet
 0001:00001A88       ovcdbhll.TOvcDbEngineHelperBase.SetIndexFieldNames
 0001:00001A8C       ovcdbhll.TOvcDbEngineHelperBase.SetIndexName
 0001:00001A90       ovcdbhll.OvcFindNearestKey
 0001:00001AA8       ovcdbhll.OvcGetAliasDriverName
 0001:00001AC4       ovcdbhll.OvcGetAliasNames
 0001:00001B18       ovcdbhll.OvcGetAliasPath
 0001:00001B34       ovcdbhll.OvcGetIndexDefs
 0001:00001B44       ovcdbhll.OvcGetIndexField
 0001:00001B54       ovcdbhll.OvcGetIndexFieldCount
 0001:00001B64       ovcdbhll.OvcGetIndexFieldNames
 0001:00001B80       ovcdbhll.OvcGetIndexName
 0001:00001B9C       ovcdbhll.OvcIsChildDataSet
 0001:00001BAC       ovcdbhll.OvcSetIndexFieldNames
 0001:00001BC0       ovcdbhll.OvcSetIndexName
 0001:00001BD4       ovcdbhll.OvcGetTableNames
 0001:00001C2C       ovcdbhll.Finalization
 0001:00001C5C       ovcdbtcb..TOvcDbTableNameComboBox
 0001:00002560       ovcdbtcb.TOvcDbTableNameComboBox.Loaded
 0001:0000257C       ovcdbtcb.TOvcDbTableNameComboBox.Populate
 0001:000025A0       ovcdbtcb.TOvcDbTableNameComboBox.GetTableName
 0001:000025DC       ovcdbtcb.TOvcDbTableNameComboBox.Notification
 0001:00002610       ovcdbtcb.TOvcDbTableNameComboBox.SetAliasName
 0001:0000263C       ovcdbtcb.Finalization
 0001:0000266C       ovcdbacb..TOvcDbAliasComboBox
 0001:00002F5C       ovcdbacb.TOvcDbAliasComboBox.Loaded
 0001:00002F78       ovcdbacb.TOvcDbAliasComboBox.Populate
 0001:00002F98       ovcdbacb.TOvcDbAliasComboBox.SelectionChanged
 0001:00002FF8       ovcdbacb.TOvcDbAliasComboBox.GetAliasName
 0001:00003034       ovcdbacb.TOvcDbAliasComboBox.GetPath
 0001:000030B0       ovcdbacb.TOvcDbAliasComboBox.GetDriverName
 0001:0000312C       ovcdbacb.TOvcDbAliasComboBox.Notification
 0001:00003160       ovcdbacb.Finalization
 0001:000031D0       ovcdbadg..TOvcfrmAliasDlg
 0001:000034EC       ovcdbadg..TOvcDbAliasDialog
 0001:000036F8       ovcdbadg.ExpandAlias
 0001:000038B0       ovcdbadg.TOvcDbAliasDialog.Create
 0001:00003978       ovcdbadg.TOvcDbAliasDialog.Execute
 0001:00003A50       ovcdbadg.TOvcDbAliasDialog.GetPath
 0001:00003A88       ovcdbadg.TOvcDbAliasDialog.GetTableName
 0001:00003A9C       ovcdbadg.TOvcfrmAliasDlg.btnBrowseClick
 0001:00003B30       ovcdbadg.TOvcfrmAliasDlg.cbAliasListChange
 0001:00003D24       ovcdbadg.TOvcfrmAliasDlg.edTableNameChange
 0001:00003D44       ovcdbadg.TOvcfrmAliasDlg.FileListBox1Change
 0001:00003DC0       ovcdbadg.TOvcfrmAliasDlg.FileListBox1DblClick
 0001:00003DE0       ovcdbadg.TOvcfrmAliasDlg.FormCreate
 0001:00003DFC       ovcdbadg.TOvcfrmAliasDlg.FormShow
 0001:00003E38       ovcdbadg.Finalization
 0001:00003FC0       ovcdbnf..TOvcDbNumericField
 0001:00004A48       ovcdbnf.TOvcDbNumericField.CMEnter
 0001:00004A64       ovcdbnf.TOvcDbNumericField.CMExit
 0001:00004A6C       ovcdbnf.TOvcDbNumericField.CMGetDataLink
 0001:00004A78       ovcdbnf.TOvcDbNumericField.Create
 0001:00004B18       ovcdbnf.TOvcDbNumericField.CreateWnd
 0001:00004B48       ovcdbnf.TOvcDbNumericField.CutToClipboard
 0001:00004BC8       ovcdbnf.TOvcDbNumericField.Destroy
 0001:00004C14       ovcdbnf.TOvcDbNumericField.DoOnChange
 0001:00004C40       ovcdbnf.TOvcDbNumericField.efEdit
 0001:00004CBC       ovcdbnf.TOvcDbNumericField.efGetSampleDisplayData
 0001:00004E38       ovcdbnf.TOvcDbNumericField.efIncDecValue
 0001:00004EB0       ovcdbnf.TOvcDbNumericField.efIsReadOnly
 0001:00004F34       ovcdbnf.TOvcDbNumericField.GetDataField
 0001:00004F50       ovcdbnf.TOvcDbNumericField.GetDataSource
 0001:00004F64       ovcdbnf.TOvcDbNumericField.GetField
 0001:00004FE4       ovcdbnf.TOvcDbNumericField.nfdbDataChange
 0001:00005048       ovcdbnf.TOvcDbNumericField.nfdbEditingChange
 0001:0000506C       ovcdbnf.FieldIsZero
 0001:00005120       ovcdbnf.TOvcDbNumericField.nfdbGetFieldValue
 0001:0000528C       ovcdbnf.TOvcDbNumericField.nfdbSetFieldProperties
 0001:00005348       ovcdbnf.TOvcDbNumericField.nfdbSetFieldValue
 0001:000055B8       ovcdbnf.TOvcDbNumericField.nfdbUpdateData
 0001:00005688       ovcdbnf.TOvcDbNumericField.nfSetPictureMask
 0001:000056A4       ovcdbnf.TOvcDbNumericField.Notification
 0001:000056EC       ovcdbnf.TOvcDbNumericField.PasteFromClipboard
 0001:0000576C       ovcdbnf.TOvcDbNumericField.Restore
 0001:0000578C       ovcdbnf.TOvcDbNumericField.SetDataField
 0001:00005844       ovcdbnf.TOvcDbNumericField.SetDataSource
 0001:00005878       ovcdbnf.TOvcDbNumericField.SetFieldType
 0001:00005918       ovcdbnf.TOvcDbNumericField.SetUseTFieldMask
 0001:00005930       ovcdbnf.TOvcDbNumericField.SetZeroAsNull
 0001:00005940       ovcdbnf.TOvcDbNumericField.WMKeyDown
 0001:00005A44       ovcdbnf.TOvcDbNumericField.WMKillFocus
 0001:00005AAC       ovcdbnf.TOvcDbNumericField.WMLButtonDblClk
 0001:00005AC0       ovcdbnf.TOvcDbNumericField.WMLButtonDown
 0001:00005AD4       ovcdbnf.TOvcDbNumericField.WMLButtonUp
 0001:00005AF4       ovcdbnf.TOvcDbNumericField.WMPaint
 0001:00005E7C       ovcdbnf.TOvcDbNumericField.WMSetFocus
 0001:00005EA8       ovcdbnf.TOvcDbNumericField.ExecuteAction
 0001:00005EE4       ovcdbnf.TOvcDbNumericField.UpdateAction
 0001:00005F20       ovcdbnf.Finalization
 0001:00006008       ovcdbpf..TOvcDbPictureField
 0001:00006B74       ovcdbpf.TOvcDbPictureField.CMEnter
 0001:00006B90       ovcdbpf.TOvcDbPictureField.CMExit
 0001:00006B98       ovcdbpf.TOvcDbPictureField.CMGetDataLink
 0001:00006BA4       ovcdbpf.TOvcDbPictureField.Create
 0001:00006C4C       ovcdbpf.TOvcDbPictureField.CreateWnd
 0001:00006C7C       ovcdbpf.TOvcDbPictureField.CutToClipboard
 0001:00006CFC       ovcdbpf.TOvcDbPictureField.Destroy
 0001:00006D48       ovcdbpf.TOvcDbPictureField.DoOnChange
 0001:00006D74       ovcdbpf.TOvcDbPictureField.efEdit
 0001:00006DF0       ovcdbpf.TOvcDbPictureField.efGetSampleDisplayData
 0001:00006F6C       ovcdbpf.TOvcDbPictureField.efIncDecValue
 0001:00006FE4       ovcdbpf.TOvcDbPictureField.efIsReadOnly
 0001:00007068       ovcdbpf.TOvcDbPictureField.GetDataField
 0001:00007084       ovcdbpf.TOvcDbPictureField.GetDataSource
 0001:00007098       ovcdbpf.TOvcDbPictureField.GetField
 0001:00007118       ovcdbpf.TOvcDbPictureField.Notification
 0001:00007160       ovcdbpf.TOvcDbPictureField.PasteFromClipboard
 0001:000071E0       ovcdbpf.TOvcDbPictureField.pfdbDataChange
 0001:00007244       ovcdbpf.TOvcDbPictureField.pfdbEditingChange
 0001:00007268       ovcdbpf.FieldIsZero
 0001:00007330       ovcdbpf.TOvcDbPictureField.pfdbGetFieldValue
 0001:000076E8       ovcdbpf.TOvcDbPictureField.pfdbSetFieldProperties
 0001:00007920       ovcdbpf.TOvcDbPictureField.pfdbSetFieldValue
 0001:0000808C       ovcdbpf.TOvcDbPictureField.pfdbUpdateData
 0001:0000815C       ovcdbpf.TOvcDbPictureField.pfSetPictureMask
 0001:00008178       ovcdbpf.TOvcDbPictureField.Restore
 0001:00008198       ovcdbpf.TOvcDbPictureField.SetDataField
 0001:00008250       ovcdbpf.TOvcDbPictureField.SetDataSource
 0001:00008284       ovcdbpf.TOvcDbPictureField.SetDateOrTime
 0001:000082B0       ovcdbpf.TOvcDbPictureField.SetFieldType
 0001:00008350       ovcdbpf.TOvcDbPictureField.SetUseTFieldMask
 0001:00008368       ovcdbpf.TOvcDbPictureField.SetZeroAsNull
 0001:00008378       ovcdbpf.TOvcDbPictureField.WMKeyDown
 0001:0000847C       ovcdbpf.TOvcDbPictureField.WMKillFocus
 0001:000084E4       ovcdbpf.TOvcDbPictureField.WMLButtonDblClk
 0001:000084F8       ovcdbpf.TOvcDbPictureField.WMLButtonDown
 0001:0000850C       ovcdbpf.TOvcDbPictureField.WMLButtonUp
 0001:0000852C       ovcdbpf.TOvcDbPictureField.WMPaint
 0001:000089A4       ovcdbpf.TOvcDbPictureField.WMSetFocus
 0001:000089D0       ovcdbpf.TOvcDbPictureField.ExecuteAction
 0001:00008A0C       ovcdbpf.TOvcDbPictureField.UpdateAction
 0001:00008A48       ovcdbpf.Finalization
 0001:00008AC8       ovcdbsf..TOvcDbSimpleField
 0001:000095E4       ovcdbsf.TOvcDbSimpleField.CMEnter
 0001:00009600       ovcdbsf.TOvcDbSimpleField.CMExit
 0001:00009608       ovcdbsf.TOvcDbSimpleField.CMGetDataLink
 0001:00009614       ovcdbsf.TOvcDbSimpleField.Create
 0001:000096B4       ovcdbsf.TOvcDbSimpleField.CreateWnd
 0001:000096E4       ovcdbsf.TOvcDbSimpleField.CutToClipboard
 0001:00009764       ovcdbsf.TOvcDbSimpleField.Destroy
 0001:000097B0       ovcdbsf.TOvcDbSimpleField.DoOnChange
 0001:000097DC       ovcdbsf.TOvcDbSimpleField.efEdit
 0001:00009858       ovcdbsf.TOvcDbSimpleField.efGetSampleDisplayData
 0001:000099D4       ovcdbsf.TOvcDbSimpleField.efIncDecValue
 0001:00009A4C       ovcdbsf.TOvcDbSimpleField.efIsReadOnly
 0001:00009AD0       ovcdbsf.TOvcDbSimpleField.GetDataField
 0001:00009AEC       ovcdbsf.TOvcDbSimpleField.GetDataSource
 0001:00009B00       ovcdbsf.TOvcDbSimpleField.GetField
 0001:00009B80       ovcdbsf.TOvcDbSimpleField.Notification
 0001:00009BC8       ovcdbsf.TOvcDbSimpleField.PasteFromClipboard
 0001:00009C48       ovcdbsf.TOvcDbSimpleField.Restore
 0001:00009C68       ovcdbsf.TOvcDbSimpleField.SetDataField
 0001:00009D20       ovcdbsf.TOvcDbSimpleField.SetDataSource
 0001:00009D54       ovcdbsf.TOvcDbSimpleField.SetFieldType
 0001:00009DF4       ovcdbsf.TOvcDbSimpleField.SetUseTFieldMask
 0001:00009E0C       ovcdbsf.TOvcDbSimpleField.SetZeroAsNull
 0001:00009E1C       ovcdbsf.TOvcDbSimpleField.sfdbDataChange
 0001:00009E80       ovcdbsf.TOvcDbSimpleField.sfdbEditingChange
 0001:00009EA4       ovcdbsf.FieldIsZero
 0001:00009F6C       ovcdbsf.TOvcDbSimpleField.sfdbGetFieldValue
 0001:0000A1CC       ovcdbsf.TOvcDbSimpleField.sfdbSetFieldProperties
 0001:0000A2FC       ovcdbsf.TOvcDbSimpleField.sfdbSetFieldValue
 0001:0000A704       ovcdbsf.TOvcDbSimpleField.sfdbUpdateData
 0001:0000A7D4       ovcdbsf.TOvcDbSimpleField.WMKeyDown
 0001:0000A8D8       ovcdbsf.TOvcDbSimpleField.WMKillFocus
 0001:0000A940       ovcdbsf.TOvcDbSimpleField.WMLButtonDblClk
 0001:0000A954       ovcdbsf.TOvcDbSimpleField.WMLButtonDown
 0001:0000A970       ovcdbsf.TOvcDbSimpleField.WMLButtonUp
 0001:0000A990       ovcdbsf.TOvcDbSimpleField.WMPaint
 0001:0000AD2C       ovcdbsf.TOvcDbSimpleField.WMSetFocus
 0001:0000AD58       ovcdbsf.TOvcDbSimpleField.ExecuteAction
 0001:0000AD94       ovcdbsf.TOvcDbSimpleField.UpdateAction
 0001:0000ADD0       ovcdbsf.Finalization
 0001:0000AEB4       ovcdbae..TOvcDbSimpleCell
 0001:0000B068       ovcdbae..TOvcDbPictureCell
 0001:0000B220       ovcdbae..TOvcDbNumericCell
 0001:0000B3D8       ovcdbae..TOvcBaseDbArrayEditor
 0001:0000B5BC       ovcdbae..TOvcDbSimpleArrayEditor
 0001:0000C034       ovcdbae..TOvcDbPictureArrayEditor
 0001:0000CAF4       ovcdbae..TOvcDbNumericArrayEditor
 0001:0000D524       ovcdbae.TOvcBaseDbArrayEditor.aeActiveChange
 0001:0000D540       ovcdbae.TOvcBaseDbArrayEditor.aeAdjustIntegralHeight
 0001:0000D57C       ovcdbae.TOvcBaseDbArrayEditor.aeAdjustRowHeight
 0001:0000D668       ovcdbae.TOvcBaseDbArrayEditor.aeColorChanged
 0001:0000D670       ovcdbae.TOvcBaseDbArrayEditor.aeDataChange
 0001:0000D6E8       ovcdbae.TOvcBaseDbArrayEditor.aeEditingChange
 0001:0000D704       ovcdbae.TOvcBaseDbArrayEditor.aeGetEditString
 0001:0000D710       ovcdbae.TOvcBaseDbArrayEditor.aeGetSampleDisplayData
 0001:0000D724       ovcdbae.TOvcBaseDbArrayEditor.aeMoveCell
 0001:0000D740       ovcdbae.TOvcBaseDbArrayEditor.aeReadRangeHi
 0001:0000D760       ovcdbae.TOvcBaseDbArrayEditor.aeReadRangeLo
 0001:0000D780       ovcdbae.TOvcBaseDbArrayEditor.aeRefresh
 0001:0000D79C       ovcdbae.TOvcBaseDbArrayEditor.aeUpdateActive
 0001:0000D7D4       ovcdbae.TOvcBaseDbArrayEditor.aeUpdateData
 0001:0000D7F0       ovcdbae.TOvcBaseDbArrayEditor.aeUpdateNumRows
 0001:0000D850       ovcdbae.TOvcBaseDbArrayEditor.aeUpdateScrollBar
 0001:0000D9B8       ovcdbae.TOvcBaseDbArrayEditor.aeWriteRangeHi
 0001:0000D9CC       ovcdbae.TOvcBaseDbArrayEditor.aeWriteRangeLo
 0001:0000D9E0       ovcdbae.TOvcBaseDbArrayEditor.ChangeScale
 0001:0000DA18       ovcdbae.TOvcBaseDbArrayEditor.CMCtl3DChanged
 0001:0000DA58       ovcdbae.TOvcBaseDbArrayEditor.CMFontChanged
 0001:0000DA84       ovcdbae.TOvcBaseDbArrayEditor.Create
 0001:0000DD2C       ovcdbae.TOvcBaseDbArrayEditor.CreateParams
 0001:0000DD8C       ovcdbae.TOvcBaseDbArrayEditor.CreateWnd
 0001:0000DDEC       ovcdbae.TOvcBaseDbArrayEditor.DefineProperties
 0001:0000DE5C       ovcdbae.TOvcBaseDbArrayEditor.Destroy
 0001:0000DEBC       ovcdbae.TOvcBaseDbArrayEditor.DoGetItemColor
 0001:0000DEEC       ovcdbae.TOvcBaseDbArrayEditor.DoOnIndicatorClick
 0001:0000DF14       ovcdbae.TOvcBaseDbArrayEditor.GetDataLink
 0001:0000DF74       ovcdbae.TOvcBaseDbArrayEditor.GetField
 0001:0000DFE0       ovcdbae.TOvcBaseDbArrayEditor.GetRangeHi
 0001:0000DFFC       ovcdbae.TOvcBaseDbArrayEditor.GetRangeLo
 0001:0000E018       ovcdbae.TOvcBaseDbArrayEditor.Paint
 0001:0000E828       ovcdbae.TOvcBaseDbArrayEditor.Reset
 0001:0000E854       ovcdbae.TOvcBaseDbArrayEditor.Scroll
 0001:0000E888       ovcdbae.TOvcBaseDbArrayEditor.SetActiveRow
 0001:0000E8E0       ovcdbae.TOvcBaseDbArrayEditor.SetAutoRowHeight
 0001:0000E8FC       ovcdbae.TOvcBaseDbArrayEditor.SetBorderStyle
 0001:0000E910       ovcdbae.TOvcBaseDbArrayEditor.SetDataField
 0001:0000E93C       ovcdbae.TOvcBaseDbArrayEditor.SetDataSource
 0001:0000E948       ovcdbae.TOvcBaseDbArrayEditor.SetDateOrTime
 0001:0000E984       ovcdbae.TOvcBaseDbArrayEditor.SetDecimalPlaces
 0001:0000E9C4       ovcdbae.TOvcBaseDbArrayEditor.SetEpoch
 0001:0000EA00       ovcdbae.TOvcBaseDbArrayEditor.SetFieldType
 0001:0000EA0C       ovcdbae.TOvcBaseDbArrayEditor.SetFocus
 0001:0000EA38       ovcdbae.TOvcBaseDbArrayEditor.SetLineColor
 0001:0000EA4C       ovcdbae.TOvcBaseDbArrayEditor.SetMaxLength
 0001:0000EA94       ovcdbae.TOvcBaseDbArrayEditor.SetOptions
 0001:0000EB04       ovcdbae.TOvcBaseDbArrayEditor.SetPadChar
 0001:0000EB3C       ovcdbae.TOvcBaseDbArrayEditor.SetPictureMask
 0001:0000EC48       ovcdbae.TOvcBaseDbArrayEditor.SetRangeHi
 0001:0000EC88       ovcdbae.TOvcBaseDbArrayEditor.SetRangeLo
 0001:0000ECC8       ovcdbae.TOvcBaseDbArrayEditor.SetRowHeight
 0001:0000ECF0       ovcdbae.TOvcBaseDbArrayEditor.SetRowIndicatorWidth
 0001:0000ED68       ovcdbae.TOvcBaseDbArrayEditor.SetShowIndicator
 0001:0000EE04       ovcdbae.TOvcBaseDbArrayEditor.SetTextMargin
 0001:0000EE34       ovcdbae.TOvcBaseDbArrayEditor.UpdateRecord
 0001:0000EE60       ovcdbae.TOvcBaseDbArrayEditor.SetUseScrollBar
 0001:0000EE74       ovcdbae.TOvcBaseDbArrayEditor.SetZeroAsNull
 0001:0000EEEC       ovcdbae.TOvcBaseDbArrayEditor.WMGetMinMaxInfo
 0001:0000EF00       ovcdbae.TOvcBaseDbArrayEditor.WMEraseBkGnd
 0001:0000EF08       ovcdbae.TOvcBaseDbArrayEditor.WMLButtonDown
 0001:0000F060       ovcdbae.TOvcBaseDbArrayEditor.WMMouseActivate
 0001:0000F06C       ovcdbae.TOvcBaseDbArrayEditor.WMNCHitTest
 0001:0000F088       ovcdbae.TOvcBaseDbArrayEditor.WMSetFocus
 0001:0000F0E4       ovcdbae.TOvcBaseDbArrayEditor.WMSize
 0001:0000F170       ovcdbae.TOvcBaseDbArrayEditor.WMVScroll
 0001:0000F3A0       ovcdbae.TOvcDbSimpleArrayEditor.aeCreateEditCell
 0001:0000F804       ovcdbae.TOvcDbSimpleArrayEditor.aeGetCellProperties
 0001:0000F8BC       ovcdbae.TOvcDbSimpleArrayEditor.Create
 0001:0000F920       ovcdbae.TOvcDbPictureArrayEditor.aeCreateEditCell
 0001:0000FDB0       ovcdbae.TOvcDbPictureArrayEditor.aeGetCellProperties
 0001:0000FE68       ovcdbae.TOvcDbPictureArrayEditor.Create
 0001:0000FEDC       ovcdbae.TOvcDbNumericArrayEditor.aeCreateEditCell
 0001:000102FC       ovcdbae.TOvcDbNumericArrayEditor.aeGetCellProperties
 0001:000103B4       ovcdbae.TOvcDbNumericArrayEditor.Create
 0001:00010420       ovcdbae.TOvcDbSimpleCell.Create
 0001:0001048C       ovcdbae.TOvcDbSimpleCell.CreateWnd
 0001:00010628       ovcdbae.TOvcDbSimpleCell.WMKeyDown
 0001:00010770       ovcdbae.TOvcDbPictureCell.Create
 0001:000107DC       ovcdbae.TOvcDbPictureCell.CreateWnd
 0001:00010978       ovcdbae.TOvcDbPictureCell.WMKeyDown
 0001:00010AC0       ovcdbae.TOvcDbNumericCell.Create
 0001:00010B2C       ovcdbae.TOvcDbNumericCell.CreateWnd
 0001:00010CC8       ovcdbae.TOvcDbNumericCell.WMKeyDown
 0001:00010E10       ovcdbae.Finalization
 0001:00010ED8       ovcdbcal..TOvcDbCalendar
 0001:00011770       ovcdbcal.TOvcDbCalendar.calDataChange
 0001:000117F8       ovcdbcal.TOvcDbCalendar.calUpdateData
 0001:00011918       ovcdbcal.TOvcDbCalendar.CMExit
 0001:0001197C       ovcdbcal.TOvcDbCalendar.CMGetDataLink
 0001:00011988       ovcdbcal.TOvcDbCalendar.Create
 0001:00011A04       ovcdbcal.TOvcDbCalendar.Destroy
 0001:00011A3C       ovcdbcal.TOvcDbCalendar.DoOnChange
 0001:00011A60       ovcdbcal.TOvcDbCalendar.GetDataField
 0001:00011A7C       ovcdbcal.TOvcDbCalendar.GetDataSource
 0001:00011A90       ovcdbcal.TOvcDbCalendar.GetField
 0001:00011A9C       ovcdbcal.TOvcDbCalendar.IsReadOnly
 0001:00011AD0       ovcdbcal.TOvcDbCalendar.Notification
 0001:00011B14       ovcdbcal.TOvcDbCalendar.SetCalendarDate
 0001:00011B88       ovcdbcal.TOvcDbCalendar.SetDataField
 0001:00011CFC       ovcdbcal.TOvcDbCalendar.SetDataSource
 0001:00011D28       ovcdbcal.TOvcDbCalendar.WMLButtonDown
 0001:00011D6C       ovcdbcal.TOvcDbCalendar.WMKeyDown
 0001:00011DB0       ovcdbcal.TOvcDbCalendar.KeyPress
 0001:00011DE4       ovcdbcal.TOvcDbCalendar.ExecuteAction
 0001:00011E20       ovcdbcal.TOvcDbCalendar.UpdateAction
 0001:00011E5C       ovcdbcal.Finalization
 0001:00011EBC       ovcdbccb..TOvcDbColorComboBox
 0001:0001277C       ovcdbccb.TOvcDbColorComboBox.ccbDataChange
 0001:000127BC       ovcdbccb.TOvcDbColorComboBox.ccbUpdateData
 0001:000127F4       ovcdbccb.TOvcDbColorComboBox.Change
 0001:000128E0       ovcdbccb.TOvcDbColorComboBox.CMGetDataLink
 0001:000128EC       ovcdbccb.TOvcDbColorComboBox.Create
 0001:00012960       ovcdbccb.TOvcDbColorComboBox.Destroy
 0001:00012998       ovcdbccb.TOvcDbColorComboBox.GetDataField
 0001:000129B4       ovcdbccb.TOvcDbColorComboBox.GetDataSource
 0001:000129C8       ovcdbccb.TOvcDbColorComboBox.GetField
 0001:000129D4       ovcdbccb.TOvcDbColorComboBox.Notification
 0001:00012A18       ovcdbccb.TOvcDbColorComboBox.SetDataField
 0001:00012B8C       ovcdbccb.TOvcDbColorComboBox.SetDataSource
 0001:00012BB8       ovcdbccb.TOvcDbColorComboBox.ExecuteAction
 0001:00012BF4       ovcdbccb.TOvcDbColorComboBox.UpdateAction
 0001:00012C30       ovcdbccb.Finalization
 0001:00012CE4       ovcdbcl..TOvcDbColumnList
 0001:000136E8       ovcdbcl.TOvcDbColumnList.ChangeScale
 0001:00013720       ovcdbcl.TOvcDbColumnList.clActiveChange
 0001:0001373C       ovcdbcl.TOvcDbColumnList.clAdjustIntegralHeight
 0001:00013788       ovcdbcl.TOvcDbColumnList.clAdjustRowHeight
 0001:00013874       ovcdbcl.TOvcDbColumnList.clCalcNumRows
 0001:000138B4       ovcdbcl.TOvcDbColumnList.clColorChanged
 0001:000138BC       ovcdbcl.TOvcDbColumnList.clDataChange
 0001:000138EC       ovcdbcl.TOvcDbColumnList.clDrawHeader
 0001:00013C2C       ovcdbcl.TOvcDbColumnList.clEditingChange
 0001:00013C40       ovcdbcl.TOvcDbColumnList.clInitScrollBarInfo
 0001:00013C6C       ovcdbcl.TOvcDbColumnList.clSetHScrollPos
 0001:00013C98       ovcdbcl.TOvcDbColumnList.clSetHScrollRange
 0001:00013CF0       ovcdbcl.TOvcDbColumnList.clSetVScrollPos
 0001:00013E4C       ovcdbcl.TOvcDbColumnList.clSetVScrollRange
 0001:00013E54       ovcdbcl.TOvcDbColumnList.clUpdateActive
 0001:00013E80       ovcdbcl.TOvcDbColumnList.clUpdateData
 0001:00013E84       ovcdbcl.TOvcDbColumnList.clUpdateNumRows
 0001:00013EF4       ovcdbcl.TOvcDbColumnList.CMCtl3DChanged
 0001:00013F34       ovcdbcl.TOvcDbColumnList.CMFontChanged
 0001:00013F80       ovcdbcl.TOvcDbColumnList.CMGetDataLink
 0001:00013F8C       ovcdbcl.TOvcDbColumnList.Create
 0001:00014298       ovcdbcl.TOvcDbColumnList.CreateParams
 0001:000142FC       ovcdbcl.TOvcDbColumnList.CreateWnd
 0001:0001433C       ovcdbcl.TOvcDbColumnList.Destroy
 0001:000143B0       ovcdbcl.TOvcDbColumnList.DoOnClickHeader
 0001:000143E0       ovcdbcl.TOvcDbColumnList.DoOnIndicatorClick
 0001:00014408       ovcdbcl.TOvcDbColumnList.DoOnUserCommand
 0001:00014428       ovcdbcl.TOvcDbColumnList.GetField
 0001:0001448C       ovcdbcl.TOvcDbColumnList.GetDataField
 0001:000144A8       ovcdbcl.TOvcDbColumnList.GetDataSource
 0001:000144BC       ovcdbcl.TOvcDbColumnList.InvalidateItem
 0001:00014520       ovcdbcl.TOvcDbColumnList.Notification
 0001:0001455C       ovcdbcl.TOvcDbColumnList.Paint
 0001:00014C58       ovcdbcl.TOvcDbColumnList.SetActiveRow
 0001:00014CA4       ovcdbcl.TOvcDbColumnList.SetAutoRowHeight
 0001:00014CC0       ovcdbcl.TOvcDbColumnList.SetBorderStyle
 0001:00014CD4       ovcdbcl.TOvcDbColumnList.SetDataField
 0001:00014D84       ovcdbcl.TOvcDbColumnList.SetDataSource
 0001:00014DB0       ovcdbcl.TOvcDbColumnList.SetHeader
 0001:00014DE0       ovcdbcl.TOvcDbColumnList.SetIntegralHeight
 0001:00014DF4       ovcdbcl.TOvcDbColumnList.SetLineColor
 0001:00014E08       ovcdbcl.TOvcDbColumnList.SetRowHeight
 0001:00014E30       ovcdbcl.TOvcDbColumnList.SetScrollBars
 0001:00014E44       ovcdbcl.TOvcDbColumnList.SetShowHeader
 0001:00014E58       ovcdbcl.TOvcDbColumnList.SetShowIndicator
 0001:00014E8C       ovcdbcl.TOvcDbColumnList.SetRowIndicatorWidth
 0001:00014EC4       ovcdbcl.TOvcDbColumnList.SetTextMargin
 0001:00014EDC       ovcdbcl.TOvcDbColumnList.WMEraseBkgnd
 0001:00014EE4       ovcdbcl.TOvcDbColumnList.WMGetDlgCode
 0001:00014EF4       ovcdbcl.TOvcDbColumnList.WMGetMinMaxInfo
 0001:00014F08       ovcdbcl.HScrollPrim
 0001:00014FBC       ovcdbcl.TOvcDbColumnList.WMHScroll
 0001:00015060       ovcdbcl.TOvcDbColumnList.WMKeyDown
 0001:00015254       ovcdbcl.TOvcDbColumnList.WMKillFocus
 0001:00015270       ovcdbcl.TOvcDbColumnList.WMLButtonDown
 0001:00015388       ovcdbcl.TOvcDbColumnList.WMMouseActivate
 0001:000153D4       ovcdbcl.TOvcDbColumnList.WMNCHitTest
 0001:000153F0       ovcdbcl.TOvcDbColumnList.WMSetFocus
 0001:0001540C       ovcdbcl.TOvcDbColumnList.WMSize
 0001:0001543C       ovcdbcl.TOvcDbColumnList.WMVScroll
 0001:0001565C       ovcdbcl.TOvcDbColumnList.ExecuteAction
 0001:00015698       ovcdbcl.TOvcDbColumnList.UpdateAction
 0001:000156D4       ovcdbcl.Finalization
 0001:00015754       ovcdbclk..TOvcDbClock
 0001:00015CC8       ovcdbclk.TOvcDbClock.clkDataChange
 0001:00015D5C       ovcdbclk.TOvcDbClock.CMGetDataLink
 0001:00015D68       ovcdbclk.TOvcDbClock.Create
 0001:00015DD4       ovcdbclk.TOvcDbClock.Destroy
 0001:00015E0C       ovcdbclk.TOvcDbClock.GetDataField
 0001:00015E28       ovcdbclk.TOvcDbClock.GetDataSource
 0001:00015E3C       ovcdbclk.TOvcDbClock.GetField
 0001:00015E48       ovcdbclk.TOvcDbClock.Notification
 0001:00015E8C       ovcdbclk.TOvcDbClock.SetDataField
 0001:00016000       ovcdbclk.TOvcDbClock.SetDataSource
 0001:0001602C       ovcdbclk.TOvcDbClock.ExecuteAction
 0001:00016068       ovcdbclk.TOvcDbClock.UpdateAction
 0001:000160A4       ovcdbclk.Finalization
 0001:000161A4       ovcdbdat..TOvcCustomDbDateEdit
 0001:00016384       ovcdbdat..TOvcDbDateEdit
 0001:00016EBC       ovcdbdat.TOvcCustomDbDateEdit.Change
 0001:00016ED4       ovcdbdat.TOvcCustomDbDateEdit.CMEnter
 0001:00016EF0       ovcdbdat.TOvcCustomDbDateEdit.CMExit
 0001:00016F84       ovcdbdat.TOvcCustomDbDateEdit.CMGetDataLink
 0001:00016F90       ovcdbdat.TOvcCustomDbDateEdit.Create
 0001:00017024       ovcdbdat.TOvcCustomDbDateEdit.DataChange
 0001:0001721C       ovcdbdat.TOvcCustomDbDateEdit.Destroy
 0001:00017268       ovcdbdat.TOvcCustomDbDateEdit.EditingChange
 0001:0001729C       ovcdbdat.TOvcCustomDbDateEdit.GetButtonEnabled
 0001:000172D0       ovcdbdat.TOvcCustomDbDateEdit.GetDataField
 0001:000172EC       ovcdbdat.TOvcCustomDbDateEdit.GetDataSource
 0001:000172F8       ovcdbdat.TOvcCustomDbDateEdit.GetField
 0001:00017304       ovcdbdat.TOvcCustomDbDateEdit.GetReadOnly
 0001:00017344       ovcdbdat.TOvcCustomDbDateEdit.GetTextMargins
 0001:0001740C       ovcdbdat.TOvcCustomDbDateEdit.KeyDown
 0001:00017444       ovcdbdat.TOvcCustomDbDateEdit.KeyPress
 0001:00017520       ovcdbdat.TOvcCustomDbDateEdit.Notification
 0001:0001755C       ovcdbdat.TOvcCustomDbDateEdit.PopupClose
 0001:0001758C       ovcdbdat.TOvcCustomDbDateEdit.PopupOpen
 0001:000175A4       ovcdbdat.TOvcCustomDbDateEdit.SetDataField
 0001:0001763C       ovcdbdat.TOvcCustomDbDateEdit.SetDataSource
 0001:00017660       ovcdbdat.TOvcCustomDbDateEdit.SetFocused
 0001:00017694       ovcdbdat.TOvcCustomDbDateEdit.SetReadOnly
 0001:000176A0       ovcdbdat.TOvcCustomDbDateEdit.UpdateData
 0001:000178B0       ovcdbdat.TOvcCustomDbDateEdit.WMCut
 0001:000178D0       ovcdbdat.TOvcCustomDbDateEdit.WMPaint
 0001:00017B4C       ovcdbdat.TOvcCustomDbDateEdit.WMPaste
 0001:00017B6C       ovcdbdat.TOvcCustomDbDateEdit.ExecuteAction
 0001:00017BA8       ovcdbdat.TOvcCustomDbDateEdit.UpdateAction
 0001:00017BE4       ovcdbdat.Finalization
 0001:00017C84       ovcdbdLb..TOvcDbDisplayLabel
 0001:0001825C       ovcdbdLb.TOvcDbDisplayLabel.CMGetDataLink
 0001:00018268       ovcdbdLb.TOvcDbDisplayLabel.Create
 0001:000182C4       ovcdbdLb.TOvcDbDisplayLabel.Destroy
 0001:000182FC       ovcdbdLb.TOvcDbDisplayLabel.dlDataChange
 0001:00018348       ovcdbdLb.TOvcDbDisplayLabel.dlGetDisplayLabel
 0001:000183C4       ovcdbdLb.TOvcDbDisplayLabel.GetDataField
 0001:000183E0       ovcdbdLb.TOvcDbDisplayLabel.GetDataSource
 0001:000183EC       ovcdbdLb.TOvcDbDisplayLabel.GetField
 0001:000183F8       ovcdbdLb.TOvcDbDisplayLabel.Notification
 0001:00018434       ovcdbdLb.TOvcDbDisplayLabel.SetDataField
 0001:00018488       ovcdbdLb.TOvcDbDisplayLabel.SetDataSource
 0001:000184AC       ovcdbdLb.TOvcDbDisplayLabel.ExecuteAction
 0001:000184E8       ovcdbdLb.TOvcDbDisplayLabel.UpdateAction
 0001:00018524       ovcdbdLb.Finalization
 0001:00018774       ovcdbed..TOvcDbEditor
 0001:00019390       ovcdbed.TOvcDbEditor.CMEnter
 0001:000193B0       ovcdbed.TOvcDbEditor.CMExit
 0001:00019424       ovcdbed.TOvcDbEditor.CMGetDataLink
 0001:00019430       ovcdbed.TOvcDbEditor.Create
 0001:000194AC       ovcdbed.TOvcDbEditor.CreateWnd
 0001:000194CC       ovcdbed.TOvcDbEditor.CutToClipboard
 0001:00019550       ovcdbed.TOvcDbEditor.Destroy
 0001:00019588       ovcdbed.TOvcDbEditor.edAddSampleParas
 0001:0001958C       ovcdbed.TOvcDbEditor.eddbDataChange
 0001:0001959C       ovcdbed.TOvcDbEditor.eddbEditingChange
 0001:000195A0       ovcdbed.TOvcDbEditor.eddbGetEditorValue
 0001:000196A4       ovcdbed.TOvcDbEditor.eddbSetEditorValue
 0001:00019A1C       ovcdbed.TOvcDbEditor.eddbUpdateData
 0001:00019A24       ovcdbed.TOvcDbEditor.GetReadOnly
 0001:00019AB4       ovcdbed.TOvcDbEditor.GetField
 0001:00019AC0       ovcdbed.TOvcDbEditor.GetDataField
 0001:00019ADC       ovcdbed.TOvcDbEditor.GetDataSource
 0001:00019AF0       ovcdbed.TOvcDbEditor.Notification
 0001:00019B28       ovcdbed.TOvcDbEditor.PasteFromClipboard
 0001:00019BAC       ovcdbed.TOvcDbEditor.Redo
 0001:00019C30       ovcdbed.TOvcDbEditor.Replace
 0001:00019CCC       ovcdbed.TOvcDbEditor.SetDataField
 0001:00019D28       ovcdbed.TOvcDbEditor.SetDataSource
 0001:00019D40       ovcdbed.TOvcDbEditor.Undo
 0001:00019DC4       ovcdbed.TOvcDbEditor.WMChar
 0001:00019E14       ovcdbed.DoChange
 0001:00019E8C       ovcdbed.TOvcDbEditor.WMKeyDown
 0001:00019F48       ovcdbed.TOvcDbEditor.ExecuteAction
 0001:00019F84       ovcdbed.TOvcDbEditor.UpdateAction
 0001:00019FC0       ovcdbed.Finalization
 0001:0001A00C       ovcdbfcb..TOvcDbFieldComboBox
 0001:0001A928       ovcdbfcb.TOvcDbFieldComboBox.ActiveChanged
 0001:0001A930       ovcdbfcb.TOvcDbFieldComboBox.Create
 0001:0001A9B8       ovcdbfcb.TOvcDbFieldComboBox.Destroy
 0001:0001A9F0       ovcdbfcb.TOvcDbFieldComboBox.DrawItem
 0001:0001AB90       ovcdbfcb.TOvcDbFieldComboBox.GetDataSource
 0001:0001AB9C       ovcdbfcb.TOvcDbFieldComboBox.GetFieldName
 0001:0001AC88       ovcdbfcb.TOvcDbFieldComboBox.Loaded
 0001:0001AC9C       ovcdbfcb.TOvcDbFieldComboBox.Populate
 0001:0001ADC4       ovcdbfcb.TOvcDbFieldComboBox.SetDataSource
 0001:0001ADDC       ovcdbfcb.TOvcDbFieldComboBox.SetOmitFields
 0001:0001AE20       ovcdbfcb.TOvcDbFieldComboBox.SetShowHiddenFields
 0001:0001AE3C       ovcdbfcb.TOvcDbFieldComboBox.ExecuteAction
 0001:0001AE78       ovcdbfcb.TOvcDbFieldComboBox.UpdateAction
 0001:0001AEB4       ovcdbfcb.Finalization
 0001:0001AFF4       ovcdbidx..TOvcIndexInfo
 0001:0001B09C       ovcdbidx..TOvcIndexSelectDataLink
 0001:0001B188       ovcdbidx..TOvcDbIndexSelect
 0001:0001B924       ovcdbidx.TOvcIndexInfo.Create
 0001:0001B998       ovcdbidx.TOvcIndexInfo.Destroy
 0001:0001B9CC       ovcdbidx.TOvcIndexInfo.RefreshIndexInfo
 0001:0001BD9C       ovcdbidx.TOvcIndexInfo.SetDisplayName
 0001:0001BDD0       ovcdbidx.TOvcIndexSelectDataLink.ActiveChanged
 0001:0001BDEC       ovcdbidx.TOvcIndexSelectDataLink.Create
 0001:0001BE28       ovcdbidx.TOvcIndexSelectDataLink.DataSetChanged
 0001:0001BE3C       ovcdbidx.TOvcIndexSelectDataLink.LayoutChanged
 0001:0001BE58       ovcdbidx.TOvcDbIndexSelect.Change
 0001:0001BED8       ovcdbidx.TOvcDbIndexSelect.ClearObjects
 0001:0001BF48       ovcdbidx.TOvcDbIndexSelect.CMVisibleChanged
 0001:0001BF78       ovcdbidx.TOvcDbIndexSelect.Create
 0001:0001C01C       ovcdbidx.TOvcDbIndexSelect.CreateWnd
 0001:0001C030       ovcdbidx.TOvcDbIndexSelect.Destroy
 0001:0001C094       ovcdbidx.TOvcDbIndexSelect.DestroyWnd
 0001:0001C0AC       ovcdbidx.TOvcDbIndexSelect.DropDown
 0001:0001C0C8       ovcdbidx.TOvcDbIndexSelect.GetAttachedLabel
 0001:0001C134       ovcdbidx.TOvcDbIndexSelect.GetDataSource
 0001:0001C148       ovcdbidx.TOvcDbIndexSelect.GetAbout
 0001:0001C16C       ovcdbidx.TOvcDbIndexSelect.GetIndexName
 0001:0001C178       ovcdbidx.TOvcDbIndexSelect.GetIndexFieldNames
 0001:0001C184       ovcdbidx.TOvcDbIndexSelect.isFindIndex
 0001:0001C2D0       ovcdbidx.TOvcDbIndexSelect.LabelAttach
 0001:0001C410       ovcdbidx.TOvcDbIndexSelect.LabelChange
 0001:0001C41C       ovcdbidx.TOvcDbIndexSelect.Notification
 0001:0001C480       ovcdbidx.TOvcDbIndexSelect.OMAssignLabel
 0001:0001C490       ovcdbidx.TOvcDbIndexSelect.OMPositionLabel
 0001:0001C538       ovcdbidx.TOvcDbIndexSelect.OMRecordLabelPosition
 0001:0001C59C       ovcdbidx.TOvcDbIndexSelect.PositionLabel
 0001:0001C634       ovcdbidx.TOvcDbIndexSelect.RefreshList
 0001:0001CA10       ovcdbidx.TOvcDbIndexSelect.RefreshNow
 0001:0001CA24       ovcdbidx.TOvcDbIndexSelect.SetBounds
 0001:0001CA60       ovcdbidx.TOvcDbIndexSelect.SetDataSource
 0001:0001CA90       ovcdbidx.TOvcDbIndexSelect.SetDisplayMode
 0001:0001CAAC       ovcdbidx.TOvcDbIndexSelect.SetMonitorIdx
 0001:0001CAD4       ovcdbidx.TOvcDbIndexSelect.SetRefreshPendingFlag
 0001:0001CADC       ovcdbidx.TOvcDbIndexSelect.SetShowHidden
 0001:0001CAF8       ovcdbidx.TOvcDbIndexSelect.SetAbout
 0001:0001CAFC       ovcdbidx.TOvcDbIndexSelect.WMDestroy
 0001:0001CB04       ovcdbidx.TOvcDbIndexSelect.WMPaint
 0001:0001CB28       ovcdbidx.Finalization
 0001:0001CB80       ovcdbise..TOvcDbSearchEdit
 0001:0001D450       ovcdbise.TOvcDbSearchEdit.CMVisibleChanged
 0001:0001D480       ovcdbise.TOvcDbSearchEdit.Create
 0001:0001D500       ovcdbise.TOvcDbSearchEdit.Destroy
 0001:0001D558       ovcdbise.TOvcDbSearchEdit.GetAttachedLabel
 0001:0001D5C4       ovcdbise.TOvcDbSearchEdit.GetDataSource
 0001:0001D5D8       ovcdbise.TOvcDbSearchEdit.GetAbout
 0001:0001D5FC       ovcdbise.TOvcDbSearchEdit.LabelAttach
 0001:0001D73C       ovcdbise.TOvcDbSearchEdit.LabelChange
 0001:0001D748       ovcdbise.TOvcDbSearchEdit.Notification
 0001:0001D7AC       ovcdbise.TOvcDbSearchEdit.OMAssignLabel
 0001:0001D7BC       ovcdbise.TOvcDbSearchEdit.OMPositionLabel
 0001:0001D864       ovcdbise.TOvcDbSearchEdit.OMRecordLabelPosition
 0001:0001D8C8       ovcdbise.TOvcDbSearchEdit.PerformSearch
 0001:0001DBC8       ovcdbise.TOvcDbSearchEdit.PositionLabel
 0001:0001DC60       ovcdbise.TOvcDbSearchEdit.SetBounds
 0001:0001DC9C       ovcdbise.TOvcDbSearchEdit.SetDataSource
 0001:0001DCC0       ovcdbise.TOvcDbSearchEdit.SetAbout
 0001:0001DCC4       ovcdbise.Finalization
 0001:0001DCF4       ovcdbmdg..TOvcfrmDbMemoDlg
 0001:0001DF04       ovcdbmdg..TOvcDbMemoDialog
 0001:0001E150       ovcdbmdg.TOvcDbMemoDialog.Create
 0001:0001E1AC       ovcdbmdg.TOvcDbMemoDialog.Destroy
 0001:0001E1EC       ovcdbmdg.TOvcDbMemoDialog.Execute
 0001:0001E474       ovcdbmdg.TOvcDbMemoDialog.GetDataField
 0001:0001E48C       ovcdbmdg.TOvcDbMemoDialog.GetDataSource
 0001:0001E494       ovcdbmdg.TOvcDbMemoDialog.SetDataField
 0001:0001E4E4       ovcdbmdg.TOvcDbMemoDialog.SetDataSource
 0001:0001E4F0       ovcdbmdg.TOvcDbMemoDialog.SetMemoFont
 0001:0001E500       ovcdbmdg.TOvcDbMemoDialog.ExecuteAction
 0001:0001E538       ovcdbmdg.TOvcDbMemoDialog.UpdateAction
 0001:0001E570       ovcdbmdg.TOvcfrmDbMemoDlg.FormCloseQuery
 0001:0001E5F4       ovcdbmdg.Finalization
 0001:0001E624       ovcdbnum..TOvcCustomDbNumberEdit
 0001:0001E80C       ovcdbnum..TOvcDbNumberEdit
 0001:0001F12C       ovcdbnum.TOvcCustomDbNumberEdit.Change
 0001:0001F144       ovcdbnum.TOvcCustomDbNumberEdit.CMEnter
 0001:0001F160       ovcdbnum.TOvcCustomDbNumberEdit.CMExit
 0001:0001F1F4       ovcdbnum.TOvcCustomDbNumberEdit.CMGetDataLink
 0001:0001F200       ovcdbnum.TOvcCustomDbNumberEdit.Create
 0001:0001F294       ovcdbnum.TOvcCustomDbNumberEdit.DataChange
 0001:0001F44C       ovcdbnum.TOvcCustomDbNumberEdit.Destroy
 0001:0001F498       ovcdbnum.TOvcCustomDbNumberEdit.EditingChange
 0001:0001F4CC       ovcdbnum.TOvcCustomDbNumberEdit.GetButtonEnabled
 0001:0001F500       ovcdbnum.TOvcCustomDbNumberEdit.GetDataField
 0001:0001F51C       ovcdbnum.TOvcCustomDbNumberEdit.GetDataSource
 0001:0001F528       ovcdbnum.TOvcCustomDbNumberEdit.GetField
 0001:0001F534       ovcdbnum.TOvcCustomDbNumberEdit.GetReadOnly
 0001:0001F560       ovcdbnum.TOvcCustomDbNumberEdit.GetTextMargins
 0001:0001F628       ovcdbnum.TOvcCustomDbNumberEdit.KeyDown
 0001:0001F660       ovcdbnum.TOvcCustomDbNumberEdit.KeyPress
 0001:0001F710       ovcdbnum.TOvcCustomDbNumberEdit.Notification
 0001:0001F74C       ovcdbnum.TOvcCustomDbNumberEdit.PopupClose
 0001:0001F77C       ovcdbnum.TOvcCustomDbNumberEdit.PopupOpen
 0001:0001F794       ovcdbnum.TOvcCustomDbNumberEdit.SetDataField
 0001:0001F82C       ovcdbnum.TOvcCustomDbNumberEdit.SetDataSource
 0001:0001F850       ovcdbnum.TOvcCustomDbNumberEdit.SetFocused
 0001:0001F884       ovcdbnum.TOvcCustomDbNumberEdit.SetReadOnly
 0001:0001F890       ovcdbnum.TOvcCustomDbNumberEdit.UpdateData
 0001:0001F8E4       ovcdbnum.TOvcCustomDbNumberEdit.WMCut
 0001:0001F904       ovcdbnum.TOvcCustomDbNumberEdit.WMPaint
 0001:0001FB80       ovcdbnum.TOvcCustomDbNumberEdit.WMPaste
 0001:0001FBA0       ovcdbnum.TOvcCustomDbNumberEdit.ExecuteAction
 0001:0001FBDC       ovcdbnum.TOvcCustomDbNumberEdit.UpdateAction
 0001:0001FC18       ovcdbnum.Finalization
 0001:0001FCFC       ovcdbplb..TOvcDbPictureLabel
 0001:00020378       ovcdbplb.TOvcDbPictureLabel.CMGetDataLink
 0001:00020384       ovcdbplb.TOvcDbPictureLabel.Create
 0001:000203F8       ovcdbplb.TOvcDbPictureLabel.Destroy
 0001:00020430       ovcdbplb.TOvcDbPictureLabel.GetDataField
 0001:0002044C       ovcdbplb.TOvcDbPictureLabel.GetDataSource
 0001:00020460       ovcdbplb.TOvcDbPictureLabel.GetField
 0001:0002046C       ovcdbplb.TOvcDbPictureLabel.Notification
 0001:000204A8       ovcdbplb.TOvcDbPictureLabel.Paint
 0001:000205CC       ovcdbplb.TOvcDbPictureLabel.plDataChange
 0001:000205D4       ovcdbplb.TOvcDbPictureLabel.plGetFieldValue
 0001:00020794       ovcdbplb.TOvcDbPictureLabel.plGetSampleDisplayData
 0001:000207CC       ovcdbplb.TOvcDbPictureLabel.SetDataField
 0001:00020820       ovcdbplb.TOvcDbPictureLabel.SetDataSource
 0001:00020844       ovcdbplb.TOvcDbPictureLabel.SetShowDateOrTime
 0001:00020868       ovcdbplb.TOvcDbPictureLabel.ExecuteAction
 0001:000208A4       ovcdbplb.TOvcDbPictureLabel.UpdateAction
 0001:000208E0       ovcdbplb.Finalization
 0001:00020CB8       ovcdbrpv..TOvcDbRvDataLink
 0001:00020D98       ovcdbrpv..TOvcDbRvField
 0001:00020F70       ovcdbrpv..TOvcDbReportView
 0001:00021AD8       ovcdbrpv..TOvcDbRVListBox
 0001:00021C78       ovcdbrpv.TOvcDbRvDataLink.Create
 0001:00021CB4       ovcdbrpv.TOvcDbRvDataLink.ActiveChanged
 0001:00021CC0       ovcdbrpv.TOvcDbRvDataLink.UpdateData
 0001:00021CCC       ovcdbrpv.TOvcDbRvDataLink.DataSetChanged
 0001:00021CD8       ovcdbrpv.TOvcDbRvDataLink.DataSetScrolled
 0001:00021CE4       ovcdbrpv.TOvcDbRvDataLink.RecordChanged
 0001:00021CE8       ovcdbrpv.TOvcDbRvDataLink.LayoutChanged
 0001:00021D00       ovcdbrpv.TOvcDbReportView.ActiveChanged
 0001:00021D48       ovcdbrpv.TOvcDbReportView.AssignStructure
 0001:00021E30       ovcdbrpv.TOvcDbReportView.BindViews
 0001:00021F18       ovcdbrpv.TOvcDbReportView.ClearTableFields
 0001:00021F58       ovcdbrpv.TOvcDbReportView.BuildFieldTable
 0001:0002230C       ovcdbrpv.TOvcDbReportView.ClearAll
 0001:00022378       ovcdbrpv.TOvcDbReportView.ClearBindings
 0001:000223E4       ovcdbrpv.TOvcDbReportView.ClearDataList
 0001:000223F0       ovcdbrpv.TOvcDbReportView.MoveDataPointer
 0001:00022440       ovcdbrpv.TOvcDbReportView.UpdateCurrentSelection
 0001:000224A0       ovcdbrpv.TOvcDbReportView.Click
 0001:000224D0       ovcdbrpv.TOvcDbReportView.Create
 0001:000225E4       ovcdbrpv.TOvcDbReportView.CreateValidFieldName
 0001:00022708       ovcdbrpv.TOvcDbReportView.Destroy
 0001:0002278C       ovcdbrpv.TOvcDbReportView.DblClick
 0001:000227BC       ovcdbrpv.TOvcDbReportView.DoBusy
 0001:00022810       ovcdbrpv.TOvcDbReportView.DoCompareFields
 0001:00022B8C       ovcdbrpv.TOvcDbReportView.DoEnumEvent
 0001:00022BC8       ovcdbrpv.TOvcDbReportView.DoGetFieldAsFloat
 0001:00022C50       ovcdbrpv.TOvcDbReportView.DoGetFieldAsString
 0001:00022CDC       ovcdbrpv.TOvcDbReportView.DoGetFieldValue
 0001:00022D3C       ovcdbrpv.TOvcDbReportView.DoGetGroupString
 0001:00022E84       ovcdbrpv.TOvcDbReportView.DoKeySearch
 0001:00022F14       ovcdbrpv.TOvcDbReportView.Enumerate
 0001:00022F3C       ovcdbrpv.TOvcDbReportView.EnumerateSelected
 0001:00022FA8       ovcdbrpv.TOvcDbReportView.EnumerateEx
 0001:0002301C       ovcdbrpv.TOvcDbReportView.GetDataSource
 0001:00023030       ovcdbrpv.TOvcDbReportView.GetFieldClassType
 0001:00023038       ovcdbrpv.TOvcDbReportView.InternalRecordCount
 0001:00023144       ovcdbrpv.TOvcDbReportView.RecordChanged
 0001:0002314C       ovcdbrpv.TOvcDbReportView.ReloadData
 0001:000232D0       ovcdbrpv.TOvcDbReportView.SetDataSource
 0001:0002331C       ovcdbrpv.TOvcDbReportView.SetName
 0001:00023500       ovcdbrpv.TOvcDbReportView.ExecuteAction
 0001:0002353C       ovcdbrpv.TOvcDbReportView.UpdateAction
 0001:00023578       ovcdbrpv.TOvcDbReportView.DataSetChanged
 0001:000235B0       ovcdbrpv.TOvcDbReportView.DataSetScrolled
 0001:000235E0       ovcdbrpv.TOvcDbReportView.Loaded
 0001:000235F4       ovcdbrpv.TOvcDbReportView.Notification
 0001:0002368C       ovcdbrpv.TOvcDbReportView.DoDrawViewField
 0001:000236F4       ovcdbrpv.TOvcDbReportView.CreateListBox
 0001:00023704       ovcdbrpv.TOvcDbRVListBox.Paint
 0001:00023748       ovcdbrpv.TOvcDbReportView.DoDetail
 0001:00023764       ovcdbrpv.Finalization
 0001:0002389C       ovcdbsed..TOvcCustomDbSliderEdit
 0001:00023A84       ovcdbsed..TOvcDbSliderEdit
 0001:000243A0       ovcdbsed.TOvcCustomDbSliderEdit.Change
 0001:000243B8       ovcdbsed.TOvcCustomDbSliderEdit.CMEnter
 0001:000243D4       ovcdbsed.TOvcCustomDbSliderEdit.CMExit
 0001:0002445C       ovcdbsed.TOvcCustomDbSliderEdit.CMGetDataLink
 0001:00024468       ovcdbsed.TOvcCustomDbSliderEdit.Create
 0001:000244FC       ovcdbsed.TOvcCustomDbSliderEdit.DataChange
 0001:000246B4       ovcdbsed.TOvcCustomDbSliderEdit.Destroy
 0001:00024700       ovcdbsed.TOvcCustomDbSliderEdit.EditingChange
 0001:00024734       ovcdbsed.TOvcCustomDbSliderEdit.GetButtonEnabled
 0001:00024768       ovcdbsed.TOvcCustomDbSliderEdit.GetDataField
 0001:00024784       ovcdbsed.TOvcCustomDbSliderEdit.GetDataSource
 0001:00024790       ovcdbsed.TOvcCustomDbSliderEdit.GetField
 0001:0002479C       ovcdbsed.TOvcCustomDbSliderEdit.GetReadOnly
 0001:000247C8       ovcdbsed.TOvcCustomDbSliderEdit.GetTextMargins
 0001:00024890       ovcdbsed.TOvcCustomDbSliderEdit.KeyDown
 0001:000248C8       ovcdbsed.TOvcCustomDbSliderEdit.KeyPress
 0001:00024978       ovcdbsed.TOvcCustomDbSliderEdit.Notification
 0001:000249B4       ovcdbsed.TOvcCustomDbSliderEdit.PopupClose
 0001:000249E4       ovcdbsed.TOvcCustomDbSliderEdit.PopupOpen
 0001:000249FC       ovcdbsed.TOvcCustomDbSliderEdit.SetDataField
 0001:00024A94       ovcdbsed.TOvcCustomDbSliderEdit.SetDataSource
 0001:00024AB8       ovcdbsed.TOvcCustomDbSliderEdit.SetFocused
 0001:00024AEC       ovcdbsed.TOvcCustomDbSliderEdit.SetReadOnly
 0001:00024AF8       ovcdbsed.TOvcCustomDbSliderEdit.UpdateData
 0001:00024B98       ovcdbsed.TOvcCustomDbSliderEdit.WMCut
 0001:00024BB8       ovcdbsed.TOvcCustomDbSliderEdit.WMPaint
 0001:00024E34       ovcdbsed.TOvcCustomDbSliderEdit.WMPaste
 0001:00024E54       ovcdbsed.TOvcCustomDbSliderEdit.ExecuteAction
 0001:00024E90       ovcdbsed.TOvcCustomDbSliderEdit.UpdateAction
 0001:00024ECC       ovcdbsed.Finalization
 0001:00024EFC       ovcdbsld..TOvcDbSlider
 0001:0002562C       ovcdbsld.TOvcDbSlider.CMExit
 0001:00025690       ovcdbsld.TOvcDbSlider.CMGetDataLink
 0001:0002569C       ovcdbsld.TOvcDbSlider.Create
 0001:00025710       ovcdbsld.TOvcDbSlider.Destroy
 0001:00025748       ovcdbsld.TOvcDbSlider.DoOnChange
 0001:00025760       ovcdbsld.TOvcDbSlider.GetDataField
 0001:0002577C       ovcdbsld.TOvcDbSlider.GetDataSource
 0001:00025790       ovcdbsld.TOvcDbSlider.GetField
 0001:0002579C       ovcdbsld.TOvcDbSlider.Notification
 0001:000257E0       ovcdbsld.TOvcDbSlider.SetDataField
 0001:00025954       ovcdbsld.TOvcDbSlider.SetDataSource
 0001:00025980       ovcdbsld.TOvcDbSlider.slDataChange
 0001:000259C0       ovcdbsld.TOvcDbSlider.slUpdateData
 0001:000259F8       ovcdbsld.TOvcDbSlider.WMLButtonDown
 0001:00025A3C       ovcdbsld.TOvcDbSlider.WMKeyDown
 0001:00025A80       ovcdbsld.TOvcDbSlider.ExecuteAction
 0001:00025ABC       ovcdbsld.TOvcDbSlider.UpdateAction
 0001:00025AF8       ovcdbsld.Finalization
 0001:00025EAC       ovcdbtbl..TOvcDbTableDataLink
 0001:00025F90       ovcdbtbl..TOvcDbTableColumn
 0001:00026088       ovcdbtbl..TOvcVisibleColumns
 0001:00026174       ovcdbtbl..TOvcCustomDbTable
 0001:00026400       ovcdbtbl..TOvcDbTable
 0001:00026E50       ovcdbtbl.TOvcDbTableDataLink.ActiveChanged
 0001:00026E60       ovcdbtbl.TOvcDbTableDataLink.AddMapping
 0001:00026FA8       ovcdbtbl.TOvcDbTableDataLink.ClearFieldMappings
 0001:00026FD4       ovcdbtbl.TOvcDbTableDataLink.Create
 0001:00027010       ovcdbtbl.TOvcDbTableDataLink.Destroy
 0001:0002703C       ovcdbtbl.TOvcDbTableDataLink.GetDefaultFields
 0001:00027060       ovcdbtbl.TOvcDbTableDataLink.GetFields
 0001:000270E0       ovcdbtbl.TOvcDbTableDataLink.DataSetChanged
 0001:000270F4       ovcdbtbl.TOvcDbTableDataLink.DataSetScrolled
 0001:00027100       ovcdbtbl.TOvcDbTableDataLink.EditingChanged
 0001:0002710C       ovcdbtbl.TOvcDbTableDataLink.LayoutChanged
 0001:00027118       ovcdbtbl.TOvcDbTableDataLink.Modified
 0001:00027120       ovcdbtbl.TOvcDbTableDataLink.RecordChanged
 0001:0002713C       ovcdbtbl.TOvcDbTableDataLink.Reset
 0001:00027164       ovcdbtbl.TOvcDbTableDataLink.UpdateData
 0001:000271BC       ovcdbtbl.TOvcDbTableColumn.Assign
 0001:000271F8       ovcdbtbl.TOvcDbTableColumn.Create
 0001:00027234       ovcdbtbl.TOvcDbTableColumn.GetField
 0001:000272EC       ovcdbtbl.TOvcDbTableColumn.GetTable
 0001:000272F0       ovcdbtbl.TOvcDbTableColumn.SetDataField
 0001:000273A4       ovcdbtbl.TOvcDbTableColumn.SetDateOrTime
 0001:000273E8       ovcdbtbl.TOvcDbTableColumn.SetField
 0001:00027408       ovcdbtbl.TOvcVisibleColumns.Add
 0001:00027418       ovcdbtbl.TOvcVisibleColumns.Clear
 0001:00027424       ovcdbtbl.TOvcVisibleColumns.Create
 0001:00027470       ovcdbtbl.TOvcVisibleColumns.Delete
 0001:0002747C       ovcdbtbl.TOvcVisibleColumns.Destroy
 0001:000274B8       ovcdbtbl.TOvcVisibleColumns.Exchange
 0001:000274C4       ovcdbtbl.TOvcVisibleColumns.IndexOf
 0001:000274F8       ovcdbtbl.TOvcVisibleColumns.GetColumn
 0001:0002751C       ovcdbtbl.TOvcVisibleColumns.GetCount
 0001:00027524       ovcdbtbl.TOvcVisibleColumns.Insert
 0001:00027544       ovcdbtbl.TOvcVisibleColumns.Move
 0001:00027578       ovcdbtbl.TOvcCustomDbTable.CalcRowCol
 0001:000277A0       ovcdbtbl.TOvcCustomDbTable.ChangeScale
 0001:00027810       ovcdbtbl.TOvcCustomDbTable.CMColorChanged
 0001:00027824       ovcdbtbl.TOvcCustomDbTable.CMCtl3DChanged
 0001:00027864       ovcdbtbl.TOvcCustomDbTable.CMDesignHitTest
 0001:000278D0       ovcdbtbl.TOvcCustomDbTable.CMFontChanged
 0001:000278F4       ovcdbtbl.TOvcCustomDbTable.Create
 0001:00027CCC       ovcdbtbl.TOvcCustomDbTable.CreateParams
 0001:00027D30       ovcdbtbl.TOvcCustomDbTable.CreateWnd
 0001:00027DE4       ovcdbtbl.TOvcCustomDbTable.ctimKillFocus
 0001:00027E44       ovcdbtbl.TOvcCustomDbTable.ctimQueryOptions
 0001:00027EB0       ovcdbtbl.TOvcCustomDbTable.ctimQueryColor
 0001:00027EB8       ovcdbtbl.TOvcCustomDbTable.ctimQueryFont
 0001:00027EC0       ovcdbtbl.TOvcCustomDbTable.ctimQueryLockedCols
 0001:00027ECC       ovcdbtbl.TOvcCustomDbTable.ctimQueryLockedRows
 0001:00027ED4       ovcdbtbl.TOvcCustomDbTable.ctimQueryActiveCol
 0001:00027EE0       ovcdbtbl.TOvcCustomDbTable.ctimQueryActiveRow
 0001:00027EEC       ovcdbtbl.TOvcCustomDbTable.ctimRemoveCell
 0001:00027F04       ovcdbtbl.TOvcCustomDbTable.ctimSetFocus
 0001:00027F14       ovcdbtbl.TOvcCustomDbTable.ctimStartEdit
 0001:00027F38       ovcdbtbl.TOvcCustomDbTable.ctimStartEditMouse
 0001:00027FF4       ovcdbtbl.TOvcCustomDbTable.ctimStartEditKey
 0001:0002804C       ovcdbtbl.TOvcCustomDbTable.DefineProperties
 0001:00028088       ovcdbtbl.TOvcCustomDbTable.Destroy
 0001:00028158       ovcdbtbl.TOvcCustomDbTable.DoOnActiveCellChanged
 0001:000281A0       ovcdbtbl.TOvcCustomDbTable.DoOnColumnMoved
 0001:000281E8       ovcdbtbl.TOvcCustomDbTable.DoOnGetCellAttributes
 0001:0002823C       ovcdbtbl.TOvcCustomDbTable.DoOnIndicatorClick
 0001:00028264       ovcdbtbl.TOvcCustomDbTable.DoOnLeftColumnChanged
 0001:000282A0       ovcdbtbl.TOvcCustomDbTable.DoOnLockedCellClick
 0001:000282E8       ovcdbtbl.TOvcCustomDbTable.DoOnMouseWheel
 0001:00028330       ovcdbtbl.TOvcCustomDbTable.DoOnPaintUnusedArea
 0001:00028378       ovcdbtbl.TOvcCustomDbTable.DoOnUnusedAreaClick
 0001:000283C0       ovcdbtbl.TOvcCustomDbTable.DoOnUserCommand
 0001:00028404       ovcdbtbl.TOvcCustomDbTable.FilterKey
 0001:000284D4       ovcdbtbl.TOvcCustomDbTable.GetColumnCount
 0001:000284E0       ovcdbtbl.TOvcCustomDbTable.GetColumnOrderStrings
 0001:0002851C       ovcdbtbl.TOvcCustomDbTable.GetColumnOrder
 0001:00028570       ovcdbtbl.TOvcCustomDbTable.GetColumnWidthsStrings
 0001:000285F0       ovcdbtbl.TOvcCustomDbTable.GetColumnWidths
 0001:0002863C       ovcdbtbl.TOvcCustomDbTable.GetDataSource
 0001:00028650       ovcdbtbl.TOvcCustomDbTable.GetFieldCount
 0001:0002865C       ovcdbtbl.TOvcCustomDbTable.GetFields
 0001:00028668       ovcdbtbl.TOvcCustomDbTable.GetSelectedField
 0001:0002868C       ovcdbtbl.TOvcCustomDbTable.GetVisibleColumnCount
 0001:00028698       ovcdbtbl.TOvcCustomDbTable.IncCol
 0001:00028730       ovcdbtbl.TOvcCustomDbTable.IncRow
 0001:00028750       ovcdbtbl.TOvcCustomDbTable.InEditingState
 0001:0002875C       ovcdbtbl.TOvcCustomDbTable.InvalidateCell
 0001:000287A4       ovcdbtbl.TOvcCustomDbTable.InvalidateColumn
 0001:000287D4       ovcdbtbl.TOvcCustomDbTable.InvalidateHeader
 0001:00028828       ovcdbtbl.TOvcCustomDbTable.InvalidateIndicators
 0001:00028878       ovcdbtbl.TOvcCustomDbTable.InvalidateNotLocked
 0001:000288F8       ovcdbtbl.TOvcCustomDbTable.InvalidateRow
 0001:00028934       ovcdbtbl.TOvcCustomDbTable.InvalidateUnusedArea
 0001:000289B8       ovcdbtbl.TOvcCustomDbTable.Loaded
 0001:00028A2C       ovcdbtbl.TOvcCustomDbTable.MakeColumnVisible
 0001:00028B14       ovcdbtbl.TOvcCustomDbTable.MoveActiveCell
 0001:00028E34       ovcdbtbl.TOvcCustomDbTable.Notification
 0001:00028FA8       ovcdbtbl.DrawEffects
 0001:000290A4       ovcdbtbl.PaintString
 0001:0002914C       ovcdbtbl.TOvcCustomDbTable.Paint
 0001:0002A16C       ovcdbtbl.TOvcCustomDbTable.ResolveCellAttributes
 0001:0002A2C8       ovcdbtbl.TOvcCustomDbTable.SaveEditedData
 0001:0002A3C0       ovcdbtbl.TOvcCustomDbTable.Scroll
 0001:0002A3E8       ovcdbtbl.TOvcCustomDbTable.SetAccess
 0001:0002A420       ovcdbtbl.TOvcCustomDbTable.SetActiveCell
 0001:0002A5E8       ovcdbtbl.TOvcCustomDbTable.SetActiveColumn
 0001:0002A5F8       ovcdbtbl.TOvcCustomDbTable.SetActiveRow
 0001:0002A604       ovcdbtbl.TOvcCustomDbTable.SetAdjust
 0001:0002A630       ovcdbtbl.TOvcCustomDbTable.SetBorderStyle
 0001:0002A644       ovcdbtbl.TOvcCustomDbTable.SetBounds
 0001:0002A6E0       ovcdbtbl.TOvcCustomDbTable.SetCellProperties
 0001:0002ABF8       ovcdbtbl.TOvcCustomDbTable.SetColumnCount
 0001:0002AC2C       ovcdbtbl.TOvcCustomDbTable.SetColumnOrderStrings
 0001:0002AD88       ovcdbtbl.TOvcCustomDbTable.SetColumnOrder
 0001:0002AE80       ovcdbtbl.TOvcCustomDbTable.SetColumnWidthsStrings
 0001:0002AF44       ovcdbtbl.TOvcCustomDbTable.SetColumnWidths
 0001:0002AF9C       ovcdbtbl.TOvcCustomDbTable.SetColors
 0001:0002AFAC       ovcdbtbl.TOvcCustomDbTable.SetColorUnused
 0001:0002AFC4       ovcdbtbl.TOvcCustomDbTable.SetColumns
 0001:0002AFE4       ovcdbtbl.TOvcCustomDbTable.SetDataSource
 0001:0002B0D0       ovcdbtbl.TOvcCustomDbTable.SetDefaultMargin
 0001:0002B0EC       ovcdbtbl.TOvcCustomDbTable.SetLinkActive
 0001:0002B1DC       ovcdbtbl.TOvcCustomDbTable.SetHeaderCell
 0001:0002B328       ovcdbtbl.TOvcCustomDbTable.SetHeaderHeight
 0001:0002B38C       ovcdbtbl.TOvcCustomDbTable.SetHeaderOptions
 0001:0002B4EC       ovcdbtbl.TOvcCustomDbTable.SetLeftColumn
 0001:0002B534       ovcdbtbl.TOvcCustomDbTable.SetLockedColumns
 0001:0002B5CC       ovcdbtbl.TOvcCustomDbTable.SetOptions
 0001:0002B788       ovcdbtbl.TOvcCustomDbTable.SetRowHeight
 0001:0002B7D4       ovcdbtbl.TOvcCustomDbTable.SetRowIndicatorWidth
 0001:0002B860       ovcdbtbl.TOvcCustomDbTable.SetScrollBars
 0001:0002B874       ovcdbtbl.TOvcCustomDbTable.SetSelectedField
 0001:0002B8B0       ovcdbtbl.TOvcCustomDbTable.SetTextStyle
 0001:0002B8C8       ovcdbtbl.TOvcCustomDbTable.StartEditing
 0001:0002BC5C       ovcdbtbl.TOvcCustomDbTable.StopEditing
 0001:0002BE38       ovcdbtbl.TOvcCustomDbTable.tbAdjustIntegralHeight
 0001:0002BEA0       ovcdbtbl.TOvcCustomDbTable.tbCalcActiveCellRect
 0001:0002BF20       ovcdbtbl.TOvcCustomDbTable.tbCalcCellRect
 0001:0002BFBC       ovcdbtbl.TOvcCustomDbTable.tbCalcColumnRect
 0001:0002C038       ovcdbtbl.TOvcCustomDbTable.tbCalcColumnsOnLastPage
 0001:0002C0E0       ovcdbtbl.TOvcCustomDbTable.tbCalcRowColData
 0001:0002C204       ovcdbtbl.TOvcCustomDbTable.tbCalcRowRect
 0001:0002C240       ovcdbtbl.TOvcCustomDbTable.tbCalcRowTop
 0001:0002C26C       ovcdbtbl.TOvcCustomDbTable.tbCalcRowBottom
 0001:0002C284       ovcdbtbl.TOvcCustomDbTable.tbCalcVisibleRows
 0001:0002C2C8       ovcdbtbl.TOvcCustomDbTable.tbCanModify
 0001:0002C458       ovcdbtbl.TOvcCustomDbTable.tbCellChanged
 0001:0002C488       ovcdbtbl.TOvcCustomDbTable.tbCellModified
 0001:0002C534       ovcdbtbl.TOvcCustomDbTable.tbColorsChanged
 0001:0002C564       ovcdbtbl.TOvcCustomDbTable.tbColumnAtRight
 0001:0002C588       ovcdbtbl.TOvcCustomDbTable.tbColumnChanged
 0001:0002C854       ovcdbtbl.TOvcCustomDbTable.tbDataChanged
 0001:0002C8DC       ovcdbtbl.TOvcCustomDbTable.tbDefineFieldMap
 0001:0002C9FC       ovcdbtbl.TOvcCustomDbTable.tbDrawActiveCell
 0001:0002CEBC       ovcdbtbl.TOvcCustomDbTable.tbDrawMoveLine
 0001:0002D00C       ovcdbtbl.TOvcCustomDbTable.tbDrawSizeLine
 0001:0002D0E4       ovcdbtbl.TOvcCustomDbTable.tbDrawUnusedArea
 0001:0002D1D4       ovcdbtbl.TOvcCustomDbTable.tbEditCellHasFocus
 0001:0002D240       ovcdbtbl.TOvcCustomDbTable.tbEditingChanged
 0001:0002D2B4       ovcdbtbl.TOvcCustomDbTable.tbFindCell
 0001:0002D2E4       ovcdbtbl.TOvcCustomDbTable.tbGetDataSize
 0001:0002D3E8       ovcdbtbl.TOvcCustomDbTable.tbGetFieldColumn
 0001:0002D428       ovcdbtbl.TOvcCustomDbTable.tbGetFieldValue
 0001:0002D924       ovcdbtbl.TOvcCustomDbTable.tbGridPenChanged
 0001:0002D954       ovcdbtbl.TOvcCustomDbTable.tbIsOnGridLine
 0001:0002D9F0       ovcdbtbl.TOvcCustomDbTable.tbIsDbActive
 0001:0002DA1C       ovcdbtbl.TOvcCustomDbTable.tbIsColumnHidden
 0001:0002DA84       ovcdbtbl.TOvcCustomDbTable.tbIsInMoveArea
 0001:0002DB10       ovcdbtbl.TOvcCustomDbTable.tbLayoutChanged
 0001:0002DBC0       ovcdbtbl.TOvcCustomDbTable.tbIsSibling
 0001:0002DC0C       ovcdbtbl.TOvcCustomDbTable.tbLoading
 0001:0002DC44       ovcdbtbl.TOvcCustomDbTable.tbMoveActCellPageLeft
 0001:0002DD10       ovcdbtbl.TOvcCustomDbTable.tbMoveActCellPageRight
 0001:0002DDE4       ovcdbtbl.TOvcCustomDbTable.tbPaintBitmapCell
 0001:0002E048       ovcdbtbl.TOvcCustomDbTable.tbPaintString
 0001:0002E35C       ovcdbtbl.TOvcCustomDbTable.tbQueryColData
 0001:0002E3E4       ovcdbtbl.TOvcCustomDbTable.tbReadColData
 0001:0002E4FC       ovcdbtbl.TOvcCustomDbTable.tbRecordChanged
 0001:0002E5AC       ovcdbtbl.GetColumnWidth
 0001:0002E73C       ovcdbtbl.TOvcCustomDbTable.tbRebuildColumns
 0001:0002E8B4       ovcdbtbl.TOvcCustomDbTable.tbScrollBarPageLeft
 0001:0002E948       ovcdbtbl.TOvcCustomDbTable.tbScrollBarPageRight
 0001:0002E998       ovcdbtbl.TOvcCustomDbTable.tbScrollNotification
 0001:0002EB28       ovcdbtbl.TOvcCustomDbTable.tbScrollTableLeft
 0001:0002EC60       ovcdbtbl.TOvcCustomDbTable.tbScrollTableRight
 0001:0002ED28       ovcdbtbl.TOvcCustomDbTable.tbSetFieldValue
 0001:0002F2F4       ovcdbtbl.TOvcCustomDbTable.tbSetFocus
 0001:0002F300       ovcdbtbl.TOvcCustomDbTable.tbUpdateActive
 0001:0002F324       ovcdbtbl.TOvcCustomDbTable.tbUpdateBufferLimit
 0001:0002F3EC       ovcdbtbl.TOvcCustomDbTable.tbUpdateHScrollBar
 0001:0002F480       ovcdbtbl.TOvcCustomDbTable.tbUpdateVScrollBar
 0001:0002F5EC       ovcdbtbl.TOvcCustomDbTable.tbWriteColData
 0001:0002F684       ovcdbtbl.TOvcCustomDbTable.UpdateData
 0001:0002F69C       ovcdbtbl.TOvcCustomDbTable.WMCommand
 0001:0002F7E0       ovcdbtbl.TOvcCustomDbTable.WMEraseBkGnd
 0001:0002F7E8       ovcdbtbl.TOvcCustomDbTable.WMGetDlgCode
 0001:0002F80C       ovcdbtbl.TOvcCustomDbTable.WMHScroll
 0001:0002F930       ovcdbtbl.TOvcCustomDbTable.WMKeyDown
 0001:0002FB54       ovcdbtbl.TOvcCustomDbTable.WMKillFocus
 0001:0002FB7C       ovcdbtbl.TOvcCustomDbTable.WMLButtonDblClk
 0001:0002FC18       ovcdbtbl.TOvcCustomDbTable.WMLButtonDown
 0001:00030014       ovcdbtbl.TOvcCustomDbTable.WMLButtonUp
 0001:000302A8       ovcdbtbl.TOvcCustomDbTable.WMMouseMove
 0001:0003036C       ovcdbtbl.TOvcCustomDbTable.WMNCHitTest
 0001:00030388       ovcdbtbl.TOvcCustomDbTable.WMSetCursor
 0001:00030534       ovcdbtbl.TOvcCustomDbTable.WMSetFocus
 0001:000305DC       ovcdbtbl.TOvcCustomDbTable.WMSize
 0001:000305F0       ovcdbtbl.TOvcCustomDbTable.WMVScroll
 0001:00030858       ovcdbtbl.Finalization
 0001:000308C0       ovcdbtim..TOvcCustomDbTimeEdit
 0001:00030A90       ovcdbtim..TOvcDbTimeEdit
 0001:000314CC       ovcdbtim.TOvcCustomDbTimeEdit.Change
 0001:000314E4       ovcdbtim.TOvcCustomDbTimeEdit.CMEnter
 0001:00031500       ovcdbtim.TOvcCustomDbTimeEdit.CMExit
 0001:00031588       ovcdbtim.TOvcCustomDbTimeEdit.CMGetDataLink
 0001:00031594       ovcdbtim.TOvcCustomDbTimeEdit.Create
 0001:00031628       ovcdbtim.TOvcCustomDbTimeEdit.DataChange
 0001:00031854       ovcdbtim.TOvcCustomDbTimeEdit.Destroy
 0001:000318A0       ovcdbtim.TOvcCustomDbTimeEdit.EditingChange
 0001:000318B4       ovcdbtim.TOvcCustomDbTimeEdit.GetDataField
 0001:000318D0       ovcdbtim.TOvcCustomDbTimeEdit.GetDataSource
 0001:000318DC       ovcdbtim.TOvcCustomDbTimeEdit.GetField
 0001:000318E8       ovcdbtim.TOvcCustomDbTimeEdit.GetReadOnly
 0001:00031928       ovcdbtim.TOvcCustomDbTimeEdit.GetTextMargins
 0001:000319F0       ovcdbtim.TOvcCustomDbTimeEdit.KeyDown
 0001:00031A28       ovcdbtim.TOvcCustomDbTimeEdit.KeyPress
 0001:00031ABC       ovcdbtim.TOvcCustomDbTimeEdit.Notification
 0001:00031AF8       ovcdbtim.TOvcCustomDbTimeEdit.SetDataField
 0001:00031B90       ovcdbtim.TOvcCustomDbTimeEdit.SetDataSource
 0001:00031BB4       ovcdbtim.TOvcCustomDbTimeEdit.SetFocused
 0001:00031BE8       ovcdbtim.TOvcCustomDbTimeEdit.SetReadOnly
 0001:00031BF4       ovcdbtim.TOvcCustomDbTimeEdit.UpdateData
 0001:00031DD4       ovcdbtim.TOvcCustomDbTimeEdit.WMCut
 0001:00031DF4       ovcdbtim.TOvcCustomDbTimeEdit.WMPaint
 0001:00032060       ovcdbtim.TOvcCustomDbTimeEdit.WMPaste
 0001:00032080       ovcdbtim.TOvcCustomDbTimeEdit.ExecuteAction
 0001:000320BC       ovcdbtim.TOvcCustomDbTimeEdit.UpdateAction
 0001:000320F8       ovcdbtim.Finalization
 0001:00032230       o32dbfe..TO32DbFlexEdit
 0001:00032E20       o32dbfe.TO32DbFlexEdit.CMEnter
 0001:00032E3C       o32dbfe.TO32DbFlexEdit.CMExit
 0001:00032E44       o32dbfe.TO32DbFlexEdit.CMGetDataLink
 0001:00032E50       o32dbfe.TO32DbFlexEdit.Create
 0001:00032EE8       o32dbfe.TO32DbFlexEdit.Destroy
 0001:00032F34       o32dbfe.TO32DbFlexEdit.CreateWnd
 0001:00032F64       o32dbfe.TO32DbFlexEdit.CutToClipboard
 0001:00032FE4       o32dbfe.TO32DbFlexEdit.PasteFromClipboard
 0001:00033064       o32dbfe.TO32DbFlexEdit.DoOnChange
 0001:00033084       o32dbfe.TO32DbFlexEdit.GetDataField
 0001:000330A0       o32dbfe.TO32DbFlexEdit.GetDataSource
 0001:000330B4       o32dbfe.TO32DbFlexEdit.GetField
 0001:00033134       o32dbfe.TO32DbFlexEdit.Notification
 0001:0003317C       o32dbfe.TO32DbFlexEdit.Restore
 0001:0003319C       o32dbfe.TO32DbFlexEdit.SetDataField
 0001:00033254       o32dbfe.TO32DbFlexEdit.SetDataSource
 0001:00033288       o32dbfe.TO32DbFlexEdit.SetFieldType
 0001:00033328       o32dbfe.TO32DbFlexEdit.SetUseTFieldMask
 0001:00033340       o32dbfe.TO32DbFlexEdit.fedbDataChange
 0001:000333A8       o32dbfe.TO32DbFlexEdit.fedbEditingChange
 0001:000333CC       o32dbfe.TO32DbFlexEdit.fedbGetFieldValue
 0001:000336C8       o32dbfe.TO32DbFlexEdit.fedbSetFieldProperties
 0001:0003372C       o32dbfe.TO32DbFlexEdit.fedbSetFieldValue
 0001:00033B50       o32dbfe.TO32DbFlexEdit.fedbUpdateData
 0001:00033B98       o32dbfe.TO32DbFlexEdit.WMKeyDown
 0001:00033C00       o32dbfe.TO32DbFlexEdit.WMChar
 0001:00033C28       o32dbfe.TO32DbFlexEdit.WMKillFocus
 0001:00033C70       o32dbfe.TO32DbFlexEdit.WMLButtonDblClk
 0001:00033C84       o32dbfe.TO32DbFlexEdit.WMLButtonDown
 0001:00033C98       o32dbfe.TO32DbFlexEdit.WMLButtonUp
 0001:00033CBC       o32dbfe.TO32DbFlexEdit.WMPaint
 0001:00033FC8       o32dbfe.TO32DbFlexEdit.WMSetFocus
 0001:00033FF8       o32dbfe.TO32DbFlexEdit.ExecuteAction
 0001:00034034       o32dbfe.TO32DbFlexEdit.UpdateAction
 0001:00034070       o32dbfe.Finalization
 0001:00034708       .O406br2005.@GetPackageInfoTable
 0001:00034710       .O406br2005.@PackageLoad
 0001:0003471C       .O406br2005.@PackageUnload
 0002:00000008       Windows.Windows
 0002:0000013C       ovcdbhll.ovcdbhll
 0002:00000144       ovcdbtcb.ovcdbtcb
 0002:0000014C       ovcdbacb.ovcdbacb
 0002:0000015C       ovcdbadg.ovcdbadg
 0002:0000019C       ovcdbnf.ovcdbnf
 0002:000001A4       ovcdbpf.ovcdbpf
 0002:000001AC       ovcdbsf.ovcdbsf
 0002:000001B4       ovcdbae.ovcdbae
 0002:000001BC       ovcdbcal.ovcdbcal
 0002:000001C4       ovcdbccb.ovcdbccb
 0002:000001CC       ovcdbcl.ovcdbcl
 0002:000001D4       ovcdbclk.ovcdbclk
 0002:000001DC       ovcdbdat.ovcdbdat
 0002:000001E4       ovcdbdLb.ovcdbdLb
 0002:000001F4       ovcdbed.ovcdbed
 0002:000001FC       ovcdbfcb.ovcdbfcb
 0002:00000204       ovcdbidx.ovcdbidx
 0002:0000020C       ovcdbise.ovcdbise
 0002:00000214       ovcdbmdg.ovcdbmdg
 0002:0000021C       ovcdbnum.ovcdbnum
 0002:00000224       ovcdbplb.ovcdbplb
 0002:0000023C       ovcdbrpv.ovcdbrpv
 0002:00000244       ovcdbsed.ovcdbsed
 0002:0000024C       ovcdbsld.ovcdbsld
 0002:0000025C       ovcdbtbl.ovcdbtbl
 0002:00000264       ovcdbtim.ovcdbtim
 0002:0000028C       o32dbfe.o32dbfe
 0002:00000294       .O406br2005..O406br2005
 0003:00000000       SysInit.TlsIndex
 0003:00000004       SysInit.PtrToNil
 0003:00000008       SysInit.Module
 0003:00000020       SysInit.TlsProc
 0003:00000030       ovcdbnf.SupportedFieldTypes
 0003:00000038       ovcdbpf.SupportedFieldTypes
 0003:00000040       ovcdbsf.SupportedFieldTypes
 0003:00000048       ovcdbae.ScrollBar
 0003:00000050       ovcdbcal.SupportedFieldTypes
 0003:00000058       ovcdbccb.SupportedFieldTypes
 0003:00000060       ovcdbclk.SupportedFieldTypes
 0003:00000068       ovcdbdat.DateFieldTypes
 0003:00000070       ovcdbidx.DX
 0003:00000074       ovcdbidx.DY
 0003:00000078       ovcdbise.DX
 0003:0000007C       ovcdbise.DY
 0003:00000080       ovcdbnum.NumFieldTypes
 0003:00000088       ovcdbrpv.InReload
 0003:0000008C       ovcdbsed.SupportedFieldTypes
 0003:00000094       ovcdbsld.SupportedFieldTypes
 0003:0000009C       ovcdbtbl.SupportedFieldTypes
 0003:000000A4       ovcdbtim.TimeFieldTypes
 0003:000000AC       o32dbfe.SupportedFieldTypes
 0004:00000000       SysInit.ModuleIsLib
 0004:00000001       SysInit.ModuleIsPackage
 0004:00000004       SysInit.HInstance
 0004:00000008       SysInit.tlsBuffer
 0004:0000000C       Windows..3
 0004:00000010       Windows.HtmlHelpModule
 0004:00000014       ovcdbhll..2
 0004:00000018       ovcdbtcb..2
 0004:0000001C       ovcdbacb..2
 0004:00000020       ovcdbadg..3
 0004:00000024       ovcdbnf..2
 0004:00000028       ovcdbpf..2
 0004:0000002C       ovcdbsf..2
 0004:00000030       ovcdbae..8
 0004:00000034       ovcdbcal..2
 0004:00000038       ovcdbccb..2
 0004:0000003C       ovcdbcl..2
 0004:00000040       ovcdbclk..2
 0004:00000044       ovcdbdat..3
 0004:00000048       ovcdbdLb..2
 0004:0000004C       ovcdbed..2
 0004:00000050       ovcdbfcb..2
 0004:00000054       ovcdbidx..4
 0004:00000058       ovcdbise..2
 0004:0000005C       ovcdbmdg..3
 0004:00000060       ovcdbnum..3
 0004:00000064       ovcdbplb..2
 0004:00000068       ovcdbrpv..4
 0004:0000006C       ovcdbsed..3
 0004:00000070       ovcdbsld..2
 0004:00000074       ovcdbtbl..6
 0004:00000078       ovcdbtim..3
 0004:0000007C       o32dbfe..2
 0005:00000000       SysInit.TlsLast


Bound resource files

ovcdbadg.DFM
ovcdbmdg.DFM
O406br2005.res
O406br2005.drf


Program entry point at 0002:00000294
